:0900000C32322E312E302E323238
:1000000AF20D13F5392E14EF34404423FE2329014F
:1000000A412C30050E0F0C0F0E1210151611584CFC
:1000000A3E095E515B401836391B5B48373A202A55
:1000000A2D292E322D2D3135302D503254255B4A73
:1000000A4D334D51367654398276683369585B419F
:0500000A6B6F44696901
:020000040800F2
:40800000A8EB0020C1140908C9140908A9390908CD140908CF140908D114090800000000000000000000000000000000E1830008D51409080000000099840008FD840008D6
:40804000DB140908DB140908DB140908DB140908DB140908DB140908654901086F49010879490108834901088D490108DB140908DB140908DB14090845E60008DB140908D6
:40808000DB140908DB140908EF220108B3260108BD260108C7260108DB14090897490108DB140908DB140908DB140908DB140908DB140908DB140908DB140908DB140908F9
:4080C000DB140908E7440108F1440108DB140908DB140908DB140908DB1409084FE60008BD490108DB140908DB140908DB140908DB140908DB140908DB140908DB140908C2
:40810000DB140908DB140908DB140908DB140908DB140908DB140908F1490108EB5D0108CB220108E3220108D7220108DB140908DB140908DB140908DB140908D1260108A5
:40814000DB260108E5260108DB140908DB140908DB140908DB140908DB140908DB140908DB140908DB140908DB140908DB140908DB140908DB140908DB14090800000000E1
:40818000DB140908DB140908DB140908DB140908DB140908DB140908DB140908DB1409080000000000000000DB14090800F002F800F0C1F80AA090E8000C82448344AAF1D6
:4081C0000107DA4501D100F0B6F8AFF2090EBAE80F0013F0010F18BFFB1A43F00103184718520F0058520F0010F8013B0A4413F0030408BF10F8014B1D1108BF10F8015BA8
:40820000641E05D010F8016B641E01F8016BF9D1002D15D010F8014B03F00C030C2BA1EB04040ABF10F8013BA4EB8314A4EB032405F1010314F8016B5B1E01F8016BF9D588
:40824000914238BF10F8013BD1D370470023002400250026103A28BF78C1FBD8520728BF30C148BF0B6070476E290AF01189702909F0FF8B662913F01C8E652913F0198EB1
:40828000672913F0168E6129AFF3008003681B0A28BF41F08001692909F0708B642909F06D8B752909F06A8B6F290AF0FE89782909F0CB8BE9290AF09989E4290AF09689C5
:4082C000F5290AF09389EF290AF0FB89F82909F0CA8B0368DB0928BF41F0800163290AF01A8973290AF01F89E3290AF0358DF3290AF03A8D002070471FB593F0D0FD9DE8D1
:4083000003008AF00AF889F0A6FC8AF0A3FA0400002000218DF0CEFC401C6060002000218DF0DEFCE06089F0A3FF1FBD10B500208AF00AFA10BD8AF0ECFD1146FFF7DCFF5A
:408340000FB400F00BF80FBC03F053FC03F06AFD03B4FFF7EBFF03BC8AF0D4FD04B08CF09BF8044800218CF0C5F98CF0A7F803F059FD0000AC03002080F309887047EFF305
:4083800009807047684680F3098804480078C00714BF0220032080F314887047ACC00F08DFF818C0EFF305831B0618BF6047EFF31483DB0708BF604700DF7047C7470908A9
:4083C000DFF818C0EFF305831B0618BF6047EFF31483DB0708BF604700DF7047154A0908EFF30980816911F8021CE1BB90E80F1010B5E047BDE81040EFF3098C8CE8070074
:40840000214B93E80600914208BF704741B91EF0100F16D11D49086820F00100086010E01EF0100F06BF2CED108A0120002081F825002CE9F00FC1F828C00CB48CF03EFFFF
:408440000CBC1A60D2F828C0BCE8F00F92F8250000280EBF6FF0020E6FF0120EBCEC108A8CF30988704710B5094A1268914209D8084C54F8214090E80F10A047EFF3098C8E
:408480008CE80F0010BD0000C803002034EF00E0983909089839090810B58CF0D3FDBDE81040154B93E80600914208BF7047EFF3098C1EF0100F06BF2CED108A0120002025
:4084C00081F825002CE9F00FC1F828C00CB48CF0F5FE0CBC1A60D2F828C0BCE8F00F92F8250000280EBF6FF0020E6FF0120EBCEC108A8CF309887047C803002010B58CF09C
:40850000A5FFCCE710B58CF05DF98CF09FFFC6E70B49D1F800C04A685CF8043B1068184442F8040B8C4528BFA1F1DC0C8A4228BFA1F1DC02C1F800C04A6020F000407047C8
:4085400074E7002040BA7047C0BA70474FEA30007047000070472DE9F04F2DED028B85B0002004900390029030208BF07FFC054660F0E6F905462E46002002F069FEBCEE1B
:40858000C00A10EE107AAFF233023946304660F0A6FA002002F03BFEB0EE408AAFF24B01304660F0AFFA32460021FE4817F0D0FB03A9FD4800F085FF00285BD002A9FA4849
:4085C00000F087FF002855D000241C208BF04EFC0746DDE9022161F00BF90746B946B7EE000A484661F08EF964208BF03FFC80465FF024FD8046C246494650465FF011FFE5
:40860000204602F08DFD8346AFF2B702594650465FF056FE204602F0CDFDBCEEC00A10EE10BAAFF2CF02594650465FF036FE02F039FF012813DD02F0B9FA834602F032FF01
:40864000BBFBF0FB02F02EFF401E0BFB00FBAFF2FB0259465046CDF804B05FF08DFF52462146D04816F086F952462146304660F033FB00BF03A9CC4800F013FF002855D057
:4086800002A9C94800F015FF00284FD002241C208BF0ECFB0746DDE9022161F0A9F80746B946B7EE000A484661F02CF964208BF0DDFB80465FF0C2FC8046C246494650462B
:4086C0005FF0AFFE204602F02BFD8346AFF27B12594650465FF0F4FD204602F06BFDBCEEC00A10EE10BAAFF29312594650465FF0D4FD02F0D7FE01280DDD02F057FA834615
:4087000002F0D0FEBBFBF0F0AFF2B7120146019050465FF031FF52462146A24816F02AF952462146304660F0D7FA00BF049805B0BDEC028BBDE8F08F2DE9F84F01249B4914
:40874000984861F02FFC974816F045F90020009000BF0221944800F064FD934800F051FE02F008F9C0EB00108500AFF2172229468C4817F02CF802F00CF9C0EB00108500EF
:40878000AFF22F222946874816F0EFFF02F011F9C0EB00108500AFF243222946814816F0FDFF02F077F90546AFF2572229467D4816F0C2FF02F0C9F98246504689F0D4FAFE
:4087C000C5B2AFF26F232A465146764817F018F802F0D9F90546AFF283222946714817F03AF802F0F6F90546AFF2972229466D4817F04AF802F026FA08B1012000E000205E
:408800000546AFF2AF222946664817F056F802F006FA08B1012000E000200546AFF2CB222946604817F062F802F0E6F908B1012000E000200546AFF2E3222946594817F039
:408840006AF802F011FB0546AFF2F7222946554817F05EF902F01BFB0546AFF207322946504817F06EF902F014FD0546AFF21B3229464C4817F0B8F902F01EFD0546AFF297
:408880002B322946474817F0A8FA02F028FD0546AFF23F322946434817F0D1FA02F032FD0546AFF24F3229463E4817F0DDFA02F0ADFD0546AFF2633229463A4817F0A3FB60
:4088C00002F0B7FD0546AFF273322946354817F0B3FB02F0C1FD0546AFF287322946314817F0C3FB02F0DEFD0546AFF2973229462C4817F0F1FB02F059FA0546AFF2AB3238
:408900002946284817F0BBFC02F063FA0546AFF2BB322946234817F0CBFC02F06CFA0546AFF2CF3229461F4817F0DBFC02F076FA0546AFF2DF3229461A4817F0E7FC02F0C5
:4089400080FA0546AFF2F3322946164817F0F3FC02F065F901284FD102F087F90546AFF20B4229460F4816F0EFFF02F091F90546AFF21F4229460B4816F0FFFF02F09BF996
:408980000546AFF22F422946064817F00FF802F0A5F90546AFF243422946024817F01FF806E00000E0390010D403002035C0000802F0B0F90546AFF263422946DE4817F0EC
:4089C00027F802F0BAF90546AFF277422946DA4817F037F802F0C4F90546AFF287422946D54817F047F802F0CEF90546AFF29B422946D14817F05AF802F0FEF801281ED1AE
:408A00006946CE4800F06DFDC8B128208BF02EFA0646009961F026F80646B04620208BF025FA07465FF0E7F907463D46414628465FF0BEF92946C04815F003FF00BF02F0CD
:408A400001F9012859D100256946BC4800F059FD20B318208BF00AFA0646009960F066FF0646B0469FEDB60A404660F0D3FF2C208BF0FCF9074660F050FD07463D46414634
:408A8000284660F018FDAFF233520121284660F0E1FD2946A84815F034FE00BF6946A74800F027FD40B318208BF0E0F90646009960F03CFF0646B0469FEDA10A404660F0BA
:408AC000A9FFA8208BF0D2F9074660F0B8FA0746B9464146484660F075FA2946484660F06CFAAFF28F520021484660F061FB4946914815F067FE00BF00BF02F016FC054622
:408B0000AFF2AF5229468C4816F09DF902F032FC0546AFF2BF522946874816F057F902F04FFC0546AFF2D3522946834816F01CF902F00DFC0546AFF2E35229467E4816F009
:408B400069F902F02AFC0546AFF2F75229467A4816F023F902F047FC0546AFF207622946754816F0E8F8FFF7F6FC04402046BDE8F88F10B55DF07BFA02F021FA044655F076
:408B800035FF02F009FA044654F058FA02F0F1F9044655F09DF802F025FA044656F0C6FC02F07FFA044657F0FFFC02F02EFA04465EF002FD02F03CFA044652F001FD02F0FD
:408BC0004AFA04465DF0DCFE02F058FA044653F019FC02F079FA044651F07AFF02F08EFA044651F0F9F8FFF7A7FD00231A465549514861F080F90023022252494E48A03015
:408C000061F079F9002303224E494B48703061F072F9002304224B494748283061F06BF90023052247494448CC3061F064F9002306224449444861F05EF900230722414938
:408C40004148303061F057F9002308223D493E486C3061F050F9002309223A493A48A03061F049F900230A2236493748D43061F042F900230B223349344861F03CF93448FE
:408C8000006830B100230C222E493148006861F032F92F48006830B100230C2229492C48006861F028F9244817F06EFA224817F0D8FA0BF03EFD05F0F6F910BD08B5FFF7BD
:408CC00058FF01F0C1FE10B1012801D114E000BF002001F0D0FE00F0A2FC6FF07F4000F039F8684600F092FC28B1002301221549009861F000F91AE001F0B9FE10B101283B
:408D00000DD000BF00F08BFC684600F07FFC28B1002301220B49009861F0EDF805E000220121054817F0BAF900BF00BF00BF00BF012001F08DFE08BDE0390010D403002018
:408D40006F12833A35C00008E03A0010003C00102002002070B505466FF07F40281A00D100BF0A2001F09AFE002410E09FED170A204602F001FA9FED150A204602F029FAB3
:408D80009FED120A204602F04DFA601CC4B2042CECDB9FED0E0A002002F044FA9FED0B0A002002F060FA002002F08AFA012002F031FB012002F041FB012002F051FB0020DF
:408DC00002F0A4FA00BF00BF70BD00000000000010B588B004462068079060680690A0680590E06804902069039060690290A0690190E069009001F051FA01F01EFB08B013
:408E000010BD704770470020704770B5FFF7FBFF0446601C0A2190FBF1F201FB1200C5B22846FFF7EFFF0A2094FBF0F100FB1140092801D1FFF7E5FF70BD10B50020FFF70A
:408E4000E1FF10BDB0EE402AF0EE602AB4EEE11AF1EE10FA01D2B0EE611AB5EEC01AF1EE10FA02D0C1EE810A01E0F7EE000A20EE823AF7EE003A73EEE03AB0EE430A03EEE1
:408E8000A20A70470246B4EEE00AF1EE10FA01D2B0EE600AB5EEC00AF1EE10FA02D080EE801A01E0B7EE001A01EE902AF8EEE11A21EE212AF7EE001A71EEC12A01EE901A21
:408EC000F8EEE11A02EEA12AFDEEC21A11EE900A7047000001480068704700007C0100202DE9F04106AC94E8F01001604FF00008C0F804808360C260066145618461C76142
:408F0000C0F8208080F824C080F8258080F82680BDE8F08170472DE9F04104460D461646002794F8260078B90127012084F8260065602662E06838B12046D4E902129047B4
:408F400084F8250094F825703846BDE8F0810000F8B5044615461E46069F2A4633462046009722F06FFD04461B4820602046F8BD10B50446204622F0C5FD0446204610BDCE
:408F800070B504462046FFF7F3FF05468AF065FF70BD024601F18300C0B2704702460020704702460120704770B50646DDE90445002070BDF8B5012008490090D1E90053F0
:408FC0002A460748FFF7C4FF0446064AAFF25F0188F04AFEF8BD000008D00F08F86F0008403C00200080000812B10E2A01D101E000E000BF00BF7047FFFFFFFFFFFFFFFFAC
:4090000010B5044600202070606838B1606818B1606802685168884700206060A06838B1A06818B1A0680268516888470020A060E06838B1E06818B1E0680268516888473D
:409040000020E060206938B1206918B1206902685168884700202061606938B1606918B1606902685168884700206061A06938B1A06918B1A0690268516888470020A061F0
:40908000E06938B1E06918B1E0690268516888470020E061206A38B1206A18B1206A02685168884700202062606A38B1606A18B1606A02685168884700206062A06A38B115
:4090C000A06A18B1A06A0268516888470020A062E06A38B1E06A18B1E06A0268516888470020E062206B38B1206B18B1206B02685168884700202063606B38B1606B18B16B
:40910000606B02685168884700206063A06B38B1A06B18B1A06B0268516888470020A063E06B38B1E06B18B1E06B0268516888470020E063206C38B1206C18B1206C0268FF
:409140005168884700202064606C38B1606C18B1606C02685168884700206064A06C38B1A06C18B1A06C0268516888470020A064E06C38B1E06C18B1E06C02685168884763
:409180000020E064206D38B1206D18B1206D02685168884700202065606D38B1606D18B1606D02685168884700206065A06D38B1A06D18B1A06D0268516888470020A0657B
:4091C000E06D38B1E06D18B1E06D0268516888470020E06510BD10B5044600206060A060E06020616061A061E06120626062A062E06220636063A063E06320646064A0649F
:40920000E06420656065A065E0652046FFF7F8FE204610BD10B504462046FFF7F1FE204610BD2DE9F04704460F462046FFF7E8FE2770207800287DD0012802D002287AD102
:4092400000E000BF0C208AF011FE0546002252217DF047FF054660600C208AF007FE0546002253217DF03DFF0546A0600C208AF0FDFD0546002254217DF033FF0546E060D0
:409280000C208AF0F3FD0546002255217DF029FF054620610C208AF0E9FD0546002251217DF01FFF0546606108208AF0DFFD06463D217DF049FF0646A06208208AF0D6FD32
:4092C00006463E217DF040FF0646E06208208AF0CDFD064613217DF037FF0646206308208AF0C4FD064614217DF02EFF064660631C208AF0BBFD804601223F217DF0F2FB8D
:409300008046A0630C208AF0B1FD054600223B217DF0E7FE0546E0630C208AF0A7FD054600223C217DF0DDFE05462064606C68B90C2001E061E061E08AF098FD81460022C8
:4093400024217DF03FFF8146606400BFA06C50B90C208AF08BFD814600221D217DF041FE8146A06400BFE06C50B90C208AF07EFD814600221E217DF034FE8146E06400BF0C
:40938000206D50B90C208AF071FD814600221C217DF027FE8146206500BF606D50B90C208AF064FD8146012217217DF01AFE8146606500BFA06D50B90C208AF057FD81469A
:4093C000012218217DF00DFE8146A06500BF606D08B9A06D80B1E06D70B90C208AF046FD814617217DF082FD8146E065E06D01688A6A0121904700BF00E000BF00BFBDE887
:40940000F08710B5044604F0A1FE10BD0146087870470246002053680B600B6803B1012070470246002093680B600B6803B10120704702460020D3680B600B6803B1012018
:4094400070470246002013690B600B6803B1012070470246002053690B600B6803B1012070470246002093690B600B6803B10120704702460020D3690B600B6803B1012034
:40948000704702460020136A0B600B6803B10120704702460020536A0B600B6803B10120704702460020936A0B600B6803B10120704702460020D36A0B600B6803B10120F0
:4094C000704702460020136B0B600B6803B10120704702460020536B0B600B6803B10120704702460020936B0B600B6803B10120704702460020D36B0B600B6803B10120AC
:40950000704702460020136C0B600B6803B10120704702460020536C0B600B6803B10120704702460020936C0B600B6803B10120704702460020D36C0B600B6803B1012067
:40954000704702460020136D0B600B6803B10120704702460020536D0B600B6803B10120704702460020936D0B600B6803B10120704710B50448FFF72EFE0446034AAFF213
:409580006B3188F071FB10BDD40300200080000810B50446F94800688047E060002020746074A074E07420756075206881682046884710BD10B50446204660F069FC0446DF
:4095C000EF4820602046FFF7E3FF204610BD10B50446204660F062FC0446204610BD70B504462046FFF7F3FF05468AF036FC70BD70B50546012406E0E24B00222146284623
:4096000060F0FCFC641C202CF6D370BD01460020DD4A12680A600A6802B10120704710B5D948006848B918208AF020FC0446FFF7C1FF0446D448046000BF10BD10B5D2485F
:40964000006870B1D048006830B1CF48006800684168CD48006888470020CB4908607BF04DFD10BD3EB50020009001900290684688F07AFBC4B22146684601F069FA0020A6
:4096800001F085FAC14801F095FA012001F0A5FA012001F0B5FA002001F0C5FA002001F0D5FA002001F0E5FA002001F0F5FA002001F005FB002001F01FFBB54801F02EFB4C
:4096C000B44801F03EFBB44801F04EFBB34801F05EFB002001F0CCFB002001F0DCFB002001F0ECFB002001F0FCFB002001F00CFC002001F01CFC002001F02CFC002001F07D
:40970000D5FEFA2001F056FB4FF4FA6001F065FB41F2707001F073FB40F27E3001F082FB40F6F85001F091FB3EBD0146487D70470146087C704710B5044601F098F910BDB3
:409740002DE9F04107460C461546002601F08FF9A04208D0204601F08EF92B4632460321384660F04BFC3046BDE8F08110B5044601F0EBF910BD2DE9F04707460D461446CB
:409780009846002601F0E1F98146142C01DA204600E0142002462946484688F00EFB48B12146284601F0D4F9434632460421384660F024FC3046BDE8F08710B5044601F086
:4097C000E2F910BD2DE9F04107460C461546002601F0D9F9A04208D0204601F0D8F92B4632460521384660F009FC3046BDE8F08110B5044601F0DAF910BD2DE9F041074613
:409800000C461546002601F0D1F9A04208D0204601F0D0F92B4632460621384660F0EEFB3046BDE8F08110B5044601F0D2F910BD2DE9F04107460C461546002601F0C9F9BB
:40984000A04208D0204601F0C8F92B4632460721384660F0D3FB3046BDE8F08110B5044601F020FE10BD2DE9F04107460C46154600263846FFF7F2FFA04208D0204601F015
:4098800015FE2B4632460821384660F0B7FB3046BDE8F08110B5044601F0AEF910BD2DE9F04107460C461546002601F06CFAA04208D0204601F06BFA2B4632461321384634
:4098C00060F09CFB3046BDE8F0812DE9F04107460C461546002601F043FAA04208D0204601F042FA2B4632461221384660F086FB3046BDE8F0812DE9F04107460C461546DB
:40990000002601F01AFAA04208D0204601F019FA2B4632461121384660F070FB3046BDE8F0812DE9F04107460C461546002601F0F1F9A04208D0204601F0F0F92B463246D3
:409940001021384660F05AFB3046BDE8F0812DE9F04107460C461546002601F0BFF9A04208D0204601F0C8F92B4632460F21384660F044FB3046BDE8F0810000082000103B
:4099800010CC0F08B53C090800000020E4D914013A9B220089C31400C5610A00EC7503002DE9F04107460C461546002601F083F9A04208D0204601F082F92B4632460E215D
:4099C000384660F01BFB3046BDE8F0812DE9F04107460C461546002601F05AF9A04208D0204601F059F92B4632460D21384660F005FB3046BDE8F0812DE9F04107460C4692
:409A00001546002601F031F9A04208D0204601F030F92B4632460C21384660F0EFFA3046BDE8F0812DE9F04107460C461546002601F0F5F8A04230D0204601F0F4F82A461D
:409A400000213846FFF7D8FF2A4600213846FFF7BDFF2A4600213846FFF7A2FF2A4600213846FFF774FF2A46FC493846FFF759FF2A46FB493846FFF73EFF2A46F949384685
:409A8000FFF723FF2A46F8493846FFF708FF2B4632460A21384660F0B1FA3046BDE8F0812DE9F04107460C461546002601F0A4F8A0420DD0204601F0A3F82A460021384695
:409AC000FFF7B0FF2B4632460921384660F096FA3046BDE8F08110B5044601F0A0F810BD10B5044601F0AEF810BD2DE9F04107460C461546002601F0A5F8A04208D02046D7
:409B000001F0A4F82B4632460B21384660F076FA3046BDE8F08110B5044601F0A6F810BD10B5044601F0B4F810BD10B5044601F0C2F810BD10B5044601F0D0F810BD10B5F4
:409B4000044601F0E7F810BD10B5044601F0F5F810BD10B5044601F003F910BD10B5044601F011F910BD10B5044601F01FF910BD2DE9F04107460C461546002601F016F958
:409B8000A04208D0204601F015F92B4632461421384660F033FA3046BDE8F08110B5044601F017F910BD2DE9F04107460C461546002601F00EF9A04208D0204601F00DF98E
:409BC0002B4632461521384660F018FA3046BDE8F08110B5044601F00EF910BD2DE9F04107460C461546002601F005F9A04208D0204601F004F92B4632461621384660F0B4
:409C0000FDF93046BDE8F08110B5044601F006F910BD2DE9F04107460C461546002601F0FDF8A04208D0204601F0FCF82B4632461721384660F0E2F93046BDE8F08110B569
:409C4000044601F0FEF810BD2DE9F04107460C461546002601F0F5F8A04208D0204601F0F4F82B4632461821384660F0C7F93046BDE8F08110B5044601F0F6F810BD2DE997
:409C8000F04107460C461546002601F0EDF8A04208D0204601F0ECF82B4632461921384660F0ACF93046BDE8F08110B5044601F0EEF810BD2DE9F04107460C46154600264C
:409CC00001F0E5F8A04208D0204601F0E4F82B4632461A21384660F091F93046BDE8F08110B5044601F0E6F810BD2DE9F04107460C461546002601F0DDF8A04208D02046A9
:409D000001F0DCF82B4632461B21384660F076F93046BDE8F08110B5044601F0DEF810BD2DE9F04107460C461546002601F0D5F8A04208D0204601F0D4F82B4632461C21A5
:409D4000384660F05BF93046BDE8F08110B5044601F0D6F810BD2DE9F04107460C461546002601F0CDF8A04208D0204601F0CCF82B4632461D21384660F040F93046BDE85F
:409D8000F08110B5044601F0CEF810BD2DE9F04107460C461546002601F0C5F8A04208D0204601F0C4F82B4632461E21384660F025F93046BDE8F08110B5044601F0C6F85F
:409DC00010BD2DE9F04107460C461546002601F0BDF8A04208D0204601F0BCF82B4632461F21384660F00AF93046BDE8F08101214174704700B502461046FFF796FC08B11C
:409E00000120907400BD0121C174704701210175704770B504460D46607DA84206D06575124B00220121204660F0E8F870BD70B504460D46207CA8420ED000212046FFF7A3
:409E4000E8FF25740A4800688047E060074B00220221204660F0D2F870BD00003A9B220089C31400C5610A00EC750300B53C09080820001070B504462046FFF759FC0928E7
:409E80007ED2DFE800F0050C264E6C9EE9F6F500FFF7E8FB01212046FFF7C9FF22E12046FFF764FC0546142298A187F086FF20B101212046FFF7ADFF03E000212046FFF749
:409EC000A8FFA07C012803D102212046FFF7AFFF08E12046FFF771FC78B12046FFF788FC58B12046FFF79FFC38B101F0DBFA20B101212046FFF78DFF03E000212046FFF7D0
:409F000088FFA07C012804D103212046FFF78FFF06E0607C012803D101212046FFF787FFE0E001212046FFF774FFA07C01280ED12046FFF7D0FD012804D104212046FFF732
:409F400076FF0BE006212046FFF771FF06E0607C012803D102212046FFF769FFC2E02046FFF7D9FD90B12046FFF7DAFD70B12046FFF7DBFD50B12046FFF7DCFD30B100E054
:409F8000ABE001212046FFF744FF03E000212046FFF73FFF2046FFF79EFD10B92046FFF729FFA07C012804D105212046FFF73FFF06E0607C012803D103212046FFF737FF24
:409FC00090E02046FFF7BBFD58B32046FFF7BCFD38B32046FFF7BDFD18B32046FFF7BEFDF8B12046FFF7ABFD05462046FFF7ACFD854216D32046FFF7A7FD05462046FFF786
:40A00000A8FD85420DD32046FFF7A3FD05462046FFF7A4FD854204D301212046FFF7F9FE03E000212046FFF7F4FE2046FFF753FD10B92046FFF7DEFEA07C012804D106213D
:40A040002046FFF7F4FE06E0607C012803D104212046FFF7ECFE45E001212046FFF7D9FEA07C012806D107212046FFF7E0FE12E032E011E0607C01280DD12046FFF72BFD14
:40A08000012804D105212046FFF7D1FE03E003212046FFF7CCFE25E001212046FFF7B9FEA07C012810D108212046FFF7C0FEFEF760FD00220121164815F0F0FF154A012118
:40A0C0002046FFF73DFB06E0607C012803D106212046FFF7ACFE05E004E008212046FFF7A6FE00BF00BF00206074A074E074207570BD10B504462046FFF7BCFE2046FFF7D1
:40A1000017FB082801D1FFF799FA10BD00000000E0390010B53C090870470146B1F1006F04D3B1F1026F01D8012070470020FCE70146B1F1805F02D39D48814205D9B1F118
:40A14000005F04D39B48814201D8012070470020FCE70146002070470146974A974800681318914203D3994201D8012070470020FCE770B5044600252046FFF7EDFF08B1CA
:40A18000032510E02046FFF7E4FF08B104250AE02046FFF7CDFF08B1022504E02046FFF7BCFF00B10125284670BD01460020844A1288914202D2834A52F82100704730B5BD
:40A1C000002500240AE02046FFF7EFFF034623B15878022801D11D4604E0641C784800888442F0D3284630BD70B5FFF7E8FF04460025FF22C821744887F0A1FE681E734977
:40A200000860002C3DD0206B0860E08C002838D0E08C0121C1EB900631E0E16A51F82600FFF7A7FF052828D2DFE800F026030D0E0F00322D06D2E06A50F82600624941F8B3
:40A2400025006D1C19E000BF17E0322D13D212D2E16A51F826100868FFF78BFF052809D2DFE800F004030506070003E000BF00BF00BF00BF00BF00E000BF00BF761E002E09
:40A28000CBD15348007840B10020514908702A464D494E480068FFF73FFF70BD10B5FFF7A3FF10BD10B504462046FFF755FF10BD10B50446002010BD10B504462046FFF74A
:40A2C00074FF0346DFED430AB0EE600A1BB3D88C08B304201CE0D96A095CCC2917D0D98C00EE901AB8EE601A00EE900AF8EE600A71EE600A9FED381A20EE811A00EE901A13
:40A30000F8EE600AC1EE201AB0EE610A03E0401CD98C8142DFD810BD10B504462046FFF744FF0346DFED2B0AB0EE600AE3B1D88CD0B1D98CD86A0844996A884214D3D3E914
:40A340000A01401AD98C081A00EE900AF8EE600A9FED211A20EE811A00EE901AF8EE600AC1EE201AB0EE610A10BD30B50025002408E02046FFF719FF034613B1587800B1EA
:40A380006D1C641C0E4800888442F2D3284630BD0B48008870477047704710B50F48FFF7FAFF04460E4AAFF20F0187F05DFC10BD000001100000032050430220C8C00F084D
:40A3C00094C00F080CB50220340400200400001008000010000000000000C842000000100080000870470020684904E00A68824200D9086849680029F8D1704700206349D8
:40A4000002E00A68104449680029FAD1704710B5FFF7F4FF5E490860FFF7E5FF5D4908605D48007840B100205B4908705948016857480068FFF7D6FF10BD10B5FFF7E7FFDF
:40A4400010BD01465148814204D35448814201D8012070470020FCE700B502461046FFF7F0FF00BD024600207047704770472DE9F84F16461F460BAC94E83006DDF82880FC
:40A480000020009020602860062089F8000000208AF8000000210F98016010980160B6F56F4F64D1412F60D1B8F1420F03D0B8F1430F58D128E037493548FFF7D3FF10B3A9
:40A4C000334A1068334A11684122354B1A7042225A70344A904200D91046324A914200D911462F4B9870020ADA70020C1A7159710A0A9A710A0CDA7108222A601A46226087
:40A500000122009200BF2EE0FFF778FF20490860FFF769FF1F4908601D4803680846D0F800B041201E490870432048701D48834200D903461B48834500D9834618498B70C7
:40A54000180AC870180C087181F805B04FEA1B2088714FEA1B40C87108202860084620600120009000BF00BF00BF00BF00BF00BF0098BDE8F88F10B50B48FFF776FF044642
:40A580000A4AAFF2171187F06FFB10BDE0BD0220080000200C00002010000020E0FD022011000020FDFFFF0004000020008000082DE9F0432DED028B81B004460F4615469B
:40A5C000002D73D1E0B22A2871D012DCA0F1110019286DD2DFE800F0636D1D242B323940474EF28289F2F2F255F2F25CF2F2F2F27400A4381528ECD2DFE800F07E858C932E
:40A600009AA1E0E0E0A8AFB6E0E0E0E0BDC4CBD2D900BB4815F094F9064600F02AFB66E1B74815F0A6F9064600F036FB5FE1B44815F0B8F9064600F042FB58E1B04815F0CD
:40A64000CAF9064600F058FB51E1AD4815F0DCF9064600F063FB4AE1A94815F0EEF9064600F06FFB43E1A64815F000FA064600F07BFB3CE1A24815F015FA064600F087FBA3
:40A6800035E19F4814F018FC064600F006FE2EE19B4815F027F9064600F0C5FA27E1984815F0D5F8064600F072FA20E121E10EE084E0934815F0E4F8064600F08EFA16E105
:40A6C0008F4815F0B8FB064600F00DFE0FE18C4814F04DFC064600F019FE08E1884815F013FA064600F0C4FB01E1854815F025FA064600F0D0FBFAE0814814F0A0FB0646F2
:40A7000000F017FEF3E07E4814F080FB064600F022FEECE07A4814F055FB064600F02EFEE5E0774814F035FB064600F03AFEDEE0734814F015FB064600F046FED7E07048AE
:40A7400014F0F5FA064600F052FED0E06C4815F056FC064600F05EFEC9E0694815F068FC064600F06AFEC2E0654815F07AFC064600F076FEBBE0624815F07DFD064600F026
:40A7800019FBB4E05E4815F08FFD064600F025FBADE05B4815F0A1FD064600F030FBA6E0574814F001FA064600F03CFB9FE0544814F0F6F9064600F048FB98E0312C15D343
:40A7C000342C13D800200090A4F13100C6B26A4631464B4814F0D3F938B100985DF0A3FC80464146304600F0A3FC7FE0372C17D100200090A4F13500C6B26A46314640488C
:40A8000014F0BDF958B100985DF0F7FC81463C4815F05EFC09FB00F8404600F0CBF965E0392C15D33C2C13D800200090A4F13900C6B26A463146324814F0A1F938B1009802
:40A840005DF0C4FCB0EE408A304600F095FC4DE0412C19D3442C17D800200090A4F14100C6B26A463146264814F089F958B100985DF010FD00EE100AB8EE400AB0EE408A13
:40A88000304600F0A6FC31E0632C18D317D800200090A4F16300C6B26A463146184814F07AFB58B100985EF017F900EE100AB8EE400AB0EE408A304600F0D5FC16E0642CDA
:40A8C00014D313D800200090A4F16400C6B26A4631460B4814F05FFB38B100985EF0ECF8B0EE408A304600F09DFC00BF00BF00BF00E000BF00BF01B0BDEC028BBDE8F083D9
:40A90000E0390010F74890F8A001704710B5044600BFF44880F8A041012200F5D071F24800F0DEFD00BF10BDEE4901F5D47103C9704770B504460D4600BFEA4800F5D470A1
:40A9400030C00822E949E848083000F0C9FD00BF70BDE748704710B5044600BFE148C0F8B041042200F5D871DF48103000F0B8FD00BF10BDDB484068704710B5044600BFAF
:40A98000D84844600422011DDA4800F0A9FD00BF10BDD4480068704710B5044600BFD1480460042201464FF0D04000F099FD00BF10BDCC488068704710B5044600BFC94865
:40A9C0008460042200F10801CA48001D00F088FD00BF10BDC348D0F8BC01704770B506460D46FFF7F7FF0446012E0CD12C4300BFBC48C0F8BC41042200F5DE71BA481C3037
:40AA000000F06EFD0CE0AC4300BFB648C0F8BC41042200F5DE71B4481C3000F061FD00BF70BDB048D0F8DC01704710B5044600BFAC48C0F8DC41042200F5EE71AA48743087
:40AA400000F04EFD00BF10BDA64890F8C801704710B5044600BFA34880F8C841012200F5E471A148603000F03BFD00BF10BD9D4890F8E001704710B5044600BF994880F819
:40AA8000E041012200F5F0719748783000F028FD00BF10BD934890F8E101704710B5044600BF904880F8E141012200F2E1118E48793000F015FD00BF10BD8A4890ED740AB7
:40AAC000704710B52DED028BB0EE408A00BF854880ED748A042200F5E8718348683000F0FFFC00BFBDEC028B10BD7E4890ED750A704710B52DED028BB0EE408A00BF794883
:40AB000080ED758A042200F5EA7177486C3000F0E7FC00BFBDEC028B10BD724890ED760A704710B52DED028BB0EE408A00BF6D4880ED768A042200F5EC716B48703000F065
:40AB4000CFFC00BFBDEC028B10BD68483A30704770B504460D46142164483A3087F0F7F9142D01DA284600E01420024621465F483A3087F035FA14225C493A315A487A306D
:40AB800000F0AEFC70BD5748D0F8F801704710B5044600BF5348C0F8F841042200F5FC715148903000F09CFC00BF10BD4D48D0F8FC01704710B5044600BF4A48C0F8FC4102
:40ABC000042200F5FE714848943000F089FC00BF10BD444890F80002704710B5044600BF404880F80042012200F500713E48983000F076FC00BF10BD3A4890F80102704710
:40AC000010B5044600BF374880F80142012200F201213548993000F063FC00BF10BD314890F80202704710B5044600BF2D4880F80242012200F202212B489A3000F050FC48
:40AC400000BF10BD274890F80302704710B5044600BF244880F80342012200F2032122489B3000F03DFC00BF10BD1E48B0F80402704710B5044600BF1A48A0F8044202227E
:40AC800000F5017118489C3000F02AFC00BF10BD1448B0F80602704710B5044600BF1148A0F80642022200F206210F489E3000F017FC00BF10BD0B48B0F80802704710B523
:40ACC000044600BF0748A0F80842022200F502710548A03000F004FC00BF10BD0148B0F80A02704700050020A0010068A8060020C0D401000400006810B5044600BFFC4832
:40AD0000A0F80A42022200F20A21FA4800F0E8FB00BF10BDF648D0F8F802704710B5044600BFF348C0F8F842042200F53E71F148EE3000F0D5FB00BF10BDED48D0F8FC0233
:40AD4000704710B5044600BFE948C0F8FC42042200F53F71E748F23000F0C2FB00BF10BDE348D0F80003704710B5044600BFE048C0F80043042200F54071DE48F63000F02C
:40AD8000AFFB00BF10BDDA48D0F80403704710B5044600BFD648C0F80443042200F54171D448FA3000F09CFB00BF10BDD048D0F80803704710B5044600BFCD48C0F808431C
:40ADC000042200F54271CB48FE3000F089FB00BF10BDC748D0F80C03704710B5044600BFC348C0F80C43042200F54371C24800F077FB00BF10BDBE48D0F81003704710B5A3
:40AE0000044600BFBA48C0F81043042200F54471B948001D00F064FB00BF10BDB448D0F81403704710B5044600BFB148C0F81443042200F54571B048083000F051FB00BFCF
:40AE400010BDAB48D0F81803704710B5044600BFA748C0F81843042200F54671A6480C3000F03EFB00BF10BDA14890F80C02704710B5044600BF9E4880F80C42012200F52F
:40AE800003719C48801C00F02BFB00BF10BD984890F80D02704710B5044600BF944880F80D42012200F20D219248C01C00F018FB00BF10BD8E4890F80E02704710B50446A1
:40AEC00000BF8B4880F80E42012200F20E218948001D00F005FB00BF10BD854890F80F02704710B5044600BF814880F80F42012200F20F217F48401D00F0F2FA00BF10BDFC
:40AF00007B48B0F81002704710B5044600BF7848A0F81042022200F504717648801D00F0DFFA00BF10BD724890F81202704710B5044600BF6E4880F81242012200F2122182
:40AF40006C48083000F0CCFA00BF10BD684890F81302704710B5044600BF654880F81342012200F213216348093000F0B9FA00BF10BD5F48D0F81402704710B5044600BFF1
:40AF80005B48C0F81442042200F5057159480A3000F0A6FA00BF10BD5548D0F81802704710B5044600BF5248C0F81842042200F5067150480E3000F093FA00BF10BD4C48A3
:40AFC000D0F81C02704710B5044600BF4848C0F81C42042200F507714648123000F080FA00BF10BD4248D0F82002704710B5044600BF3F48C0F82042042200F508713D4834
:40B00000163000F06DFA00BF10BD3948D0F82402704710B5044600BF3548C0F82442042200F5097133481A3000F05AFA00BF10BD2F48D0F82802704710B5044600BF2C48CC
:40B04000C0F82842042200F50A712A481E3000F047FA00BF10BD2648D0F82C02704710B5044600BF2248C0F82C42042200F50B712048223000F034FA00BF10BD1C48D0F8FB
:40B080003002704710B5044600BF1948C0F83042042200F50C711748263000F021FA00BF10BD1348D0F83402704710B5044600BF0F48C0F83442042200F50D710D482A30BF
:40B0C00000F00EFA00BF10BD0948D0F83802704710B5044600BF0648C0F83842042200F50E7104482E3000F0FBF900BF10BD0000000500204202006844030068F348D0F83D
:40B100003C02704710B5044600BFF048C0F83C42042200F50F71EE4800F0E2F900BF10BD01460020042902DAEA4A52F82100704770B504460D46042C0EDA00BFE54840F8F2
:40B140002450E34A121D02EB8400E24A02EB8401042200F0C5F900BF70BDDFEDDF0AB0EE600A042807DADB49103101EB8001D1ED000AB0EE600A704710B52DED028B044657
:40B18000B0EE408A042C12DA00BFD248103000EB840080ED008ACE4A143202EB8400CD4A103202EB8401042200F09AF900BFBDEC028B10BDDFEDC80AB0EE600A042807DAD4
:40B1C000C449203101EB8001D1ED000AB0EE600A704710B52DED028B0446B0EE408A042C12DA00BFBB48203000EB840080ED008AB74A243202EB8400B64A203202EB8401BF
:40B20000042200F06DF900BFBDEC028B10BDDFEDB20AB0EE600A20B9AC49D1ED9C0AB0EE600A704710B52DED028B0446B0EE408A5CB900BFA54880ED9C8A042200F51C7135
:40B24000A348343000F04CF900BFBDEC028B10BDDFEDA10AB0EE600A20B99C49D1ED9D0AB0EE600A704710B52DED028B0446B0EE408A5CB900BF954880ED9D8A042200F5A9
:40B280001D719348383000F02BF900BFBDEC028B10BD8E48D0F87802704710B5044600BF8A48C0F87842042200F51E7188483C3000F016F900BF10BD844890F87C0270470C
:40B2C00010B5044600BF814880F87C42012200F51F717F48403000F003F900BF10BD7B48D0F88002704710B5044600BF7748C0F88042042200F520717548443000F0F0F8AA
:40B3000000BF10BD7148D0F8F402704710B5044600BF6E48C0F8F442042200F53D716C48B83000F0DDF800BF10BD6848D0F83003704710B5044600BF6448C0F830430422FE
:40B3400000F54C71654800F0CBF800BF10BD5F48D0F83403704710B5044600BF5B48C0F83443042200F54D715C48001D00F0B8F800BF10BD5548D0F83803704710B5044606
:40B3800000BF5248C0F83843042200F54E715348083000F0A5F800BF10BD4C48D0F83C03704710B5044600BF4848C0F83C43042200F54F7149480C3000F092F800BF10BDA6
:40B3C0004248D0F84003704710B5044600BF3F48C0F84043042200F550714048103000F07FF800BF10BD3948D0F84403704710B5044600BF3548C0F84443042200F551712C
:40B400003648143000F06CF800BF10BD2F4890F88402704710B5044600BF2C4880F88442012200F521712A48483000F059F800BF10BD264890F88502704710B5044600BF4B
:40B44000224880F88542012200F285212048493000F046F800BF10BD1C4890F88602704710B5044600BF194880F88642012200F2862117484A3000F033F800BF10BD13489C
:40B48000B0F8CC01704710B5044600BF0F48A0F8CC41022200F5E6710D48703800F020F800BF10BD094890F8F002704710B5044600BF064880F8F042012200F53C7104483C
:40B4C000B43000F00DF800BF10BD000000050020740200684007002000000000107500682DE9F04104460F4615460026FE4884420ED36019401EFD49884209D8FA48211AF7
:40B500002A46384609F057FD00B915E0202613E0B4F1D04F0FD36019401EF54988420AD8A4F1D0412A46384609F0B2FF08B9002602E0202600E0082626B1EE48008830431F
:40B54000EC4908803046BDE8F08110B50024FFF796FF032800D10124204610BD2DE9F04107460C4615460026DF4884420ED36019401EDE49884209D8DB48211A2A46384690
:40B5800009F047FD00B924E0202622E0B4F1D04F0FD36019401ED64988420AD8A4F1D0412A46384609F0FDFF08B9002611E020260FE0B4F1006F0BD36019401ECE498842C1
:40B5C00006D82A462146384686F042FC002600E0082626B1C74800883043C64908803046BDE8F0812DE9FE4F06468946174698460020009083464FF480720023384641469D
:40B6000086F09AF805464FF4807200233846414686F092F8924615B9BAF1000F2AD0ADB1002411E006EB0420029009EB042001904FF48072DDE90110FFF790FF0090009884
:40B640004BEA000B601CC4B2AC42EBD3BAF1000F12D006EB0520029009EB052001901FFA8AF2DDE90110FFF779FF009000984BEA000B01E04FF0400B5846BDE8FE8F2DE96B
:40B68000FE4F06468946174698460020009083464FF4807200233846414686F04DF805464FF4807200233846414686F045F8924615B9BAF1000F2AD0ADB1002411E006EB3D
:40B6C0000420029009EB042001904FF48072DDE90110FFF705FF009000984BEA000B601CC4B2AC42EBD3BAF1000F12D006EB0520029009EB052001901FFA8AF2DDE9011085
:40B70000FFF7EEFE009000984BEA000B01E04FF0400B5846BDE8FE8FFEB5002001900090002600274FF45C71744886F032FCEC200290012202A97248FFF7D2FE68B90020A6
:40B74000029001226E4902A8FFF708FF28B99DF80800EC2801D1781CC7B212200290012202A96748FFF7BCFE68B9002002900122634902A8FFF7F2FE28B99DF8080012286A
:40B7800001D1781CC7B2022F07D05A48008840F08000584908800124D7E00122594901A8FFF7DCFE08B9701CC6B201225549491C6846FFF7D3FE08B9701CC6B2022E07D158
:40B7C0009DF80400012803D19DF80000122831D04FF4E471494886F0DCFB4FF4E472002346494FF0D040FFF74AFF4FF4AA72002345494348DC30FFF742FF282200234349BD
:40B800004348FFF73CFF28220023404928314148FFF735FF01200190012201A93948FFF75FFE12200090012269463648401CFFF757FE07E04FF4E47200234FF0D0412F48D4
:40B84000FFF7D0FE02222E49DE312F48801CFFF785FE05462948B0F8CA01012800D10DB301244FF4AA71284886F093FB4FF4AA72002325492248DC30FFF701FF2822002325
:40B88000224928312348FFF7FAFE00BF01211B48A0F8CA11022200F5E5711948DE30FFF71FFE0FE002244FF4AA7200231449DC311548FFF797FE282200231649134828305B
:40B8C000FFF790FE022212491048FFF747FE05460A48B0F82003022800D15DB300BF02200649A1F8200317E000010168FF000169FF7F00680C000010FF7F0F0800050020CD
:40B90000240100681B000068C8060020200800200075006800500068022201F548716248FFF7DEFD00BF2822002360495E48FFF7A6FE05E0282200235B495C48FFF752FEE9
:40B94000FFF703FE08B95AF0DAFC2046FEBD7FB5002000900190029003900120544908805449087009F07EF80020514908800846008800285BD1FFF7CFFE4F4908804F4B81
:40B980004FA20F21684685F08DFF0025002408E04C48005D1DF80410884200D00125601C84B20F2CF4DB4448008801280DD10020404908700F226946424886F08EFA0F221B
:40B9C00040494148FFF78CFD35E0012D33D10020FEF7F2FFFFF7EAF910B9FA20FFF7EAF9FFF7F7F918B94FF4FA60FFF7F6F9FFF702FA18B941F27070FFF701FAFFF70EFAD6
:40BA000018B940F27E30FFF70DFAFFF71AFA18B940F6F850FFF719FA0F226946294886F05CFA0F2227492848FFF75AFD03E020480088214908807FBD1E48007870471E487F
:40BA4000008870471C49098881431B4A1180704717480088704770B504460D4600261B4884420BD31A48854208D8184AA91AA01A09F0A8F900B902E0202600E0082626B14B
:40BA80000B48008830430A490880304670BD10B50446012C03D10320FFF7F5FC02E00020FFF7F1FC10BD000000750068200800200C0000100E0000100A0000109CBE000813
:40BAC000257300000C0500200C00006800010168FF00016901DF70470EB50020029001909A48006840F480309849086000BF9748006800F4003001900298401C0290019846
:40BB000020B941F2883102988842F0D18F48006800F4003010B10120019001E0002001900198012864D18A488849091D0860081F006840F08070091F086000BF00200090DD
:40BB400082484030006840F080508049403108600846006800F08050009000BF7D48006840F4E0307B49086000BF7A48406800F480300028F9D07748006840F40030754918
:40BB8000086000BF7348406800F400300028F9D06E48083000686D49083108600846006840F4004008600846006840F4A050086000BF6648006800F000700028F9D040F20D
:40BBC00005606549086061480830006820F003005E49083108600846006840F00200086000BF5A480830006800F00C000828F8D10EBD10B588F050FCFFF76EFF85F0A8FC10
:40BC00000AF0A7F807F0D1FB0021544888F072FD5349886388F052FC002010BD2DE9F34FA7B007460020239000BF009047483030006840F480504549303108600846006844
:40BC400000F48050009000BF002024908246B7F1FF3F00D01FB9239829B0BDE8F08F002410E027FA04F000F0010050B1A2460AEB4A003C4951F8200000F54050D0F8FCBF97
:40BC800002E0641C202CECD300BF00240DE00AEB4A00344951F8200043F6F4710844A0EBC40003A941F82400641C202CEFD32E48259025A87DF0A3FD00252FE003A850F826
:40BCC0002500066803A850F82500D0F80480B6F1FF3F02D1B8F1FF3F1ED046451CD8249850B930680290012202A925A87DF0CCFD019001202490361DB1460AE0D9F8000016
:40BD00000290012202A925A87DF09DFD019009F10409C145F2D900E002E06D1C202DCDD300BF0A483030006820F480500749303108602899019808600198834502D1012041
:40BD4000239001E000202390239885E7003802400C5A400700700040003C0240BCBE0908300A0020CCBE0908003002402DE9FC41044615461E46DDE908782A4633462046FD
:40BD8000CDE900781CF09EF80446224820602046BDE8FC8110B5044620461CF0D9F80446204610BD70B504462046FFF7F3FF054688F053F870BD0146022070470146487908
:40BDC000FE2801DA012070470020FCE71CB50446207902280CDA6079FE2809DA00202179C1EBC1110C4A02EBC101627941F82200FE2060714FF0FF3100910191DDE9000106
:40BE0000C4E9020100BF20461CF02DFA1CBD7047704700003CD00F08E43E0010004870472CE9001010B50446AFF300802046BDE81040FCF78DBA704770477047000000004F
:40BE40000000000000000000000000003037373031373134353500000000000030373730313731343335000000000000526176656E20496E647573747269657320496E633A
:40BE80000000000000000000000000004A756E2D32382D32303138000000000032322E312E302E323200000000000000556E766572666572746820477261696E20436172A3
:40BEC00074204D6F64756C6500000000303737303137313533380000000000000000000000000000000000000000000000000000000000000000000000000000FFFFFFFF45
:40BF0000FFFFFFFFFFFFFFFFFFFFFFFFFFFFFFFFFFFFFFFFFFFFFFFFFFFFFFFFFFFFFFFFFFFFFFFFFFFFFFFFFFFFFFFFFFFFFFFFFFFFFFFFFFFFFFFFFFFFFFFFFFFFFFFF41
:40BF4000FFFFFFFFFFFFFFFFFFFFFFFFFFFFFFFFFFFFFFFFFFFFFFFFFFFFFFFFFFFFFFFFFFFFFFFFFFFFFFFFFFFFFFFFFFFFFFFFFFFFFFFFFFFFFFFFFFFFFFFFFFFFFFFF01
:40BF8000FFFFFFFFFFFFFFFFFFFFFFFFFFFFFFFFFFFFFFFFFFFFFFFFFFFFFFFFFFFFFFFFFFFFFFFFFFFFFFFFFFFFFFFFFFFFFFFFFFFFFFFFFFFFFFFFFFFFFFFFFFFFFFFFC1
:40BFC000FFFFFFFFFFFFFFFFFFFFFFFFFFFFFFFFFFFFFFFFFFFFFFFFFFFFFFFFC03E18083F40180800C00008FFF10F0804880008FBBF000800800008FF8700082F01D57FE1
:40C0000070472DE9F04104460D4617469846069EA0B2324629466EF0DFFE324629462046FEF7C6FA33462A462146F9482AF0C1FCBDE8F0812DE9F84305460C4616461F46E3
:40C04000DDF820800F2C3ED2DFE804F008162425262728292A2B2C2D2E3D3C00E0B23B463246002100902846FFF7CBFFE2B241462846FCF7B9FF2FE0E0B23B463246002192
:40C0800000902846FFF7BDFFE2B241462846FCF7ABFF21E000BF00BF00BF00BF00BF00BF00BF00BF00BF00BFE0B23B463246002100902846FFF7A5FFE2B241462846FCF773
:40C0C00093FF09E000BFE0B23B463246002100902846FFF796FF00BF00BFBDE8F88338B504460020034602460E2100902046FFF7A1FF38BDC7480068704738B50446002016
:40C1000000906946204652F062F940B100980068C149026A009890471720FFF7E0FF38BDBE480068704710B50446FFF7F9FFA04207D0BA4804601620FFF7D1FF2046FFF74D
:40C14000DCFF10BDB6480068704710B50446FFF7F9FFA04207D0B24804601520FFF7BFFF0020FFF7E0FF10BD10B50446FFF7C2FFA04207D0A74804601420FFF7B0FF002070
:40C18000FFF7E3FF10BD10B51420FFF7A8FF10BD10B51520FFF7A3FF10BD10B51620FFF79EFF10BD9F480068704738B50446FFF7F9FFA04215D09B48046000200090694625
:40C1C000204653F0F8FC009820B19748009953F037F902E0944852F099FF1820FFF77FFF00BF38BD91480068704710B50446FFF7F9FFA04204D08D4804601920FFF76FFFD5
:40C2000010BD10B51920FFF76AFF10BD88480068704710B50446FFF7F9FFA04204D0844804601A20FFF75BFF10BD10B51A20FFF756FF10BD7F480068704710B50446FFF7DC
:40C24000F9FFA04207D07B4804601B20FFF747FF0020FFF7CAFF10BD10B51B20FFF73FFF10BD75480068704710B50446FFF7F9FFA04204D0704804601C20FFF730FF10BDE9
:40C2800010B51C20FFF72BFF10BD6C480068704710B50446FFF7F9FFA04204D0674804601D20FFF71CFF10BD10B51D20FFF717FF10BD63480068704710B50446FFF7F9FF3A
:40C2C000A04204D05E4804601E20FFF708FF10BD10B51E20FFF703FF10BD5A480068704710B50446FFF7F9FFA04204D0554804601F20FFF7F4FE10BD10B51F20FFF7EFFE5E
:40C3000010BD51480068704738B504464F484EF0A1FAA0420DD000200090694620464EF007FE4A4800994EF06CFB2020FFF7D7FE00BF38BD46480068704738B5044643480C
:40C340004C3853F09FFDA0420ED0002000906946204654F0F6FD3D484C38009954F099F82120FFF7BCFE00BF38BD3A480078704710B5044637480078A04204D03548047024
:40C380002220FFF7ACFE10BD3348704710B504462CB120683049C2692046904703E014212D4885F0D4FD2320FFF799FE10BD2B48704710B504462CB120682849C269204637
:40C3C000904703E01421254885F0C1FD2420FFF786FE10BD2248704710B504462CB120681F49C2692046904703E014211C4885F0AEFD2520FFF773FE10BD1A48704710B5CB
:40C4000004468CB320681749C2692046904730E0F455001010000010C008002018000010140000101C000010A83A00102000001024000010280000102C0000103000001030
:40C4400034000010380000103C000010FC3B00104000001044000010700800208408002098080020AC080020FFE71421044885F06EFD2620FFF733FE10BD0248704700009F
:40C48000AC080020C0080020F0EE401A02EE101AB8EE422ADFEDFE2A82EE223AB0EE430A90ED142AD0ED062A9FEDFA3A62EE832A00EE222A80ED142A90ED122AD0ED132AB4
:40C4C00002EE802AD0ED112A72EE222A90ED152A02EE802AD0ED102A32EE222A80ED102A90ED112AD0ED132A02EE802A80ED112A90ED122AD0ED132A02EE802A80ED122AB4
:40C5000090ED132AD0ED162A32EE222A80ED132A90ED102AD0ED172A32EE222AD0ED102A82EE823AF0EE430A90ED102AD0ED172A32EE222AD0ED122A82EE823AB0EE431A7E
:40C5400090ED102AD0ED102A00EEE22A80ED102A90ED112AD0ED112A00EEE22A80ED112A90ED122AD0ED102A01EE622A80ED122A90ED132AD0ED112A01EE622A80ED132A6F
:40C5800090ED142AD0ED0E2A9FEDC23A12EE832AD0ED142A40EE822AC0ED142A90ED142AD0ED0E2A9FEDBB3A12EE832A61EE812A62EE222A90ED072A9FEDB73A03EE622ABA
:40C5C00080ED072A90ED142AD0ED1A2A9FEDB13A02EEC32AF6EE002A62EE222A90ED1A2A9FEDAD3A03EE222A80ED1A2A7047AB4800687047AA480068704770B52DED028B1B
:40C60000A84800685DF05BFE05469FEDA70A10EE104A09F0D7FAA3490860FFF7E8FF962807DAB2EE048AA14890ED020A80ED070A1FE09E4890ED060AB0EEC00ADFED9C0A18
:40C64000B4EEE00AF1EE10FA11D2FFF7D3FF00EE100AB8EEC00AB0EEC00ADFED960AB4EEE00AF1EE10FA02D2B7EE008A01E09FED8E8A91480068D0ED000A8F4890F90400E5
:40C6800000EE100AB8EEC00A20EE800A8A4880ED020A90ED020AD0ED040A20EE200AD0ED030A864890ED061A00EE810A8248D0ED050A7E4890ED061A00EE810A7E48D0EDF0
:40C6C000070A30EE600A10EE104A204687F00DFC08B979488461784890ED0F0A006A90ED001A754890F9240000EE900AF8EEE00A11EE200A704880ED0A0AD0ED0A0AB0EE12
:40C70000600A87F092FBDFED640A20EE200A6A48D0ED0C0A20EE200AD0ED0B0A674890ED0E1A00EE810A6448D0ED0D0A5F4890ED0E1A00EE810AFFF75AFF00EE900AF8EEBB
:40C74000E00A5A4890ED061A60EE810A9FED5C1AC0EE811A30EE210A10EE104A204687F0C4FB08B954488463B0EE480A29465248FFF78AFE51480068D0ED000A4F4890F98C
:40C78000040000EE100AB8EEC00A20EE800A4B4880ED020A90ED020AD0ED030A20EE200AD0ED040A444890ED061A00EE810A4348D0ED050A3D4890ED061A00EE810A3E48E9
:40C7C000D0ED070A30EE600A10EE104A204687F08CFB08B939488461384890ED0F0A006A90ED001A354890F9240000EE900AF8EEE00A11EE200A314880ED0A0AD0ED0A0A73
:40C80000B0EE600A87F011FBDFED230A20EE200A2A48D0ED0B0A20EE200AD0ED0C0A264890ED0E1A00EE810A2448D0ED0D0A1F4890ED0E1A00EE810A10EE104A204687F067
:40C8400054FB08B91D488463B0EE480A29461B48FFF71AFE15480068D0ED000A134890F9040000EE100AB8EEC00A20EE800A0F4880ED020A90ED020AD0ED050A20EE200AAB
:40C88000D0ED030A0D4890ED061A00EE810A19E000007A4439FA8E3CE12E65425400001058000010640000100000000000220010E12EE5410000964394210010282100103B
:40C8C00000481946FE48D0ED040AFE4890ED061A00EE810AFA48D0ED070A30EE600A10EE104A204687F001FB08B9F5488461F448D0ED0F0A006A90ED001AF14890F924007F
:40C9000000EE100AB8EEC00A51EE000AEC48C0ED0A0AD0ED0A0AB0EE600A87F086FA5FED220A20EE200AE648D0ED0D0A20EE200AD0ED0B0AE44890ED0E1A00EE810AE04843
:40C94000D0ED0C0ADF4890ED0E1A00EE810A10EE104A204687F0C9FA08B9D9488463BDEC028B70BD70B5044609F02CF90546D748016828465DF0B3FCD5490968611A4FF464
:40C980007A725143B1FBF0F0D2490860D048046009F018F9CD4908600521CF48006887F06DFE90BBCD48016828465DF098FCB0F57A7F01D9C9480560C848016828465DF023
:40C9C0008EFC60434FF47A71B0FBF1F0C44AD2E90032C01842F10001C14A03C200BFC048D0E90021BF48C0E90221082200F10801BD48FEF775FD00BFB84805600920FFF732
:40CA00006EFBB548006887F02DFE70BD70B504460025B6488078A04204D0B44884700720FFF75DFB284670BD70B504460025AF48007BA04204D0AD4804730820FFF74FFB89
:40CA4000284670BDA948807870472DE9F04F8BB0A7488468A7488768A748D0F80890A748D0F80880A24840680A90A24840680990A14840680890A148406807909C48007B9D
:40CA800006909C48007B05909B48007B04909B4890F80CB080780390FE20029007200190002000900398082828D2DFE800F00E041824252727264FF6FF20804504D847463B
:40CAC00007980990CDF814B018E04FF6FF20804504D8444607980A90CDF818B00EE04FF6FF20804506D8C14607980890CDF810B00120009002E000BF00BF00BF00BF4FF69C
:40CB0000FF20814525D8009810B9B9F5807F06D8009801281DD140F21510814519D94D46009880B900EE105AB8EE400ADFED740A20EE200ABCEEC00A10EE105AB5F57B4FEB
:40CB400001D34FF6FF25089E04980290022001904CE04FF6FF20844208D8874206D925460A9E06980290002001903FE04FF6FF20874208D8844206D93D46099E05980290F5
:40CB80000120019032E04FF6FF20874205D9844203D900250720019028E000EE104AB8EE400ADFED580A20EE200ABCEEC00A10EE10AA34B925460A9E069802900020019074
:40CBC00014E0A4EB0A00B8420AD204EB0A00B84206D93D46099E059802900120019005E025460A9E0698029000200190FFF72AFF0199884203D13D484068B0420AD0029832
:40CC0000FFF712FF0198FFF701FF384846602846FFF7A8FE0BB0BDE8F08F10B504463A480078844204D0384804700520FFF757FA10BD0146002200200AE0344B53F82030F2
:40CC400023B9324B43F82010012203E0431CD8B20828F2DB1046704730B503460024002017E02A4D55F820508DB1284D55F820502D7B9D420BD1254D55F820502D888D42D4
:40CC800005D1224D55F820501560012403E0451CE8B20828E5DB204630BD2DE9FC470546002600270020019028461AF0EEFB044628688169284688471FFA80F8286827E08B
:40CCC0000022001094210010282100106C00001054000010580000106000001068000010480000102008002008750068D8200010F8200010E8200010082100101821001065
:40CD00008AE38A3FCDCCCC3E5C000010B82000106946C268284690474FF6486084420AD0401C844207D04FF6E860844203D04FF22200844225D128461AF0DDFB814601AA1B
:40CD40002146FFF789FFE0B928686946C26828469047012815D1B8F1080F12DB102087F085F8019028461AF0C6FB0199087301990C80F9480078401CF74908700198FFF746
:40CD800058FF0198002867D0A4F570402238002847D0A0F6266020B101281CD0A02858D12CE008F00FFFED494860009800780099497840EA0120E949886028461AF09BFB82
:40CDC000E64908730098C079C0F381073846FFF724FF01263FE008F0F5FEE1494860009800780099497840EA0120DD49886028461AF081FBDA49087301262CE008F0E2FE83
:40CE0000D8494860009880780099C97840EA0120D449886028461AF06EFBD2490873012619E008F0CFFED0494860009800780099497840EA0120CC49886028461AF05BFBD2
:40CE4000C94908730098C079C0F382008870012601E0002600BF00BF012E07D1C348006A20B1C249086A012187F02CFCBDE8FC879FEDBF0ABF4880ED030AB7EE000A80EDD6
:40CE8000040A9FEDBB0A80ED050A9FEDB90A80ED0B0AB7EE000A80ED0C0A9FEDB50A80ED0D0A9FEDB30A80ED140A9FEDB30A80ED150A9FEDB20A80ED160AB1EE000A80ED31
:40CEC000170AB7EE000A80ED100A9FEDA90A80ED110A9FEDA70A80ED120A9FEDA50A80ED130AB7EE000AA64880ED030A9FEDA00A80ED040A9FED9E0A80ED050AB7EE000A62
:40CF000080ED0B0A9FED9A0A80ED0C0A9FED980A80ED0D0A9FED960A80ED140A9FED960A80ED150A9FED950A80ED160AB1EE040A80ED170AB7EE000A80ED100A9FED8C0A50
:40CF400080ED110A9FED8A0A80ED120A9FED880A80ED130A9FED860A8A4880ED030A9FED840A80ED040AB7EE000A80ED050A9FED800A80ED0B0A9FED7E0A80ED0C0AB7EEDC
:40CF8000000A80ED0D0A70470EB501247E4887F045FB7E49086008F015FE05460321734880F82510FFF764FF0022AFF211314FF2220021F042F90022AFF221314FF64860A7
:40CFC00021F03BF90022AFF22D314FF6496021F034F90022AFF23D314FF6E86021F02DF900BF4FF0FF31002087F078FB8DE80700009840281CD00098082819D1019800F4CB
:40D00000804080B10021594880F825100020574908625E48006887F019FB87F08FFB064687F0A4FB04E0019800F0010000B101244A48007BFF280DD04849486840F2DC5175
:40D040005DF016F930B1FF20444908734FF6FF70886001244248007BFF280DD04049486840F2DC515DF004F930B1FF203C4908734FF6FF70886001243A48007BFF280DD0DE
:40D080003849486840F2DC515DF0F2F830B1FF20344908734FF6FF70886001243248007BFF280FD03049486840F2DC515DF0E0F840B1FF202C4908734FF6FF708860072085
:40D0C00088700124012C06D1FFF7BFFC002408F079FD05460BE04FF4FA6128465DF0C8F828B10020FFF73EFC08F06CFD0546FFF784FA76E77047704770B505460026062DA0
:40D1000029D2DFE805F003476F99C3ED00241FE0E0B2FFF7F0FF1B48006AD0ED000A194890F9240000EE100AB8EEC00A20EE800AF6EE000AB4EEE00AF1EE10FA06DBE1B213
:40D140000022134812F0F8FA012603E0601CC4B2042CDDDB00BFEDE05E000010F8200010E82000100821001018210010300A0020000000009421001017B7D13895BFD6334B
:40D180002821001000220010B8BE090860000010E0390010002421E0211DC8B2FFF7ABFFA448006AD0ED000AA24890F9240000EE100AB8EEC00A20EE800AF6EE000AB4EEF3
:40D1C000E00AF1EE10FA07DB201DC1B200229A4812F0B2FA012603E0601CC4B2042CDBDB00BFA7E0002423E004F10801C8B2FFF782FF9048006AD0ED000A8E4890F924004E
:40D2000000EE100AB8EEC00A20EE800AF6EE000AB4EEE00AF1EE10FA08DB04F10800C1B20022854812F088FA012603E0601CC4B2042CD9DB00BF7DE0002423E004F10C0190
:40D24000C8B2FFF758FF7B48006AD0ED000A794890F9240000EE100AB8EEC00A20EE800AF6EE000AB4EEE00AF1EE10FA08DB04F10C00C1B20022704812F05EFA012603E07D
:40D28000601CC4B2042CD9DB00BF53E0002423E004F11001C8B2FFF72EFF6648006AD0ED000A644890F9240000EE100AB8EEC00A20EE800AF6EE000AB4EEE00AF1EE10FA31
:40D2C00008DB04F11000C1B200225B4812F034FA012603E0601CC4B2042CD9DB00BF29E0002423E004F11401C8B2FFF704FF5148006AD0ED000A4F4890F9240000EE100A7C
:40D30000B8EEC00A20EE800AF6EE000AB4EEE00AF1EE10FA08DB04F11400C1B20022464812F00AFA012603E0601CC4B2042CD9DB00BF00BF00BF304670BD10B53E4812F060
:40D34000F7F90446C01704EB9070801010BD70B500210C460D4601213848006887F08EF928B9374830C83548006887F07BF92046294670BD70B504460D46072601212F48AB
:40D38000006887F07BF9B0B92D4830C000BF0838D0E900202B49C1E90220082208312A48FEF79EF800BF00262448006887F05AF90920FEF794FE304670BD244890ED1A0AF1
:40D3C0007047224890ED190A7047214890ED1A0A70471F4890ED190A70471E48007B70471D480068704770B5044600251A480068A04204D0184804600620FEF770FE28464B
:40D4000070BD1FEDA50A70470A4890ED190A704712480078704770B5044600250F480078A04204D00D4804700420FEF758FE284670BD000000220010E03900106000001064
:40D440004800001020080020087500682821001094210010D8200010500000105D00001030B52DED028B83B09FED960AF0EE408A002008EE100A002402AA0021924811F0A5
:40D480008AFD20B102985BF014FBF0EE408A01A98D4812F08EFC20B101985AF0EDFC08EE100A69468948FCF734F828B1009800684169009888470446834812F041FA00EEF7
:40D4C000100AB8EE400ADFED820A80EE201A11EE105A28468EF072FC7E4A03C27A4812F048FA00EE100AB8EE400ADFED790A80EE201A11EE105A28468EF060FC754AC2E9C2
:40D500000401714812F04EFA00EE100AB8EE400A704880ED020A6C4812F05DFA00EE100AB8EE400ADFED6C0A80EE201A694880ED061A654812F0CFFA664981F82000624823
:40D5400012F0F4FC00EE100AB8EE400A614880ED070AC0ED0A8AB8EE480A80ED0B0A80F83040594812F050FA05468EF006F95B4A03C2554812F061FA05468EF0FEF8574A7E
:40D58000C2E90201504812F071FA05468EF0F5F8524AC2E904014C4812F084FA05468EF0ECF84E4AC2E906019FED4D0B4E4880ED000B9FED4E0B80ED020B9FED4E0B80ED08
:40D5C000040B9FED4E0B80ED060B03B0BDEC028B30BD10B5FFF744FF4A4877F06BFF10BD0EB502A93948FBF79CFF68B301A93748FBF79FFF40B369463448FBF7A2FF18B3E9
:40D600004148007808B1012000E00020014602980068826A029890473B48407808B1012000E00020014601980068826A019890473548807808B1012000E000200146009882
:40D640000068826A0098904730480078012807D12D48C07820B9002211461B4812F03FFA2948C078294908700EBD10B5FFF7F8FE254A1849234877F09AFFFFF7B1FF10BD9C
:40D680002148007808B1012070470020FCE71E48407808B1012070470020FCE71A48807808B1012070470020FCE77047704710B5144879F02EF80446154A164984F0D4FAED
:40D6C00010BD000000000000E0390010D403002000007A44F80900208FC2753D802000100000000000C05240602000100000000000004940000000000000394000000000C7
:40D7000000000000D8080020700000107400001000800008156708080246012053798B4200D05171704710B504460020207100212046FFF7F1FF0020083460762076A08071
:40D74000A076E0762077E0602082606154F8080920B1A06886F081FB0020A060206920B1206986F07AFB0020206110BD70B504460D4625602046FFF7D6FF204670BD10B5AF
:40D780000446A06820B1A06886F067FB0020A060204610BD024600201171704701460879704710B50346002093F82140012C00D10220012403F8214F59709A70213B10BD2D
:40D7C000014691F82000704701464879704730B5044600252046FFF7F7FF20B901212046FFF79AFF0125284630BD30B5044600252046FFF7E9FF042804D103212046FFF793
:40D800008BFF0125284630BD2DE9F04104460D46002700262046FFF7D7FF04281FD1206920B1206986F019FB00202061284684F09BFA00F10108404686F013FB064628461B
:40D8400084F092FA00F1010842462946304684F0C7FB266106212046FFF75EFF01273846BDE8F0812DE9F04104460D46002700262046FFF7A9FF04281FD1206920B12069B4
:40D8800086F0EBFA00202061284684F06DFA00F10108404686F0E5FA0646284684F064FA00F1010842462946304684F099FB266107212046FFF730FF01273846BDE8F0815D
:40D8C00030B5044600252046FFF77EFF092804D10B212046FFF720FF0125284630BD2DE9F04105460F464FF00008002400262846FFF76AFF042817D101E0601C84B2385D4C
:40D900000028FAD1204686F0ACFA064666B122463946304684F09CFA0C212846FFF7FCFEAE60AC814FF001084046BDE8F0812DE9F04105460F464FF0000800240026284618
:40D94000FFF742FF09281ED1A868E0B901E0601C84B2385D0028FAD1601C84B2204686F080FA06467EB122463946304684F070FA2C21601E3154AE60AC810A212846FFF7B4
:40D98000CBFE4FF001084046BDE8F0812DE9F04104460F464FF00008002500262046FFF713FF09281CD1A068D0B90B2086F059FA05463B46F7A20B21284683F073FFC6B2D5
:40D9C0000B2E0DDC65B1002E0ADD2C21701E2954A560A6810A212046FFF79EFE4FF001084046BDE8F08130B5044600252046FFF7EBFE09280ED1A06860B92046FFF7E0FE4B
:40DA000040B9E548A0600120A0810A212046FFF783FE0125284630BD2DE9F04105460F464FF00008002400262846FFF7CDFE09281DD1A868D8B901E0601C84B2385D00283E
:40DA4000FAD1601C84B2204686F00BFA064676B122463946304684F0FBF90A21601E3154AE60AC812846FFF757FE4FF001084046BDE8F0812DE9F04104460D4616461F4665
:40DA80004FF000082046FFF79FFE09280FD175B1002E0CDD5FB165612683E7610020E169088008212046FFF737FE4FF001084046BDE8F0812DE9F04104460F4615464FF001
:40DAC000000800262046FFF77FFE092813D1A06888B9284686F0C5F9064666B12A463946304684F0B5F9A660A5810A212046FFF713FE4FF001084046BDE8F0812DE9F04344
:40DB00000546894614461E46079FB846012C03D129464046FFF73EFE324621464046FFF740FEBDE8F0832DE9F05F06468B4614461F46DDE90B8ADDF828905546012C0BD1C3
:40DB400031462846FFF726FEE869A0F8008042464946686984F07CF93A4621462846FFF720FEBDE8F09F10B586B004468BA0006805908BA207CA02AB07C3206820B900216B
:40DB80002046FFF7C9FDDEE0206826F02CF820B900212046FFF7C0FDD5E094F821000128F1D1002084F8210084F820002046FFF70BFE0F2816D2DFE800F0C1C00816BF244D
:40DBC000323380C3559BA9C2C40094F82200012804D103212046FFF79FFD03E00D212046FFF79AFDAEE094F82200012804D104212046FFF791FD03E005212046FFF78CFD5B
:40DC0000A0E094F82200012804D103212046FFF783FD03E00D212046FFF77EFD92E000BF94F8220001280ED109212046FFF774FD206920B1206986F010F9002020610020CF
:40DC400084F824000DE094F82400052805DA94F82400401C84F8240003E00D212046FFF75BFD6FE094F8220001280FD1A06828B1A06886F0F2F80020A060A08109212046CA
:40DC8000FFF74AFD002084F8240015E094F82400052805DA94F82400401C84F824000BE0A06828B1A06886F0D8F80020A060A0810D212046FFF730FD44E094F822000128FD
:40DCC00007D109212046FFF727FD002084F824000DE094F82400052805DA94F82400401C84F8240003E00D212046FFF715FD29E094F82200012804D104212046FFF70CFDCF
:40DD000003E00D212046FFF707FD1BE094F82200012804D104212046FFF7FEFC03E00D212046FFF7F9FCA06828B1A06886F095F80020A060A08105E000BF00BF00BF00BFE0
:40DD400000BF00BF00BF94F8200000287AD12046FFF73AFD0F280AD2DFE800F0090A0F2DCA3E4F6492CB7AA6B7CC080000BFC2E002212046FFF7D0FCBDE0AFF27F232246E4
:40DD800005A9206825F0D7FF80B1012084F8200010E0000025750000750000105C0000002E5C4D434D43303135315C000D212046FFF7B2FC9FE0AFF2BB23224602A920684B
:40DDC00025F0B9FF18B1012084F8200003E00D212046FFF7A1FC8EE0AFF2DF23224602A9206826F0C8F918B1012084F8200003E00D212046FFF790FC7DE0206968B1AFF224
:40DE000003300090234606222169206825F0F5FF18B1012084F8200003E00D212046FFF77BFC68E0206970B1AFF22F300090234603222169206825F0E0FF20B1012084F885
:40DE4000200004E058E00D212046FFF765FC52E0A068A0B1A08990B1AFF25F30CDE90040A389211DA268206826F0A2F818B1012084F8200003E00D212046FFF74DFC3AE05E
:40DE8000AFF25D30CDE90040238B211D6269206826F0D4F818B1012084F8200003E00D212046FFF739FC26E0AFF2AF332246211D206825F0F9FF18B1012084F8200003E0C8
:40DEC0000D212046FFF728FC15E0AFF2CF30009023460022A168206826F0AEF918B1012084F8200003E00D212046FFF715FC02E000BF00BF00BF00BF06B010BD10B5044602
:40DF0000206825F070FE10BDF8B50746002405E0774800EBC4000471601CC4B2142CF7DBFDF715FD73480068804705460AE04A2006F08BF918B10A2086F0A2FA02E007F038
:40DF400041FE054628465CF0BAF9B0F5FA6FEED306F008FEFDF770FD10B90020FCF778FD0DF0F5FF644886F095FB644908600021634886F0BFFB5E49886507E0642086F004
:40DF80007FFA6048006864305E490860584890F85D000B2805DA5B48006842F210718842ECD301220021B52006F0F4F904F0C2F9FAF784FE0021544886F09CFB4C498861EF
:40DFC0000021524886F096FB494908610021504886F090FB4649886000214E4886F08AFB4349886700214C4886F084FB4049086600214A4886F07EFB3D498866002148489E
:40E0000086F078FB3A4908650021464886F072FB374908630021444886F06CFB344988620021424886F066FB314908620021404886F060FB2E49886400213E4886F05AFBE4
:40E040002B49C1F8800000213B4886F053FB2849C1F888000021394886F04CFB2449C1F890000021364886F045FB2149C1F898006846FBF7CBFA28B10021324886F03AFB30
:40E080001B49086700201A49886386F057FB064686F06CFBF8BD10B50021194886F02AFB1349886510BD10B51148006C28B90021254886F01FFB0E49086410BD10B5002182
:40E0C0001E4886F017FB0A49C1F8900010BD10B50748006A50B1064890F82500032805D10349086A4FF4004186F0ECFA10BD0000300A00200820001004C0090878000010F4
:40E10000E0C009087C00001030C0090820C0090810C0090840C00908D0C00908F0C00908C0C00908A0C00908B0C0090890C0090800C1090860C0090850C0090870C0090813
:40E1400080C0090820C1090810C1090810B578F09EFE04462CB106F0ECFA0020F749087002E00120F5490870204610BD2DE9F0472DED028B04460027204678F0ABFE00F01E
:40E18000FF08B8F1560F79DA20688168204688471B2874D2DFE800F00E1420262C327338FD43494F555B736174B2C3D4FCFBFAF9F8F7F6000021404608F024F907464CE182
:40E1C000B8F1510F07DBB8F1550F04DC0121404608F018F9074640E10321404608F012F907463AE10421404608F00CF9074634E10121404608F006F907462EE10221404665
:40E2000008F000F9074628E140460EF04FFAB0F1FF3F01D0012000E0002007461DE10A21404608F0EFF8074617E10921404608F0E9F8074611E10B21404608F0E3F807463F
:40E240000BE10621404608F0DDF8074605E10721404608F0D7F80746FFE00C21404608F0D1F8074625462068416A20468847064628683146826A28469047EEE0EEE0EBE0E5
:40E2800040460DF089FF81460F21404608F0BAF80746AB4800EB890090ED000AB5EEC00AF1EE10FA0DD02068416B20468847A44800EB8900D0ED000AB4EE600AF1EE10FA39
:40E2C00001D1012000E00020074025462068416B20468847B0EE408A2C462868816B2846884726462068C16A20468847B0EE408A34463068016B30468847AEE00D214046BC
:40E3000008F080F8074625462068416A20468847064628683146826A284690479DE00E21404608F06FF8074625462068416A20468847064628683146826A284690478CE028
:40E3400040460DF029FF81461021404608F05AF807467B4800EB890090ED000AB5EEC00AF1EE10FA0DD02068416B20468847744800EB8900D0ED000AB4EE600AF1EE10FA97
:40E380000AD107E067E065E063E061E05FE05DE01DE05AE0012000E00020074025462068416B20468847B0EE408A2C462868816B2846884726462068C16A20468847B0EE17
:40E3C000408A34463068016B3046884745E040460EF05BF881461121404608F013F80746574800EB890090ED000AB5EEC00AF1EE10FA0DD02068416B20468847504800EB0C
:40E400008900D0ED000AB4EE600AF1EE10FA01D1012000E00020074025462068416B20468847B0EE408A2C462868816B2846884726462068C16A20468847B0EE408A3446C0
:40E440003068016B3046884707E000BF00BF00BF00BF00BF00BF00BF00BF00BF3846BDEC028BBDE8F08770B50446204678F032FDC5B20021284607F0C5FF70BD002008E083
:40E480009FED300A2E4901EB800181ED000A411CC8B20F28F4D3704710B50446E0B20EF0D2F810BD10B50446E0B20EF0C8FC10BD10B50446E0B20EF0F9F810BD10B50446DC
:40E4C000E0B20EF0D5FF10BD70B504460D46E0B229460DF0BFFD70BD10B52DED028B0446B0EE408AE0B2B0EE480A0DF0C6FDBDEC028B10BD10B52DED028B0446B0EE408AC1
:40E50000E0B2B0EE480A0DF01BFEBDEC028B10BD70B504460D46E0B229460DF0EDFE70BD10B52DED028B0446B0EE408AE0B2B0EE480A0DF0F4FEBDEC028B10BD190000209D
:40E54000DC1200200000000010B52DED028B0446B0EE408AE0B2B0EE480A0DF06AFFBDEC028B10BD01480078704700001900002010B5002807DA0A07140E7C4A00F00F030A
:40E580001B1FD45403E00A07130E794A135410BD784A0168116001791171704710B57648764908604FF4E13048604FF44071734881610C21416100210161C1608160C161F1
:40E5C00081F057FF6E486F4908604FF00060486040216C4881600021C1604FF480610161002141618161C1614FF40031016200214162032181624FF40001C16289100163AC
:40E600007BF0D8F900BF5F485C49086308465D49886300BF00210E20FFF7AAFF0E2000F099F80D212720FFF7A3FF272000F092F801225549514882F07DF910B1012053495F
:40E64000087010BD10B54F487BF00BFC10BD10B54A4882F0D8FD10BD10B501224A49474882F068F9044614B1012048490870204610BD10B5044646480078012826D10020B1
:40E6800007E0444909880144434A515C1154411C88B2424909883F4A1288891A8142F0DC3E4800883B490988401A3C49088000203849088039480088C0F1800200213648DB
:40E6C000803083F03CFC0020314908702E480178324802880088401C304B18802E48815418460088802802DB00201946088001F0FBFE1B2806D02A49D1F88000032185F0AE
:40E70000E1FF05E02649D1F88800022185F0DAFF01221D49194882F00DF910B101201B49087010BD704710B504461E4801F0EAFC022805DB1A49D1F88000022185F0C2FFE4
:40E7400010BD70B504460D462A4621460B4882F08AF970BD00F01F02012191404209920002F1E022C2F800117047000018ED00E000E400E0B81300200048004018130020FF
:40E7800058600240581300201A0000201B0000201E0100201A010020D813002018010020300A00207C2200107CB505460E461DB1052D01D0042D02D10020401C00BFFA219E
:40E7C000FC48006885F05AFF60BBFB480088ADF804008DF806508DF80760F84C0198009004F10800216800EB8100009901602068401C01462060204685F0F2F82060D4E943
:40E800000001884202D16068401C00E06068606000BFE848006885F025FF0221E8485BF018FB00BF7CBDE74A116070472DE9F04786B00446E448007800F0010070B9E24807
:40E8400085F06CFB50B1E1484FF040FF0646E04AE04983F009FADC48AFF30080DE48007800F0010070B9DC4885F058FB50B1DB484EF02CFA0646D64AD94983F0F5F9D64880
:40E88000AFF30080D748007800F0010070B9D54885F044FB50B1D4484EF0E8FF0646CC4AD24983F0E1F9CF48AFF30080D048007800F0010070B9CE4885F030FB50B1CD48F9
:40E8C00057F07DFE0646C24ACB4983F0CDF9C848AFF30080C948007800F0010070B9C74885F01CFB50B1C6484DF0ABFB0646B84AC44983F0B9F9C148AFF30080C248007822
:40E9000000F0010070B9C04885F008FB50B1BF484CF01AFC0646AE4ABD4983F0A5F9BA48AFF30080BB48007800F0010070B9B94885F0F4FA50B1B84858F086FC0646A44A66
:40E94000B64983F091F9B348AFF3008000270025A846A946AA46002000902078002871D10090607807286ED2DFE800F00495FEFDFCFBFA00AA4800688047064631469048E4
:40E980001438FFF750FF142101A883F002FB1422A11D01A883F05CFA0020A2490870A078E17840EA0120844908802079617940EA01209D4908809D48007D30B914229B49ED
:40E9C00001A883F0FAF9002850D0994A694601A850F09BFA80B1964800680068C16894480068884793490860934B52460921744814385BF003FB2CE050F09FF9322823D22D
:40EA000072484FF07EFF8C4B142201A96F484FF043FF6E4856F019FD70B1032000906B484FF0A6FE83490860834B52460A21644814385BF0E3FA0CE004200090401F7D494B
:40EA4000086006E0F3E3F3E305200090801F79490860744801789DF80000FFF7A5FE4FF0FF30764908607649086007E0022000906C4801789DF80000FFF796FE14216B4832
:40EA800083F087FA142201A9684883F026FA0020664908753EE26248006880470646314647481438FFF7BFFE142101A883F071FA1422A11D01A883F0CBF9012059490870DE
:40EAC000A078E17840EA01203B4908802079617940EA01205449088056480068B0F1FF3F66D05248007D012806D114224F4901A883F063F900285BD0524B6A464D48016855
:40EB000001A84EF08EFD80B14E4800680068C1684C480068884749490860474B52460B21274814385BF06AFA37E04EF090FCB0F5FA7F2DD229484EF005FA3F4B142201A908
:40EB400026484EF0B7F93C4A3A48016823484EF0D8F9224856F079FCA0B10320009004E067E391E2D7E12EE183E01C484EF000F932490860304B52460C21114814385BF0AC
:40EB80003DFA0AE004200090401F2C49086004E005200090801F29490860224801789DF80000FFF701FE4FF0FF302549086053E04AE000001C00002022000020BC220010B8
:40EBC000902200102800002064000020E023001000800008F3E60508600000200C240010F3CC05085C0000203C24001093D805085800002084240010E5650608540000201A
:40EC0000B824001069C0050850000020EC2400106FB105084C000020282500106F720608082000104800002024000020582500106800002084000020BB3C090888000020F0
:40EC40008C0000206C00002002200090FE4801789DF80000FFF7A8FD1421FC4883F099F9142201A9F94883F038F90120F74908756FE3F7480068804706463146F548FFF7E4
:40EC8000D2FDA079E17900EB0120217A00EB0140617A00EB0167142101A883F07AF9142204F10A0101A883F0D3F80220E6490870A078E17840EA0120E74908802079617980
:40ECC00040EA0120E5490880E5480068B0F1FF3F64D0DE48007D022806D11422DB4901A883F06BF8002859D0DE4B6A46DC48016801A84FF0BDFBF8B1DA4800680068816A11
:40ED0000D848006888470646B7420ED0D5480168D5484EF05BFFD54A3946D3484EF027FFD0480168D04856F0F4FCD04B52460D21C8485BF063F92AE04FF0C6FAB0F57A7FF3
:40ED400023D2C9484EF034FFC84A3946C6484EF00EFFC64B142201A9C3484EF0A7FEC34ABF480168C0484EF0EFFEBF4856F06DFB40B103200090BD4B52460E21B5485BF033
:40ED80003DF904E00420009001E005200090AE4801789DF80000FFF707FD07E002200090A94801789DF80000FFF7FEFC1421A74883F0EFF8142201A9A44883F08EF8022004
:40EDC000A2490875C5E2A2480068804706463146A048FFF728FDA079E17900EB0120217A00EB0140617A00EB016564204543142101A883F0CEF8142204F10A0101A883F03E
:40EE000027F8032090490870A078E17840EA0120914908802079617940EA01208F4908808A48007D032806D11422884901A882F0C4FF00285AD08E4A694601A858F0EEF81D
:40EE400048B38B4800680068016A89480068884706466420B6FBF0F0301AA84205D26420B6FBF0F03044A8420ED881480168814857F011FD7D4A29467E4857F0CAFC7C489F
:40EE800001687C4856F0A7FE784B52460F2171485BF0B4F823E057F0EFFF32281DD2754857F0EBFC714A2946724857F0B2FC6F4B142201A96F4857F085FC6E4856F0C5FAE6
:40EEC00040B103200090694B5246102161485BF095F804E00420009001E0052000905A4801789DF80000FFF75FFC07E002200090554801789DF80000FFF756FC14215348E5
:40EF000083F047F8142201A9504882F0E6FF03204E4908751DE24E4800688047064631464C48FFF780FCA079E17900EB0120217A00EB0140617A00EB0165142101A883F0C9
:40EF400028F8142204F10A0101A882F081FF04203D490870A078E17840EA01203E4908802079617940EA01203C4908803748007D042805D11422354901A882F01EFFE8B363
:40EF80003D4A694601A84DF08BFDF0B13A4800680068016A384800688847A8420ED03648016836484DF0B9F9304A294633484DF072F931480168314856F070FE2B4B524653
:40EFC000112124485BF01AF825E04DF097FC32281FD22A484DF093F9244A294627484DF05AF9224B142201A924484DF02DF9234856F02BFA50B10320009000E012E01B4B01
:40F000005246122113485AF0F9FF04E00420009001E0052000900C4801789DF80000FFF7C3FB07E002200090074801789DF80000FFF7BAFB1421054882F0ABFF142201A905
:40F04000024882F04AFF1BE04800002058250010082000107C220010220000202400002088000020700000203C240010BB3C0908740000208424001078000020B8240010AF
:40F080000420F949087564E1F8480068804706463146F748FFF7C7FBA079E17900EB0120217A00EB0140617A00EB0168A07AE17A00EB0120217B00EB0140617B00EB016910
:40F0C000142101A882F065FF142204F10F0101A882F0BEFE0520E7490870A078E17840EA0120E54908802079617940EA0120E3490880DD48007D052806D11422DA4901A8F1
:40F1000082F05BFE00287DD0DD4A694601A84CF072FEB8B3A07B28BBD94800680068016AD74800688847404508D1D54800680068416AD34800688847484513D0D048016810
:40F14000D0484CF0B7F9D04A4146CE484CF048F9CD4A4946CB484CF056F9C9480168C94856F0C1FCC84B52461321C1485AF046FFC34800680068C168C14800688847C349BE
:40F18000086038E0FFE74CF062FD19282ED2A07B58BBBC484CF080F9BB4A4146B9484CF01FF9B94A4946B7484CF02DF9B64B142201A9B4484CF0EDF8B24856F046F968B1BC
:40F1C00003200090AF484CF011F8B0490860AE4B52461421A6485AF011FF0CE004200090401FAA49086006E00CE0FFE705200090801FA64908609F4801789DF80000FFF709
:40F20000D3FA07E0022000909A4801789DF80000FFF7CAFA1421944882F0BBFE142201A9914882F05AFE05208F49087591E092E07FE08E4800688047064631468C48FFF7B1
:40F24000F2FA142101A882F0A4FE1422A11D01A882F0FEFD062087490870A078E17840EA0120854908802079617940EA01208349088086480068B0F1FF3F45D07A48007DAB
:40F28000062805D11422784901A882F096FD70B37F4B6A467D48016801A858F07EFC30B1794B5246152172485AF0A8FE25E058F08BFB64281FD2774858F002F9724B14220D
:40F2C00001A9744858F0B4F86F4A70480168714858F0D5F86F4856F0B8F848B103200090694B5246162162485AF088FE05E00BE00420009001E0052000905E4801789DF8E8
:40F300000000FFF751FA07E002200090594801789DF80000FFF748FA1421534882F039FE142201A9504882F0D8FD06204E4908750FE0142101A882F02CFE14214A4882F0F8
:40F3400028FE0820484908754FF6FE704A49088000BF00BF00BF00BF06B0BDE8F08701464D48007870470EB501214C4880F88D10032180F88D1000BF3D48FFF7F0FF012871
:40F3800019D1811E4648006885F01AF98DE80700009820280ED1019C3CB12046FFF746FA21463F48006885F0FDF821463C48006885F0F8F8E0E70021384880F875100020E8
:40F3C0003649086785F0BAF9044685F0CFF9D3E770B50546284684F0C9FC022813D1314C204684F0F4FA60B904F10800616800EB8100002101606068411C204684F0F0FA96
:40F40000606000BF00BF70BD10B5044620680169204688470020E06210BD10B50446204684F0A4FC50B1012802D0022808D106E007210F4814305AF00CFD02E000BF00BF18
:40F4400000BF00BF10BD10B50446204684F08EFC50B3012802D0022829D127E00621044814305AF0F6FC23E058250010082000107C2200104800002022000020240000204E
:40F480007C000020EC240010BB3C09088C000020800000202825001020000020300A002044000020BC220010FFE700BF00BF00BF00BF10BD10B50446204684F057FC48B10F
:40F4C000012802D0022807D105E00521F8485AF0C0FC02E000BF00BF00BF00BF10BD10B50446204684F042FC48B1012802D0022807D105E00421EE485AF0ABFC02E000BF24
:40F5000000BF00BF00BF10BD10B50446204684F02DFC48B1012802D0022807D105E00321E3485AF096FC02E000BF00BF00BF00BF10BD2DE9F04FA1B006460F46F5B2B94611
:40F540004FF0000A092D76D2DFE805F0FD05147CC7FCFBFAF900D648143800F0D3FD022803DBD4481CF002FD08B1012000E000208246B0E100201F902090CF4884F027FA0E
:40F5800000285CD13221CD48006885F077F8002855D1C94C0DF178088346204684F017FA48B94FF0010B04F10800616800EB81000068C8F8000000BFBBF1010F3FD101205B
:40F5C0008DF87C009DF87B008DF87D009DF87A008DF87E00BDF87800C0B28DF87F00BDF87800000A8DF88000FF208DF881008DF882008DF88300B148006885F033F8AC48DE
:40F60000143800F07FFD022813DB0020AC490390CDE9040106900620AA49A64A0823CDE9002102901FAA4FF6B221A7481FF001F910B9012001E04DE10020824601E04FF08A
:40F64000010A48E1682107A882F0A3FC08208DF81C00FCF799FE0446142221460DF11D0082F0F6FBFCF7A3FE0446142221460DF1310082F0EDFBFCF7ADFE044614222146CC
:40F680000DF1450082F0E4FBFCF7B7FE0446142221460DF1590082F0DBFB14228B490DF16D0082F0D5FB0020AFF2A3110390CDE904010690062083497E4A6523CDE900215F
:40F6C000029007AA4FF6B0217F481FF0B2F808B9012000E000208246FDE018211BA882F058FC00208DF86C00FCF74EFE834682F03BFB142801D9142004E0FCF745FE8346FA
:40F7000082F032FB0446FCF73FFE8046224641460DF16D0082F09CFB0020AFF23D210390CDE90401069006206649624A1523CDE9002102901BAA4FF6B021634804E0C8E050
:40F740007CE042E008E0C3E01FF073F808B9012000E000208246BEE018211BA882F019FC01208DF86C00FCF722FE834682F0FCFA142801D9142004E0FCF719FE834682F072
:40F78000F3FA0446FCF713FE8046224641460DF16D0082F05DFB0020AFF2E7210390CDE90401069006204749424A1523CDE9002102901BAA4FF6B02143481FF03AF808B92C
:40F7C000012000E00020824685E018211BA882F0E0FB02208DF86C00FCF7FCFD834682F0C3FA142801D9142004E0FCF7F3FD834682F0BAFA0446FCF7EDFD8046224641469F
:40F800000DF16D0082F024FB0020AFF2C5310390CDE90401069006202A49264A1523CDE9002102901BAA4FF6B02127481FF001F808B9012000E0002082464CE018211BA863
:40F8400082F0A7FB05208DF86C00FCF7D6FD834682F08AFA142801D9142004E0FCF7CDFD834682F081FA0446FCF7C7FD8046224641460DF16D0082F0EBFA0020AFF2654159
:40F880000390CDE90401069006200E49094A1523CDE9002102901BAA4FF6B0210A481EF0C8FF08B9012000E00020824613E0000090220010403C0020BC2200101C000020CC
:40F8C000D1F30008C4230010D80100109CBE000800BF00BF00BF00BFBAF1000F04D1294609F114005AF0B5FA21B0BDE8F08F38B50446204600F0B8FB0446FE482060AFF213
:40F90000CD330222082104F1140000945AF0BCF9A0F1140400230D22F74920465AF0EBFA2046FFF771FDF54884F078FEF44908600021F44884F01EFEF3490860204638BD8C
:40F9400010B50446EB48206004F114005AF0C6F9A0F11404204600F096FB0446204610BD70B504462046FFF7EBFF054684F075FA70BD2DE9F04105460C4617461E46002EC3
:40F9800048D00E2E64D1242C20D004DC182C07D0232C3CD10FE0252C23D0262C37D12BE0DA4800F0AFFB022804DB0321D74814305AF04FFA2CE0D54800F0A4FB022804DBEF
:40F9C0000421D24814305AF044FA21E0CF4800F099FB022804DB0521CC4814305AF039FA16E0CA4800F08EFB022804DB0621C74814305AF02EFA0BE0C44800F083FB022857
:40FA000004DB0721C14814305AF023FA00E000BF00BF1EE08A2C0CD08D2C0BD0B02C14D1BB4810F037FB18B92868C168284688470CE000BF0121B54814305AF00AFA03214C
:40FA4000B24814305AF005FA00E000BF00BF00E000BF00BFBDE8F081704710B504466421E06A5AF005FC38B104F114005AF03DF9A84800688047E06210BD70B505460C46EB
:40FA8000284600F03FFBA04213D06C7200231A46042128465AF0B2FA012C08D1002211469B4810F0FBFA00209B49087000E000BF00BF70BD2DE9F04781460D4692461C4600
:40FAC00025F0E0062778607847EA00272CB3072E21D2DFE806F0201D041E1F200C0000BF03218A48FFF7C9FF00BF00BF14E020780006617840EA0140A17840EA0120E1784A
:40FB000040EA01080822211D404600F031FB03E000BF00BF00BF00BF00BFBDE8F08770B504461546084640F08006314621F0E002012A0AD0022A04D0032A07D0042A07D187
:40FB400005E000BF00BF00BF03E000BF00BF00BF00BF00BF70BD714A11707047014670480068704770B505466848FFF7F7FF0446664800F0C7FA012822DB6448FFF7EFFB20
:40FB800001281DD143F6982120465AF071FBB8B104215E48FFF7DFFF40F20D205CF02EFF40F20E205CF02AFF40F20F205CF026FF40F211205CF022FF4FF404705CF01EFFA9
:40FBC00070BD0146574800887047564A118070470146554800887047534A118070470146524800687047514A1160704701465048006870474E4A1160704701464D480068FE
:40FC000070474C4A1160704701464B4800687047494A1160704770B506460C460025204600F0EBFC022000F0EEFC284670BD2DE9F04180460C46002500260027D4F80160E1
:40FC4000D4F80570304600F0CCFC384600F0CFFC012000F0D8FC2846BDE8F0812DE9FC410446002001900027206801A9C2682046904701287ED1204617F007FCA0F57A402E
:40FC8000B138002877D0012803D0B0F5A26F73D11FE10198007800286FD0022802D004286CD1AEE02549086A6FF0010184F052FD2249086E6FF0010184F04CFD1F49886830
:40FCC000002184F047FD1D490869002184F042FD1A49D1F88800002184F03CFD1749D1F88000002184F036FD1449886A012184F031FD25E094CD0F0835C0000868C10908C6
:40FD00001C00002074C10908440000207C220010E03900100820001028010020200000202800002022000020240000202C000020300000203400002038000020300A0020D5
:40FD4000864800688047054629468548FEF76BFD1421844882F0FBF808208249087501988078019AD27800EB022081B27C48FFF72CFF04E0C5E092E0C1E070E08DE001983F
:40FD80000079019A527900EB022081B27448FFF723FF01217248FFF7DEFEFEF78FF94FF6FF7071490880002145F2F82014F014FD43F2794146F66D2014F00EFD6B480188A7
:40FDC00046F66E2014F008FD43F2A64146F66A2014F002FD41F6300146F66C2014F0FCFC40F67C5146F66B2014F0F6FC40F6BC6146F6901014F0F0FC40F2F13014F09EFF4C
:40FE00004BE05748FFF7E4FE06465548FFF7D9FE401C1FFA80F8002E05DD642008FB00F0B0FBF6F500E00025642D01D9642500E000BF642D04D102214948FFF78CFE03E04B
:40FE400003214748FFF787FE00214548FEF7EBFC474B3A46192142485AF0D0F81DE032214448006884F060FB06462068816920468847232804D8206881692046884700E02E
:40FE8000232005462A463046019981F0E1FF31463848006884F09FFB00BF00BF30E0019800780F2812D10198407800F0010060B1002000906A4600212F480FF06CF818B146
:40FEC0002B49009858F05AFE00BF00E000BF00BF16E001980078112802D012280CD105E00199491C1E48FFF7A2FE06E0019841881B48FFF790FE00E000BF00BF00E000BF04
:40FF000000BFBDE8FC817CB51548FFF7F0FC04461A4AAFF2D35181F0A7FE194C002020606060642104F1080082F011F800BF2546124A1449284681F097FE0320124901232C
:40FF4000124ACDE900101946114821F010F804460A4A104981F088FE7CBD0000082000107C2200106D25001022000020F8020020BB3C090844000020E03900100080000866
:40FF8000BC220010FF39090880C109086CC10908C4230010F312030870B50446FE48006820B9FE4884F03AFBFB49086003F07AF8054681F03BFE012060720020F8490870BC
:40FFC0000620F84908800020F7490870F7490870F7490870F7490870F7490880F74908800120F74908700020F6490880F6490870F6490870F6490860401EF64908604FF465
:020000040801F1
:400000007A70F54908800020F4490870F448046000200DE00021F34A1154F34A1154F34A11540022F14B00F140015A54411CC8B24028EFDB1121EE4881F089FF03F032F8C2
:4000400005462B46EBA21121E94881F02BFC2C21EB4881F07CFF2C21EA4881F078FF206881682046884770BD10B50446204659F00FFF0446E44820602046FFF78DFFD848CC
:400080000460204610BD10B50446DF482060C248006818B1C048006884F0D8FA204659F0FDFE0446204610BD70B504462046FFF7EAFF054683F0D1FE70BD70B505460124D8
:4000C00007E0D24B00222146284659F097FF601C84B2072CF5DB70BD70B505460024BB48007868B9B8480078012809D1C8480178BD48FEF726FB18B90120B4490870012469
:40010000204670BD0146487A704770B505460C462846FFF7F7FFA04213D06C7200231A460421284659F06AFF012C08D100221146B8480FF0B3FF00209D49087000E000BF98
:4001400000BF70BD70B58AB004460D46164601202B4622460146CDE9006002A817F030FB02A81EF022F902A817F0CAFB0AB070BD70B58AB004460D46164601202B46224686
:400180000146CDE9006002A817F01AFB02A81EF00CF902A817F0B4FB0AB070BD30B50246002391B18AB18848007870B9002004E0145C8D4D2C54441CE0B28842F8DB9448A1
:4001C00001700120804C20700123184630BD10B502460B460020002100BF04E0545C0444E0B24C1CE1B29942F8DB10BD2DE9F043A1B081460D4616461C464FF00008002E79
:400200003CD0082C3ADC802101A881F0C2FE04F10C0777208DF8040088208DF8050099208DF80600F8B28DF80700FF208DF80800280E8DF80900280C8DF80A00280A8DF82F
:400240000B00E8B28DF80C00224631460DF10D0081F0FEFDFF21F81E01AA1154401C1154781EC1B201A8FFF7B2FF791E01AA5054F9B201A8FFF792FF804600BF404621B0F5
:40028000BDE8F0834A48007870472DE9F041A0B005460C464FF0FF388021684681F079FE00260027002D43D0002C41D0206800283ED020683F283BD221782846FFF787FF7D
:4002C000216868542068401C20607E2238467F1C0DF8002000BF1BE0A85D7E2805D0A85D7D2802D0A85D7C280CD17C2238467F1C0DF80020A85DC043C2B238467F1C0DF8C5
:40030000002004E0AA5D38467F1C0DF80020761C2068B042E0D87D2238467F1C0DF80020276069462846226881F092FD4FF00008404620B0BDE8F0812DE9F043A1B0814691
:400340000D4616461C46DDF8A080002714B3802101A881F01EFE174800788DF804008DF805508DF80660424621460DF1070081F06FFD08F103000090694601A8FFF785FF5E
:40038000002805DB0098C1B201A8FFF707FF0746012F41E047E000001401002098C10908260100202A01002027010020250100202801002029010020180100201A010020FA
:4003C0001E0100201C0100202C0100202D0100203001002034010020380100203A0100203C010020AA14002058140020D8130020EA14002055485020534E25750000000054
:40040000FB14002027150020C4C90F082B3C090824010020E039001004D1FE480078401CFC49087000BF384621B0BDE8F0832DE9F041A2B004460026206821A9C2682046EA
:40044000904700284CD0204617F063F80546802101A881F09EFDFFF715FF01282FD1280E8DF80400280C8DF80500280A8DF80600E8B28DF807002068816920468847074671
:400480003A4602A8219981F0E3FC2068816920468847001DC7B2062141F0200000BF00BF00BF00BF00BF00BF804601AB00224146D94800970068FFF73FFF06460FE0FFF739
:4004C000E1FE60B92068816920468847C7B23B462946D148219A0068FFF788FE064600BF304622B0BDE8F081CC480078704770B504460025C948007884420BD0C74804704F
:40050000C548006830B100232A460121C248006859F074FD284670BD70B504460D460226122D14DC9CB1002004E0215CBC4A1154411CC8B2A842F8DB0020B9494874002302
:400540001A460621B448006859F058FD0026304670BD10B502460023002008701060B0481060002008E0AE4C245C1CB1012311240C7003E0441CE0B21228F4DB184610BD5C
:40058000A8480088704770B504460025FF2C01DD022508E0A348048000232A4602219E48006859F02BFD284670BD9F480078704710B504469C48047000231A4603219648DF
:4005C000006859F01BFD10BD0020704797490870704797490860704795480068704795487047954908607047934800687047934908607047914800687047914908807047ED
:400600008F48008870478F49087070478D480078704710B504462046FFF774FD032805D189480FF037FD08B1012010BD0020FCE72DE9F04781460C4615461E462F784FF003
:40064000000804F47000B0F5700F04D24FF47F4000EA142801E0C4F30F284FF6C170804507D1202F05D1794B00221821784859F0C5FC324629462046FFF764FDBDE8F08738
:400680002DE9FE4F05460C464FF0FF300290002600274FF0000B4FF00008002001900090002D3CD0002C3AD04FF07D094FF0800A52464946204681F076FB8046B8F1000F31
:4006C0002DD0A8EB040000F1010B01270FE0E05D7C2807D17F1CE05DC043C2B23046761C2A5403E0E25D3046761C2A547F1CABF10100B842EBD80020A855701E285C019067
:40070000701EC1B22846FFF762FD00900021701E2954DDE90010884201D1002002900298BDE8FE8F2DE9F04190B005460E4690464021684681F02DFC002400276EB33146C1
:400740006846FFF79DFF002827DB9DF801409DF80270204600F0800119B900BF04F0200040B128680DF103033A462146D0F818C02846E04700BF012020EAD41068B100BF6F
:40078000012020EA941040B128680DF103033A462146D0F81CC02846E04710B0BDE8F0812DE9F047054600261FE12A482A490988445C2A480088402802DB002027490880C4
:4007C000274826490988445423480088401C2249088008460088802801DB00200880214800680B2859D820481E490968405CA04207D01C48006804284CD91A4800680928CC
:4008000048D21A4817490968445416480068401C14492DE0290100203C01002026010020981400202A010020270100202801002020010020EA1400203001002034010020AC
:40084000380100203A010020E03900102B3C09087C220010D81300201A0100201C010020AA140020400100209CC10908531500200860084600680B280FD34021FB4881F075
:4008800066FBFB480068421EFA49F84881F0E0FA012602E00020F6490860FFF725FE1B2801D1012E12D10A2C0AD11720FFF71FFE4021EE4881F04BFB0020EF49088094E0F1
:4008C000ED480088401CEC4908808EE0FFF7DAFC01281BD1E54800787E2803D00020E649088004E0E4480088401CE34908807D2C7BD10120E1490870DF480278DB4928464B
:40090000FFF710FF0020DC4908806EE0D7480078772803D00020D849088066E0D8480068C8B9D5480088032815D1D048007877280ED1CE48407888280AD1CC48807899288C
:4009400006D1CA48CC490988405CCD49086002E00020C9490880CA480068401EC649098888423DD1C14840790006C049897940EA0140BE49C97940EA0120BC49097A40EA5E
:4009800001074FF00008B948C0780C3800F0FF09BB480068401EB54911F800A001F10908B7480078401EC1B2B048FFF710FC504509D14B46424639462846FFF739FE0120FB
:4009C000AE49087002E0A94890F813A04021A74881F0BDFA0020A8490880A949086004E0A5480088401CA4490880A6480088A649098888427FF4D9AEBDE8F087002008E007
:400A0000A249095C01B906E00021A04A1154411CC8B28028F4DB00209A4908809A4908807047002004E00021994A1154411CC8B24028F8DB0020974908709749087097492C
:400A40000870704701469448007870472DE9FC5F05460F4614464FF001080020019005B901AD1FB10021781E295401E000202870FFF73AFD1D287CD2DFE800F00F1D2A4477
:400A800054F6F57C8CB4F4F3CCF2F1F0EFEEEDECEBEAE9E8E7E6E5E4E3000021892002F090FB7F480FF0F6FA10B10120FFF71FFD4FF00008A7E30121892002F082FB794823
:400AC00000688047784908600220FFF710FD9AE341F288317448006859F0CAFB28B1FDF7BBFD7248FEF790FC0BE071A1284683F0A8F930B10320FFF7FAFCFFF77FFF4FF0FC
:400B0000000880E36C4881F02FF9C6B231466A48FDF717FE18B90420FFF7E9FC01E04FF0000870E3402C07D10020FFF7E0FCFFF765FF4FF000081BE060A1284683F081F9DA
:400B40000646A6B105F17F00864210D2B07D0A280DD1B146112109F10400FFF7DDFC0720FFF7C5FCFFF74AFF4FF0000800BF00BF49E342E3524881F0F7F8C6B231465048CC
:400B8000FDF7DFFD18B90820FFF7B1FC01E04FF0000838E3402C07D10020FFF7A8FCFFF72DFF4FF000081CE046A1284683F049F90646AEB105F17F00864211D296F82B0095
:400BC0000A280DD1B1462C224946404881F040F90920FFF78CFCFFF711FF4FF0000800BF00BF10E33A4B3BA212213C4880F05AFE3A480A3881F0B8F8C6B2314637480A3804
:400C0000FDF79FFD18B90C20FFF771FC01E04FF00008F8E2402C07D10020FFF768FCFFF7EDFE4FF000080BE02DA1284683F009F930B10A20FFF75BFCFFF7E0FE4FF00008CD
:400C4000E1E2D9E2BEE2A3E297E26CE230E20CE2FBE162E13FE126E1F4E0DBE0AEE096E085E051E040E0DAE17CE10000AA14002040010020531500201C0100201E01002020
:400C800044010020180100201A010020D813002058140020240100202C0100202D010020E039001008200010480100207C22001052454144590D0A00900000204D4143005F
:400CC000B40000204346475000000000FB140020EA14002025730D0A00000000A00000204F4B0D0A00000000F84881F03DF8C6B23146F648FDF725FD18B90B20FFF7F7FB86
:400D000001E04FF000087EE2402C07D10020FFF7EEFBFFF773FE4FF0000827E0AFF25C01284683F08EF80646FEB105F17F0086421BD296F82B000A2817D1B1462C22494602
:400D4000E34881F085F82C22E249E14880F0C7FF18B10D20FFF7CBFB02E00F20FFF7C7FBFFF74CFE4FF0000800BF00BF4BE2DA4880F0FAFFC6B23146D748FDF7E2FC18B999
:400D80000E20FFF7B4FB01E04FF000083BE2402C07D10020FFF7ABFBFFF730FE4FF000080BE0CEA1284683F04CF830B10020FFF79EFBFFF723FE4FF0000824E2C9480278B2
:400DC000C9A1CB4880F058FDC9480078C9498872C7484078C872C3480088C0F30722C2A1C34880F049FDC2480078C2490873C04840784873084680F0B7FFC6B23146BD489D
:400E0000FDF79FFC18B91020FFF771FB01E04FF00008F8E1402C07D10020FFF768FBFFF7EDFD4FF000080CE0AFF24C11284683F008F830B11120FFF75AFBFFF7DFFD4FF0A2
:400E40000008E0E1ACA000680090FFF799FBC6B23246A5A1684680F00FFD9DF80000A74988729DF80100C872FFF78AFB060A32469DA1684680F000FD9DF800009F490873D8
:400E80009DF801004873084680F06EFFC6B231469A48FDF756FC18B91220FFF728FB01E04FF00008AFE1402C07D10020FFF71FFBFFF7A4FD4FF000080CE0AFF2DC11284691
:400EC00082F0BFFF30B11320FFF711FBFFF796FD4FF0000897E188A000680090FFF765FB0646324680A1684680F0C6FC9DF80000834988729DF80100C872084680F034FF0D
:400F0000C6B231467E48FDF71CFC18B91420FFF7EEFA01E04FF0000875E1402C05D10020FFF7E5FA4FF000081BE0AFF24C21284682F087FF30B10520FFF7D9FAFFF75EFD82
:400F40004FF000086FA1284682F07BFF48B10020FFF72EFB0520FFF7CAFAFFF74FFD4FF0000850E10026B146B246FFF709FB1E280DDDFFF71AFB012807D11E20FFF703FB72
:400F8000FFF7FEFA00F01F0605E01F2603E0FFF7F7FA00F01F06FFF708FB00F0010046EA4016FFF711FB00F0030046EA801652A00068009032464CA1684680F05DFC9DF89F
:400FC0000000524988729DF80100C8724A4646A1684680F051FC9DF800004C4908739DF801004873524640A1684680F045FC9DF80000464988739DF80100C873084680F02E
:40100000B3FE00F0FF0B59464048FDF79AFB18B90620FFF76CFA01E04FF00008F3E0402C05D10020FFF763FA4FF000080CE0AFF25031284682F005FF30B11720FFF757FABA
:40104000FFF7DCFC4FF00008DDE0314880F08CFEC6B231462E48FDF774FB18B91620FFF746FA01E04FF00008CDE0402C05D10020FFF73DFA4FF0000819E0AFF29C312846A6
:4010800082F0DFFE38B11720FFF731FAFFF7B6FC4FF000080BE01FA1284682F0D2FE30B11720FFF724FAFFF7A9FC4FF00008AAE01A4880F059FEC6B231461848FDF741FB16
:4010C00018B91820FFF713FA2CE029E0B400002027150020FB1400200D01002053415645440D0A004C010020253032780000000050010020BD00002030300000CE000020B0
:40110000DF000020455252340D0A0000EE00002001010020455252320D0A0000070100204FF000086FE0402C05D10020FFF7DFF94FF0000820E036A1284682F082FE28B1D5
:401140001720FFF7D4F94FF0000815E0AFF23C01284682F076FE28B11520FFF7C8F94FF0000809E02CA1284682F06BFE20B11920FFF7BDF9FFF742FC45E0402C07D028A1E1
:40118000284682F05EFE10B11A20FFF7B0F93AE0402C02D14FF0000813E023A1284682F050FE70B11B20FFF7A2F903212048FEF764FCFFF723FC1F48006880470646FFF719
:4011C00008FA20E0402C0CD11B480078012812D10020194908701648FEF716F94FF0000809E016A1284682F02CFE20B11048FEF70BF94FF0000806E000BF0020FFF777F9DC
:401200004FF0000800BF00BF4046BDE8FC9F0000455252310D0A00004144560D0A00000052494E4720000000444154410D0A00007C22001008200010250100204449534330
:4012400000000000B64800787047B6480078704710B50446B44804700178BF2003F059F810BD10B513E0012083F00AF9601CC4B2332C0CDD0020FFF7EBFF1E2083F000F9F9
:401280000120FFF7E5FF1E2083F0FAF80024A748007802F0DAFF0028E5D110BD01460020042901DAA24A505C7047A2480078704710B50446042C11DA994804700178BE20E2
:4012C00003F027F8FFF7F1FF012803D1332083F0D7F803E04FF4857083F0D2F810BD30B52DED028B81B000200090B7EE000AB0EE408AFFF7A7FF0546012411E0681CC11762
:4013000000EB91718910A0EB8101CDB22846FFF7C5FF18B12846FFF7CBFF03E0601CC4B2042CEBDB00BFFFF78DFF0346FFF7B6FFC0B3FFF796FF0321684604F0C5F9009862
:4013400000F400000121B1EBD05F07D17A48009988430090BFEE000AB0EE408AFFF775FF00EE100AF8EE400A9DED000AB8EE400A20EE080A9FED711A20EE010A80EE201AC1
:40138000BDEEC10A10EE101AFFF75CFF6C4A42F820106C48006880470146FFF753FF6A4A42F8201001B0BDEC028B30BD00B50D21FFF77BFF18B1012803D10D2101E064210D
:4013C00000BF00BF084600BD00B50246FFF73DFF012806D0022806D0402806D0802808D105E0002105E0022103E0042101E0062100BF00BF084600BD70B504464D48047058
:40140000FFF723FF0346FFF7DFFF4A49097840EA01052946BD2002F07CFF70BD70B5044640480470FFF711FF0346FFF7CDFF0146FFF73BFF41EA00052946BD2002F069FF84
:4014400070BD10B50446414804700178B52001F0B8FE10BD08B500200090FFF7F9FE0120FFF7EFFF642083F00BF80220FFF720FF8020FFF7D3FF0120FFF7BEFF0120FFF78E
:40148000E7FE642082F0FCFFFFF7EBFE0421684604F01AF9642082F0F3FF08BD0EB503212B4880F86D10FFF7D5FF00BFFFF77EFF04462146002083F011F98DE80700009843
:4014C00008280FD1019800F4804058B10021204880F86D1000201E49886683F02FF9044683F044F9FFF7FBFEE0E701460020042902DA134A52F821007047014600200429C5
:4015000002DA114A52F821007047042801DA084A115470470D4800787047034800787047840000108500001088000010910000108000001086000010FFFF7F00FA02954306
:401540006015002054A80F087015002087000010300A002010B5002807DA0A07140EFE4A00F00F031B1FD45403E00A07130EFB4A135410BD70B504460D460026082C0BDAF1
:401580000120A040C6B23146B32002F0C2FE0021B42002F0BEFE27E0082C09D110260021B32002F0B6FE3146B42002F0B2FE1BE0092C09D120260021B32002F0AAFE3146EC
:4015C000B42002F0A6FE0FE00F2C05DAA4F10A0084B20120A040C6B20021B32002F099FE3146B42002F095FE2946B12002F091FE70BD10B5044601EE102AF8EE411A01EE87
:40160000103AB8EE411A81EE812AB0EE420AB7EE001AB4EEC10AF1EE10FA04DDB7EE001AB0EE410A08E0B5EEC00AF1EE10FA03D29FEDCB1AB0EE410AB7EE001A71EE401AD8
:4016400001EE101AB8EE411A61EE811A01EE104AB8EE411AF0EE610A41EE000ABCEEE01A11EE100A10BD10B5044604F00F040121692001F0A6FD04F00101412001F0A1FDD5
:40168000C4F34001392001F09CFDC4F38001602001F097FDE108692001F093FD10BD7FB506460C4615460720029000200390019400956946304676F0EEFB7FBDF8B50446E8
:4016C0000D46164600BF00200090A648006840F48000A44908600846006800F48000009000BF2560002060600021A160012121610021A16121626162E162A162E160E66192
:40170000216301216161984885421ED19748A063846397489549086000204860002193488160C1602915016189004161890081610021C1614FF400310162002141620121C1
:4017400081620021C162016346E08A48854220D18948A063846386483030874908604FF000704860002184488160C1602915016189004161890081610021C1614FF40031DA
:40178000016200214162012181620021C162016322E07A4885421FD17948A063846374481830774908604FF080604860002174488160C16029150161890041618900816127
:4017C0000021C1614FF40031016200214162012181620021C1620163204675F038FFA06B78F0E8F8A06B00686149884207D100213820FFF7AFFE382000F084FD1AE0A06B60
:4018000000685B493031884207D100213A20FFF7A1FE3A2000F076FD0CE0A06B006854491831884206D100213920FFF793FE392000F068FDF8BD8CB04FF0020800260025B2
:401840000321504880F86510062247494E48FFF735FF052247494D48FFF730FF082247494B48FFF72BFF00210846FFF783FE46480068406840F020004349096848600822C6
:4018800001214148FFF70BFF032202213E48FFF706FF0F2203213C48FFF701FF092204213948FFF7FCFE112205213748FFF7F7FE122206213448FFF7F2FE0A2201213348DB
:4018C000FFF7EDFE0B2202213048FFF7E8FE0C2203212E48FFF7E3FE0D2204212B48FFF7DEFE0E2205212948FFF7D9FE002201212748FFF7D4FE012202212548FFF7CFFEA6
:40190000022203212248FFF7CAFE062204212048FFF7C5FE072205211D48FFF7C0FE092206211B48FFF7BBFE0E2207211848FFF7B6FE0F2208211648FFF7B1FE1548006879
:4019400020F480000849C1F8040300BF0021084682F0C4FE09AB1FE018ED00E000E400E00000000030380240002001401C19002010640240002101407C1900200022014074
:40198000DC190020300A00203C1A0020841A0020CC1A00200423014007C3099808280FD10A9800F4804058B10021FD4880F865100020FB49086682F0C1FE044682F0D6FE56
:4019C0000027F4E33846FFF74EFEF6480068806840F00100F34909688860062082F050FD062201A9EF4876F075F9814641F28831012082F073FE09AB07C3099808287DD1BF
:401A0000B9F1000FFBD1E848006880470446E748C0F8F840C0F8FC40E5490598C1F8F8000698C1F8FC00E3490598C1F8F8000698C1F8FC00102F1ED2DFE807F0081E344A38
:401A400061778DA3B9F1F0EFEEEDECEBD74804600464C0F88040D64901980860029808640398C1F88000D34901980860029808640398C1F88000ACE2CC4844604464C0F829
:401A80008440CB4901984860029848640398C1F88400C84901984860029848640398C1F8840096E2C14884608464C0F88840C04901988860029888640398C1F88800BD49C0
:401AC00001988860029888640398C1F8880080E2B648C460C464C0F88C40B5490198C8600298C8640398C1F88C00B2490198C8600298C8640398C1F88C006AE26BE2AB4880
:401B000004610465C0F89040A94901980861029808650398C1F89000A64901980861029808650398C1F8900053E2A04844614465C0F894409E490198486102984865039892
:401B4000C1F894009B4901984861029848650398C1F894003DE2954884618465C0F89840934901988861029888650398C1F89800904901988861029888650398C1F89800CA
:401B800027E28A48C461C465C0F89C4088490198C8610298C8650398C1F89C0085490198C8610298C8650398C1F89C0011E27F4804620466C0F8A04044200BF09DFC30B1DC
:401BC00050200BF099FC40B10020019005E050200BF092FC08B9002001903A200BF08CFC30B145200BF088FC40B10020029005E045200BF081FC08B90020029039200BF025
:401C00007BFC68B138200BF077FC78B1002003900CE013E1FCE0E5E0CEE0AAE060E016E038200BF069FC08B900200390604901980862029808660398C1F8A0005D49019870
:401C40000862029808660398C1F8A000C1E1574844624466C0F8A44036200BF04DFC30B137200BF049FC40B10020019005E037200BF042FC08B90020019032200BF03CFCB1
:401C800030B133200BF038FC40B10020029005E033200BF031FC08B9002002902E200BF02BFC30B12F200BF027FC40B10020039005E02F200BF020FC08B9002003903C49A5
:401CC00001984862029848660398C1F8A400394901984862029848660398C1F8A40078E1324884628466C0F8A84035200BF004FC30B134200BF000FC40B10020019005E016
:401D000034200BF0F9FB08B90020019031200BF0F3FB30B130200BF0EFFB40B10020029005E030200BF0E8FB08B90020029017200BF0E2FB30B118200BF0DEFB40B1002068
:401D4000039005E018200BF0D7FB08B900200390174901988862029888660398C1F8A800144901988862029888660398C1F8A8002FE10E48C462C466C0F8AC400C4901985F
:401D8000C8620298C8660398C1F8AC0009490198C8620298C8660398C1F8AC0019E10000300A00203C1A002054A80F08E817002080150020B4160020FD4804630467C0F8EA
:401DC000B040FC4901980863029808670398C1F8B000F94901980863029808670398C1F8B000F6E0F24844634467C0F8B440F14901984863029848670398C1F8B400EE4936
:401E000001984863029848670398C1F8B400E0E0E74884638467C0F8B840E64901988863029888670398C1F8B800E34901988863029888670398C1F8B800CAE0DC48C4631A
:401E4000C467C0F8BC40DB490198C8630298C8670398C1F8BC00D8490198C8630298C8670398C1F8BC00B8F10E0F13D2DFE808F007131F2B37434F5B67737F8B97A3CC48E0
:401E8000C0F8C040CB490498C1F8C000CA490498C1F8C0009BE0C648C0F8C440C5490498C1F8C400C4490498C1F8C4008FE0C048C0F8C840BF490498C1F8C800BE49049888
:401EC000C1F8C80083E0BA48C0F8CC40B9490498C1F8CC00B8490498C1F8CC0077E0B448C0F8D040B3490498C1F8D000B2490498C1F8D0006BE0AE48C0F8D440AD490498F8
:401F0000C1F8D400AC490498C1F8D4005FE0A848C0F8D840A7490498C1F8D800A6490498C1F8D80053E0A248C0F8DC40A1490498C1F8DC00A0490498C1F8DC0047E09C488D
:401F4000C0F8E0409B490498C1F8E0009A490498C1F8E0003BE09648C0F8E44095490498C1F8E40094490498C1F8E4002FE09048C0F8E8408F490498C1F8E8008E49049807
:401F8000C1F8E80023E08A48C0F8EC4089490498C1F8EC0088490498C1F8EC0017E08448C0F8F04083490498C1F8F00082490498C1F8F0000BE07E48C0F8F4407D490498D7
:401FC000C1F8F4007C490498C1F8F40000BF00BF00BF00BF00BF794875F023FF774875F002FC77480068806840F00100744909688860052201A9724875F06CFE814641F257
:402000008831012082F06AFB09AB07C30998082867D1B9F1000F64D130461DF0F7F9044668480068804706466148C0F80061C0F80461C0F80861C0F80C61C0F810615D499E
:402040000198C1F800010298C1F804010398C1F808010498C1F80C010598C1F81001564AD2F80011534A0C23D2F800012246FFF7C0FA5149C1F800010A46D2F804114D4A4B
:402080000C23D2F804012246FFF7B3FA4A49C1F804010A46D2F80811464A0C23D2F808012246FFF7A6FA4449C1F808010A46D2F80C11404A0C23D2F80C012246FFF799FAFC
:4020C0003D49C1F80C010A46D2F81011394A0C23D2F810012246FFF78CFA3749C1F8100100BF374875F09DFE354875F07CFB36480068806840F00100334909688860082209
:4021000001A9314875F0E6FD814641F28831012082F0E4FA09AB07C3099808287ED1B9F1000F7BD128461DF071F9044625480068804705461E48C0F81451C0F81851C0F8FB
:402140001C51C0F82051C0F82451C0F82851C0F82C51C0F8305117490198C1F814010298C1F818010398C1F81C010498C1F820010598C1F824010698C1F828010798C1F890
:402180002C010898C1F830010B4AD2F81411094A0C23D2F814012246FFF72BFA0649C1F814010A46D2F81811024A0C230EE06DE0E817002080150020B41600203C1A0020F6
:4021C000841A002054A80F08CC1A0020D2F818012246FFF70EFA5149C1F818010A46D2F81C114F4A0C23D2F81C012246FFF701FA4A49C1F81C010A46D2F82011484A0C238F
:40220000D2F820012246FFF7F4F94449C1F820010A46D2F82411424A0C2300E02FE0D2F824012246FFF7E5F93C49C1F824010A46D2F828113A4A0C23D2F828012246FFF723
:40224000D8F93649C1F828010A46D2F82C11344A0C23D2F82C012246FFF7CBF92F49C1F82C010A46D2F830112D4A0C23D2F830012246FFF7BEF92949C1F8300100BF294814
:4022800075F0CFFD274875F0AEFA7F1C102FFFF499AB08F101001FFA80F8B8F10D0F01DD4FF0020800214046FFF764F9FFF74EBB10B504461C4890F86500032804D11A492D
:4022C000086E012182F0FEF910BD10B51749886B77F0C7FD10BD10B51549886B77F0C1FD10BD10B50F49886B77F0BBFD10BD10B50E4875F0E9FB0E4875F0E6FB094875F046
:40230000E3FB10BD00F01F02012191404209920002F1E022C2F8001170470000B416002080150020CC1A0020300A00203C1A0020841A00207CB500260020FB4981F8CC0067
:40234000FA4981F8CC00F848D0F8C80028B9F84882F064F9F449C1F8C800F448D0F8C80028B9F44882F05AF9F049C1F8C8000020092103460246CDE900100221EE4800787D
:4023800000F078FF0020092103460246CDE900100221EA48007800F06DFF0020092103460246CDE900100221E548007800F062FF0020092103460246CDE900100221E14845
:4023C000007800F057FFE048D74908600C2048600021D54881604FF08071C1604FF4202101614FF4001141610021017601214176002181760121C1760021017701214177FA
:402400000020C94988620021C748C1620163416381630121C163002101640121416481640021C164C948C14908600C2048600021BE4881604FF08071C1604FF420210161ED
:402440004FF4001141610021017601214176002181760121C17600210177012141770020B24988620021B148C16201634163012181630E21C163002101640121416481643C
:402480000E21C164132077F057F8152077F054F8142077F051F83F2077F04EF8412077F04BF8402077F048F89F4876F052FA0446ACB99D4928319C4876F054FB044674B95E
:4024C000994876F0DFFB04464CB90321964876F043FE04461CB90120934981F8CC00934876F037FA0546ADB9904928318F4876F039FB054675B98D4876F0C4FB05464DB9D8
:4025000011218A4876F028FE05461DB90120874981F8CC0004B1264605B12E4630467CBD70B588B0054600260020009000BF287D18B1022803D17C4C03E07C4C01E0002499
:4025400000BF00BF002C6ED094F8CC0001286AD10121D4F8C80082F091F800287BD100BF687D50B1012809D1284614F0D2FF0390002002900420049008E000BF284614F091
:40258000C8FF029000200390049000BF00BF002005902868816928468847069000208DF81C006248844203D13F2076F0D2FF05E05D48844202D1132076F0CBFF286801A9A0
:4025C000C26828469047012834D16B4602A92046019A76F0DBFB30B1012825D0022824D0032824D122E00098012804D0022809D0042815D10DE02822294604F150007FF062
:402600006CFC0DE02822294604F178007FF065FC06E02822294604F1A0007FF05EFC00BF00BF012605E016E000BF00BF00BF002600BF00BF3D48844203D13F2076F07CFF92
:4026400005E03948844202D1132076F075FFD4F8C80082F007F8304608B070BD2DE9F84305460C4691464FF002083048854202D14FF0000804E02C48854201D14FF002084D
:40268000B8F1020F13DAA06820B1042803D16668012703E000BF2668002700BF00BFCDF80080237C4A463146384658F099F9BDE8F88310B51C4876F088FD10BD10B51A4864
:4026C00076F083FD10BD10B5174876F07EFD10BD10B5164876F079FD10BD10B5134876F074FD10BD10B5114876F06FFD10BD10B504460E48844204D1012150301BF0B7FEA6
:4027000006E00948844203D1012150301BF0AFFE10BD10B504460548844219D1012178301BF0A5FE1BE00000341B0020041C0020A8C10908ACC10908950000109600001030
:40274000970000109800001000640040006800404348844203D1012178301BF088FE10BD10B504463F48844204D10121A0301BF07EFE06E03A48844203D10121A0301BF0C8
:4027800076FE10BD10B504463648844204D1002150301BF06CFE06E03148844203D1002150301BF064FE10BD10B504462D48844204D1002178301BF05AFE06E0284884425F
:4027C00003D1002178301BF052FE10BD10B504462448844204D10021A0301BF048FE06E01F48844203D10021A0301BF040FE10BD10B58AB0044604E001AA03A92046FFF7EE
:402800002DFF01AB03AA0021204676F0CCFB0028F2D00AB010BD10B58AB0044604E001AA03A92046FFF71AFF01AB03AA0121204676F0B9FB0028F2D00AB010BD10B5084874
:4028400081F0DEF80446084A08497FF00DFA054881F0D6F80446044A04497FF005FA10BD341B0020041C002000800008333A09082DE9F04106460C4615460027002E61D087
:40288000B4F1D04F0ED36019401E8149884209D8A4F1D0412A46304602F083FE002851D101274FE07B4884420ED36019401E7A49884209D87748211A2A46304602F0A9FB62
:4028C00000283FD101273DE0744884420ED36019401E72493F31884208D87048211A2A46304602F08BFC68BB01272BE0B4F1805F0BD36019401E6A49884206D82A46214639
:4029000030467FF0A5FA01271CE0B4F1005F0BD36019401E6349884206D82A46214630467FF096FA01270DE0B4F1006F0AD36019401EB0F1026F05D22A46214630467FF014
:4029400087FA01273846BDE8F0812DE9F04106460C4615460027002E51D0B4F1D04F0ED36019401E4A49884209D8A4F1D0412A46304602F08DFD002841D101273FE0454894
:4029800084420DD36019401E4349884208D84148211A2A46304602F00EFB08BB01272EE03E4884420ED36019401E3C493F31884208D83A48211A2A46304602F0CDFB78B995
:4029C00001271CE0B4F1805F0BD36019401E3449884206D82A46314620467FF039FA01270DE0B4F1005F0AD36019401E2D49884205D82A46314620467FF02AFA01273846F6
:402A0000BDE8F08170B504460D460026002D3CD0B4F1D04F0CD36019401E1D49884207D8A4F1D040294602F018FE00BB01262CE0184884420ED36019401E1749884209D8E3
:402A4000144AA21A5119134AA01A02F0BBF970B901261AE0B4F1805F0AD36019401E1049884205D8294620467FF071FA01260CE0B4F1005F09D36019401E0A49884204D821
:402A8000294620467FF063FA0126304670BD0000FF7F006800010168FF00016900000168FFFF0010FFFF0220FE4800787047FE4800787047FC4908707047FC48007870478A
:402AC000FA4908707047FA4800787047F8490870704710B5022200218D2001F05BFC022200218E2001F056FC022200218F2001F051FC02220021902001F04CFC02220021A9
:402B0000912001F047FC02220021922001F042FC02220021932001F03DFC02220021942001F038FC02220021952001F033FC02220021962001F02EFC02220021972001F02D
:402B400029FC02220021982001F024FC02220021992001F01FFC022200219A2001F01AFC022200219B2001F015FC022200219C2001F010FC022200219D2001F00BFC0222F4
:402B800000219E2001F006FC022200219F2001F001FC02220021A02001F0FCFB02220021A12001F0F7FB02220021A22001F0F2FB02220021A32001F0EDFB02220021A420AC
:402BC00001F0E8FB02220021A52001F0E3FB02220021A62001F0DEFB02220021A72001F0D9FB02220021A82001F0D4FB02220021A92001F0CFFB02220021AA2001F0CAFB27
:402C000000221146AC2001F0C5FB00221146AD2001F0C0FB00221146AE2001F0BBFB00221146AF2001F0B6FB00221146B02001F0B1FB00220121D72001F0ACFB00220121D7
:402C4000D82001F0A7FB00220121D92001F0A2FB00221146DA2001F09DFB00221146B12001F098FB00221146B22001F093FB01220021B32001F08EFB00221146B42001F09B
:402C800089FB00221146CC2001F084FB00221146D12001F07FFB00221146CD2001F07AFB00221146CE2001F075FB00221146CF2001F070FB00221146D02001F06BFB0022AC
:402CC0001146D22001F066FB00221146D32001F061FB00221146D42001F05CFB00221146D52001F057FBFFF7E2FE044622460021B52001F04FFBFFF7E0FE044622460021BA
:402D0000B62001F047FBFFF7DEFE044622460021B72001F03FFB00220121D62001F03AFB00221146B82001F035FB00221146B92001F030FB00221146BA2001F02BFB002217
:402D40001146BB2001F026FB00221146BC2001F021FB00221146BD2001F01CFB00221146BE2001F017FB00221146BF2001F012FB00221146C02001F00DFB00221146C120F3
:402D800001F008FB00221146C22001F003FB00221146C32001F0FEFA00221146C42001F0F9FA00221146C52001F0F4FA00221146C62001F0EFFA00221146C72001F0EAFAA4
:402DC00000221146DC2001F0E5FA00221146DB2001F0E0FA00221146DE2001F0DBFA00221146DD2001F0D6FA00221146E02001F0D1FA00221146DF2001F0CCFA00221146FE
:402E0000E22001F0C7FA00221146E12001F0C2FA00221146E42001F0BDFA00221146E32001F0B8FA00221146E62001F0B3FA00221146E52001F0AEFA00221146E82001F0CD
:402E4000A9FA00221146E72001F0A4FA00221146EA2001F09FFA00221146E92001F09AFA00221146EC2001F095FA00221146EB2001F090FA00221146ED2001F08BFA00226A
:402E80001146EE2001F086FA00221146EF2001F081FA00221146F02001F07CFA00221146F12007E05301002054010020550100205601002001F06EFA00221146F22001F03C
:402EC00069FA00221146F32001F064FA00221146F42001F05FFA00221146F52001F05AFA00221146F62001F055FA00221146F72001F050FA00221146F82001F04BFA002267
:402F00001146F92001F046FA00221146FA2001F041FA10BD2DE9F04F89B04FF0200B4FF00A0A03214E4880F85D1001214D48007800F047F9012081F0A3FA002149480078C2
:402F400000F03FF9012081F09BFA01214548007800F037F90A2081F093FA0A2242A145487EF02BFF28B10A2243A142487EF025FF28B9444F444D00204449087004E0444FB9
:402F8000444D01204149087020244FF0000915E009EB0400A84202D9A5EB0900C4B22246394601A857F094F800B909E02744214601A802F0A6F800B102E0A144A945E7D3E0
:402FC0003548007801F041F980463448007801F03CF90646B8F1000F16D0012E14D14FF00B0A81F04DFA01212D48007800F0E9F8012081F045FA00212948007800F0E1F843
:40300000322081F03DFA10E0B8F1010F03D116B94FF00D0A09E0B8F1000F04D1012E02D14FF00C0A01E04FF00E0ABAF10B0F09D1FFF74FFD3521C02001F06BF93521C42049
:4030400001F067F9064880F85DA000200449886581F074FB814681F089FB09B0BDE8F08F300A0020A2000010303634303137313333320000A86F00083036343031373134AC
:403080003636000000010D6803F20400530100200001016818E40800A1000010A3000010A0000010F0B5FE4A0024204621460FE00A2600230446A4FB067C01FB06C500FBF2
:4030C0000351384612F8013B303B181841EBE3711378302B02DB1378392BE9DDF0BDF14800787047EF49087070470020EC4950310978412909DBEA49503109785A2904DC6C
:40310000E749503109784139C8B27047F0B5E44A60320024204621460FE00A2600230446A4FB067C01FB06C500FB0351384612F8013B303B181841EBE3711378302B02DBF7
:403140001378392BE9DDF0BD0020D54920310978412909DBD249203109785A2904DCD049203109784139C8B27047F0B5CC4A30320024204621460FE00A2600230446A4FB70
:40318000067C01FB06C500FB0351384612F8013B303B181841EBE3711378302B02DB1378392BE9DDF0BD01464FF6FF70012905DB8C2903DCBC4A02EBC10290887047012034
:4031C0007047F8B504460E460127FB2C50DAB748005D082808D2DFE800F0040508090B0A240600BF00BF00BF41E000BF00BF00BF012E0AD1AC4A02EBC4029188AA4A52F839
:403200003400012277F063F909E0A74A02EBC4029188A54A52F83400002277F058F9002725E0A4F18D0085B205EB4500A0490844407806FA00F0C0B2009005EB450008446D
:40324000807850B105EB450008448178012088409DF800100843C0B2009005EB4500944A115C0122684601F077FF074600BF00BF3846F8BD2DE9F04786B004460D461646CE
:403280001F46DDE90E894FF0010A012C78DB8C2C7EDC854850F83400002879D04FF0000A814800EBC40080880190029503960497CDF814807F49681A8D422DD00DDC032D09
:4032C00054D005DCDDB1012D32D0022D59D13EE0112D2ED0122D54D13AE0B0F5881F19D006DCB0F5803F14D0B0F5801F49D114E0B0F5001F12D0B0F5041F42D10BE002209B
:403300006A490855684951F8340001A976F03CFF3DE000BF00BF00BF00BF00BF032063490855614951F8340001A976F02DFF2EE000BF05205D4908555B4951F8340001A9DD
:4033400076F022FF49462046FFF73BFF1FE000BF042056490855544951F8340001A976F013FF49462046FFF72CFF10E001204F4908554D4951F8340001A976F005FF06E05E
:4033800006E00020494908554FF0010A00BF00BF504606B0BDE8F087002003E00021434A1154401CFB28F9D370471FB50520424908706420414908704220414908700620C4
:4033C0004049087007204049087008203F49087031203F49087082203E4908701F203E49087084203D4908701B203D4908701C203C49087019203C4908701A203B490870CC
:4034000016203B4908701E203A4908702B203A4908702C20394908703C20394908703D20384908705120384908706D20374908705B20374908705F2036490870652036490D
:403440000870632035490870442035490870FFF7A3FFFFF7B4FE002866D07AF051FE04467AF0CAFFB4FBF0F0012809D97AF0C4FF40002C49B0FBF1F0401E80B2039007E01B
:403480007AF0BAFF2749B0FBF1F0401E80B203907AF036FE04467AF0BBFFB4FBF0F044E0786F0008A4000010FCC2090882250010B0C1090800001110890000108A0000100C
:4034C0008B0000108C0000108D0000108E0000108F000010900000109100001092000010930000109400001095000010960000109700001098000010990000109A000010A4
:403500009B0000109C0000109D0000109E0000109F000010A0000010A1000010A2000010A300001040420F00FDE3012809D97AF06FFF4000FE49B0FBF1F0401E80B20290DB
:4035400007E07AF065FFFA49B0FBF1F0401E80B2029000BF00200190F648006840F00100F44908600846006800F00100019000BF00BF002001900846006840F00200086002
:403580000846006800F00200019000BF00BF002001900846006840F0040008600846006800F00400019000BF00BF002001900846006840F0080008600846006800F00800E3
:4035C000019000BF00BF002001900846006840F0100008600846006800F01000019000BF00BF002001900846006840F0200008600846006800F02000019000BF00BF0020D4
:4036000001900846006840F0400008600846006800F04000019000BF00BF002001900846006840F0800008600846006800F08000019000BF00BF002001900846006840F427
:403640008071BC480160006800F48070019000BF00BF00200190B748006840F40010B54908600846006800F40010019000BF00BF002001900846006840F48000086008463D
:40368000006800F48000019000BF00BF00200190A8481430006840F00100A649143108600846006800F00100019000BF00BF00200190081F006840F00200091F08600846FF
:4036C000006800F00200019000BF00BF002001900846006840F0040008600846006800F00400019000BF00BF002001900846006840F0080008600846006800F0080001905F
:4037000000BF00BF002001900846006840F0100008600846006800F01000019000BF00BF00200190081D006840F00200091D08600846006800F00200019000BF00BF002062
:4037400001900846006840F4803008600846006800F48030019000BF00BF002001900846006840F4003008600846006800F40030019000BF00BF002001900846006840F496
:40378000802008600846006800F48020019000BF00BF00200190081F006840F04000091F08600846006800F04000019000BF00BF002001900846006840F480200860084682
:4037C000006800F48020019000BF00BF002001900846006840F4804008600846006800F48040019000BF00BF002001900846006840F4800008600846006800F48000019044
:4038000000BF00BF002001900846006840F0007008600846006800F00070019000BF00BF002001900846006840F0806008600846006800F08060019000BF00BF0020019051
:40384000081D006840F48070091D08600846006800F48070019000BF00BF002001900846006840F4007008600846006800F40070019000BF00BF002001900846006840F429
:40388000806008600846006800F48060019000BF00BF002001900846006840F0100008600846006800F01000019000BF00BF002001900846006840F48050086008460068CA
:4038C00000F48050019000BF1B49029888621B49039808601A49039808601A4903980860194902980860194902988862184902980860184902980860174903980860002006
:40390000009003460246014601900120FFF7B2FC0020009003460246014601900220FFF7A9FC00200090034602460146019015E040420F00303802400000014028040040FD
:4039400028080040280C004028040140004001402844014028480140281800400320FFF789FC0020009003460246032101900420FFF780FC00200090034602460121019079
:403980000520FFF777FC0020052103460246CDE9001002210620FFF76DFC0020052103460246CDE9001002210720FFF763FC0020052103460246CDE9001002210820FFF71A
:4039C00059FC0020009003460246012101900920FFF750FC0020009003460246012101900A20FFF747FC0020009003460246012101900B20FFF73EFC00200090034602462C
:403A0000012101900C20FFF735FC0020009003460246012101900D20FFF72CFC0020009003460246032101901120FFF723FC0020009003460246032101901220FFF71AFCD1
:403A40000020009003460246012101901620FFF711FC0020009003460246012101901720FFF708FC0020009003460246012101901820FFF7FFFB002100910B460A460191F3
:403A800001211920FFF7F6FB0121002003460246CDE900011A20FFF7EDFB0020042102230246CDE9001012211B20FFF7E3FB0021042002230A46CDE9000112211C20FFF792
:403AC000D9FB002100910B460A46019101211D20FFF7D0FB0121002003460246CDE900011E20FFF7C7FB002105200B460A46CDE9000102211F20FFF7BDFB002100910B46BC
:403B00000A46019101212020FFF7B4FB002100910B460A4621200191FFF7ACFB002100910B460A4622200191FFF7A4FB0020009003460246014601902320FFF79BFB002114
:403B400000910B460A4624200191FFF793FB0020009003460246014601902520FFF78AFB002100910B460A46019103212620FFF781FB002100910B460A46019101212720D1
:403B8000FFF778FB0020009003460246012101902820FFF76FFB002100910B460A46019101212920FFF766FB002100910B460A46019101212A20FFF75DFB00200721034629
:403BC0000246CDE9001002212B20FFF753FB002107200B460A46CDE9000102212C20FFF749FB0020009003460246014601902D20FFF740FB002100910B460A462E200191F2
:403C0000FFF738FB002100910B460A462F200191FFF730FB002100910B460A4630200191FFF728FB0121002003460246CDE900013120FFF71FFB002100910B460222322054
:403C40000191FFF717FB0020009003460222014601903320FFF70EFB002100910B46022234200191FFF706FB0020009003460222014601903520FFF7FDFA002100910B4625
:403C8000022236200191FFF7F5FA002100910B46022237200191FFF7EDFA0020009003460222014601903820FFF7E4FA002100910B460A46019101213920FFF7DBFA0021B9
:403CC00000910B460A463A200191FFF7D3FA0020009003460246012101903B20FFF7CAFA002107200B460A46CDE9000102213C20FFF7C0FA00200090034602460221019016
:403D00003D20FFF7B7FA002100910B460A463E200191FFF7AFFA002100910B460A46019101213F2000E08FE2FFF7A4FA002100910B460A46019101214020FFF79BFA00213F
:403D400000910B460A46019101214120FFF792FA0121002003460246CDE9000111214220FFF788FA0020009003460246014601904320FFF77FFA002100910B460A46442042
:403D80000191FFF777FA012000210B460A46CDE9001001464520FFF76DFA002100910B460A46019101214620FFF764FA002100910B460A46019111214720FFF75BFA0020AE
:403DC000009003460246014601904820FFF752FA002100910B460A4649200191FFF74AFA002100910B460A464A200191FFF742FA0020009003460246014601904B20FFF79D
:403E000039FA002100910B460A464C200191FFF731FA0020009003460246012101904D20FFF728FA002100910B4602224E200191FFF720FA002100910B460A460191012126
:403E40004F20FFF717FA002100910B460A4650200191FFF70FFA002100910B460A46019101215120FFF706FA002100910B46022252200191FFF7FEF90020009003460222D5
:403E8000014601905320FFF7F5F9002100910B460A4654200191FFF7EDF90020009003460246014601905520FFF7E4F9002100910B460A4656200191FFF7DCF90021009165
:403EC0000B460A46019101215720FFF7D3F90020009003460246012101905820FFF7CAF90020009003460246014601905920FFF7C1F9002100910B460A465A200191FFF778
:403F0000B9F9012000210B460A46CDE9001011215B20FFF7AFF9002100910B460A46019101215C20FFF7A6F9002100910B460A465D200191FFF79EF9002100910B460222AD
:403F40005E200191FFF796F9002100910B460A46019101215F20FFF78DF9002100910B460A46019101216020FFF784F9002100910B46022261200191FFF77CF90021009159
:403F80000B46022262200191FFF774F90020009003460246112101906320FFF76BF9002100910B460A46019111216420FFF762F90020009003460246014601906520FFF7B4
:403FC00059F9002100910B46022266200191FFF751F9002100910B460A4667200191FFF749F90020009003460246014601906820FFF740F900200090034602460121019088
:404000006920FFF737F9002100910B4602226A200191FFF72FF90020009003460246014601906B20FFF726F9002100910B460A466C200191FFF71EF90020009003460246F8
:40404000012101906D20FFF715F9002100910B460A466E200191FFF70DF9002100910B460A466F200191FFF705F9002100910B460A4670200191FFF7FDF8002100910B46C2
:40408000022273200191FFF7F5F8002100910B46022274200191FFF7EDF80020009003460222014601907520FFF7E4F8002100910B46022276200191FFF7DCF80020009087
:4040C00003460246012101907720FFF7D3F8002100910B460A46019102217820FFF7CAF8002100910B460A46019102217920FFF7C1F80020009003460246012101907A20EE
:40410000FFF7B8F80020009003460246012101907B20FFF7AFF8002100910B460A46019101217C20FFF7A6F80020009003460246012101907D20FFF79DF8002100910B4657
:4041400002227E200191FFF795F80020009003460222014601907F20FFF78CF80020009003460222014601908020FFF783F8002100910B460A46019101218120FFF77AF844
:40418000002105200B460A46CDE9000102218220FFF770F8002100910B460A46019101218320FFF767F8002105200B460A46CDE9000102218420FFF75DF800200090034696
:4041C0000222014601908520FFF754F8002100910B460A46019101218620FFF74BF80020009003460246012101908720FFF742F8002100910B460A46019101218820FFF786
:4042000039F8002100910B460A46019101218920FFF730F80020009003460222014601908A20FFF727F80020009003460222014601908B20FFF71EF8002100910B460222F8
:404240008C200191FFF716F81FBDF8B50446002600200090FB2C41DA5C48005D082807D2DFE800F0040507080A09191A00BF00BF33E000BF00BF00BF554A02EBC4029188B9
:40428000534A52F8340076F01AF9012800D100E00020064621E000BFA4F18D0085B205EB45004C4A115C0122684600F0A7FF98B905EB450047490844807868B105EB4500C4
:4042C00008444178012088409DF80010084008B1012000E00020064600BF00BF3046F8BD01460020012913DB8C2911DC384A52F831206AB1364A52F831205269344B03EB78
:40430000C1039B881A400AB1012200E0002210467047F8B505460E460127FB2D38DA2B48405D08280CD2DFE800F0040507080A090C0600BF00BF00BF00BF00BF00BF00BF56
:4043400025E0A5F18D0084B204EB440021490844407806FA00F0C0B2009004EB44000844807850B104EB440008448178012088409DF800100843C0B2009004EB4400154AEF
:40438000115C0122684600F0E7FE074600BF00BF3846F8BD2DE9F04104460D46164601278D2C0FDBFB2C0DDA012D03D107200749085502E006200549085531462046FFF777
:4043C000A8FF07463846BDE8F081000082250010FCC20908B0C1090810B5002807DA0A07140E4B4A00F00F031B1FD45403E00A07130E484A135410BD10B504464648006853
:4044000020B9464880F00AF943490860444876F03AF9002142488160FE21C160002181614161C16101624FF4804101613D483C494860084676F097F80B212120FFF7CCFF0A
:404440000B212220FFF7C8FF212000F056F8222000F053F810BD2DE9F84304460D4616461F46DDF820804FF001094FF47A712A48006880F003F968B93B4632462946204678
:40448000CDF8008076F084FA81462348006880F0E9F801E04FF003094846BDE8F8832DE9FE4F05460E4617461C46DDE90C8A4FF001094FF47A711848006880F0DFF868B94A
:4044C00001233A46314628468DE8100578F00FF981461148006880F0C5F801E04FF003094846BDE8FE8F10B50D4879F05CFA10BD10B50B4879F05EFB10BD00F01F02012118
:4045000091404209920002F1E022C2F80011704718ED00E000E400E0A800001064C7090880260010801A060010B5002807DA0A07140EF84A00F00F031B1FD45403E00A07C8
:40454000130EF54A135410BD01460620B1F5807F38D012DC102930D008DC012925D0022925D0042925D0082936D124E0202926D0402925D080292FD123E0B1F5805F26D021
:4045800009DCB1F5007F1ED0B1F5806F1DD0B1F5006F21D11AE0B1F5005F19D0B1F5804F17D0B1F5004F17D114E0062014E0072012E0082010E009200EE00A200CE000BF2E
:4045C00000BF00BF00BF172006E000BF00BF00BF00BF00BF282000BF00BF70470146FF20B1F5807F3BD012DC102930D008DC012925D0022925D0042925D008293FD124E062
:40460000202926D0402926D0802938D125E0B1F5805F2CD009DCB1F5007F22D0B1F5806F21D0B1F5006F2AD11FE0B1F5005F20D0B1F5804F1FD0B1F5004F20D11DE00020B7
:404640001DE001201BE0022019E0032017E0042015E0052013E0062011E007200FE008200DE009200BE00A2009E00B2007E00C2005E00D2003E00E2001E00F2000BF00BF63
:40468000704710B5062074F064FF0F210620FFF74BFF072074F05DFF0F210720FFF744FF082074F056FF0F210820FFF73DFF092074F04FFF0F210920FFF736FF0A2074F02C
:4046C00048FF0F210A20FFF72FFF172074F041FF0F211720FFF728FF282074F03AFF0F212820FFF721FF362074F033FF06213620FFF71AFF002005E00021884A42F8201049
:40470000411CC8B21028F7DB8548006880B1002084490870824800687FF09FFB002080490860814800687FF098FB00207E49086010BD2DE9FC47FFF7A4FF002463E001A9EF
:40474000204672F023FB00285BD001980068C16801988847002854D101980068816801988847092802D00A2849D100E000BF019872F0B0FB00F0FF08404607F0EBFE074691
:40478000FEF711FD0646FFF729FF0546102D35DA019872F09FFBC6B2304607F0DBFE6349495D884215D1019872F094FB00F0FF09484607F0CFFE8046FEF7F5FC0746FFF7DD
:4047C000C3FE064674F0B8FE5449019841F8250014E0DFF84C81534E019F307800904FF000090098FF2807D26A464146384681F095FB81460098307000BF00BF00E000BF3B
:4048000000BF601C84B272F0BEFAA04297DC4548007800281DDD434800787FF022FB4249086000240EE03E49096851F8240072F051FBC6B2304608F01BFE3B490968085579
:40484000601C84B2374800788442ECDB362074F073FEBDE8FC87014635480068084020B93348001D0068084008B1012070470020FCE77CB504462046FEF795FC064630465D
:40488000FFF7ACFE05463046FFF7E5FF48B10020009003460246014601902046FEF7EAFC0CE00020009003460246224901902046FEF7E0FC102D01DA1C4844557CBD10B5F7
:4048C000FFF7DFFE002404E0002018490855601CC4B2102CF8DB01201749C860592088623120C86205200860002014490860002112480838C1600161416100200C49091D8A
:404900000860091F08600A490C310860091F086010BD000018ED00E000E400E0E426001058010020600100205C01002024270010003C014000001110001000400838014026
:4049400070B505462846FFF749FE0446102C08DA3F4850F8240020B13D4951F8240072F01EF970BD10B5012075F0D3FD10BD10B5022075F0CEFD10BD10B5042075F0C9FD77
:4049800010BD10B5082075F0C4FD10BD10B5102075F0BFFD10BD10B5202075F0BAFD402075F0B7FD802075F0B4FD4FF4807075F0B0FD4FF4007075F0ACFD10BD10B54FF43C
:4049C000806075F0A6FD4FF4006075F0A2FD4FF4805075F09EFD4FF4005075F09AFD4FF4804075F096FD4FF4004075F092FD10BD70B500251748006900F0010038B3002435
:404A00001BE01549096851F8240072F063FAC6B2304608F02DFD054610480068005D38B9012D05D10C49096851F8240072F0B7F80A4800680555601CC4B20948007884423A
:404A4000DFDB0448006920F001000249086170BDE426001000100040580100205C010020600100201CB5FE48006820B9FD487FF0D5FDFB490860FC48FC490860FC4888634A
:404A8000FC4808630020052102231A46CDE900101946F9480078FEF7EDFB0020052102231A46CDE900101946F4480078FEF7E2FB0020052102231A46CDE900101946F04823
:404AC0000078FEF7D7FB0120002102230A46CDE900100146EB480078FEF7CCFB0120002102230A46CDE900100146E7480078FEF7C1FB0120002102230A46CDE9001001466C
:404B0000E2480078FEF7B6FB012000210B460A46CDE900100146DE480078FEF7ABFB0021D24881604FF48270D04948600021CF48C1600221016101214161890481611021B0
:404B4000C16100214162816201620721C16279F02CFDC6480068006840F04000C349096808601CBD1CB5CB48006820B9CA487FF055FDC8490860C948C9490860C9480863A8
:404B8000C94888630020052102231A46CDE900101946C6480078FEF76DFB0020052102231A46CDE900101946C1480078FEF762FB0020052102231A46CDE900101946BD486E
:404BC0000078FEF757FB002000900223024601210190B9480078FEF74DFB002000900223024601460190B5480078FEF743FB002000900223024601460190B1480078FEF778
:404C000039FB002000900223024601210190AD480078FEF72FFB0021A14881604FF482709F49486000219E48C160016101214161890481610021C161416281620162072123
:404C4000C16279F0B2FC96480068006840F040009349096808601CBD38B50446012540F6B8317F4800687FF009FD00287ED1012185480078FEF7A5FA012184480078FEF761
:404C8000A0FA00217F480078FEF79BFA784877498863784808630620096B087073484FF47A630122016B79F055FD0546002D62D1012174480078FEF784FA002171480078DD
:404CC000FEF77FFA6B486949086369488863D820096B0870200C6549096B4870200A6349096B88706149096BCC7060484FF47A530422016B79F02EFD0546002D3BD10121D0
:404D000060480078FEF75DFA00215E480078FEF758FA584855490863554888630520096B08704FF47A6000905048826B0123016B79F000FE0546F5B900BF02207FF0A0FB32
:404D40004C484A4908634A488863A520096B08704FF47A6000904548826B0123016B79F0E9FD05464148806B007800E00CE000F001000028E1D1012142480078FEF721FA6B
:404D8000374800687FF06EFC284638BD70B50446A00C84042046FFF75FFF054685B904F58030FFF759FF054655B904F50030FFF753FF054625B904F54030FFF74DFF05460A
:404DC000284670BD2DE9F04104460F46A00C8404264607E03046FFF73FFF054605B103E006F58026BE42F5D92846BDE8F0812DE9F84380460E461746012440F6B8311848BE
:404E000000687FF03BFC002875D101211E480078FEF7D7F901211D480078FEF7D2F9002118480078FEF7CDF9114810498863114808630620096B08700C484FF47A630122B4
:404E4000016B79F087FC0446002C7DD101210D480078FEF7B6F900210A48007834E000006401002068C70908003001405427001004280010043000108C0000108E00001009
:404E80008D000010890000108A0000108B0000108F000010680100206CC7090800380040AC2700101638001004380010900000109200001091000010A2000010A3000010CE
:404EC000A1000010A0000010FEF77BF9F948FA490863FA4888630220096B0870300CF649096B4870300AF449096B8870F249096BCE70002507E05BE018F80510EE48026B38
:404F0000281D11546D1CBD42F6D307EB4700C0EBC7104FF47A6C0CEBC003381D82B2E648016B79F017FC0446002C38D10121E4480078FEF746F90021E1480078FEF741F9CF
:404F4000DC48DD49086300E029E0DC4888630520096B08704FF47A600090D748826B0123016B79F0E7FC0446CCB900BFD148D2490863D2488863A520096B08704FF47A60DE
:404F80000090CD48826B0123016B79F0D3FC0446C948806B007800F001000028E6D10121C7480078FEF70DF9C64800687FF05AFB2046BDE8F8832DE9F04707460D469146E1
:404FC0004FF0000A2C46280A060205EB090818E006F58070804508D2A8EB0402611BC8192146FFF704FF824608E006F580710A1B611BC8192146FFF7FAFE824606F58076B7
:405000003446444502D2BAF1000FE1D05046BDE8F0872DE9F84F82460E4693464FF00108344606EB0B0940F6B831A64800687FF025FB002862D1804657E00121A248007883
:40504000FEF7BFF80121A1480078FEF7BAF800219B480078FEF7B5F8984897498863954808630320096B0870200C9349096B4870200A9149096B88708F49096BCC7004F515
:405080008070814502D2A9EB040701E04FF48077002505E0A5218848026B281D11546D1CBD42F7D34FF47A7107FB01F000F57A600090381D83B28048826B016B79F03AFCD9
:4050C0008046042507E07D48415D6019801B001F0AF800106D1C381DA842F4D8012178480078FEF76EF804F580744C4502D2B8F1000FA2D0734800687FF0B4FA4046BDE802
:40510000F88F2DE9F04105460E46012740F6B8316F4800687FF0B2FAD8B9002412E06D486D4908636D488863285D096B08706A484FF47A630122016B79F00CFB074607B11D
:4051400002E0641CB442EAD300BF614800687FF089FA3846BDE8F0812DE9F04107460E4615464FF0010840F6B831564800687FF085FA00283FD1012154480078FEF721F8AA
:4051800001214F480078FEF71CF800214E480078FEF717F8474848490863484888630220096B0870300A4449096B48704249096B8E70002405E0395D3F48026BE01C11548A
:4051C000641CAC42F7D305EB4500C0EBC5104FF47A6C0CEBC003E81C82B23748016B79F0B9FA8046012138480078FDF7EAFF354800687FF037FA4046BDE8F0812DE9F84371
:4052000007460E4615464FF0010840F6B8312D4800687FF033FA002849D1012128480078FDF7CFFF012129480078FDF7CAFF002125480078FDF7C5FF20481F4988631D48DE
:4052400008630320096B0870300A1B49096B48701949096B8E70002405E0A5211648026BE01C1154641CAC42F7D34FF47A7105FB01F000F57A600090E81C83B20E48826BE9
:40528000016B79F057FB8046032404E00B48015DE01E3954641CE81CA042F7D801210A480078FDF78EFF074800687FF0DBF94046BDE8F8830430001054270010042800106D
:4052C00089000010640100208A0000108B0000106801002016380010AC270010043800102DE9F0470746884616461D464FF001094FF0FF0A17B1012F06D102E04FF0120A81
:4053000005E04FF0220A02E04FF0FF0A00BF00BFBAF1FF0F48D040F6B831FE4800687FF0ADF9002840D10121FB480078FDF749FF0121FA480078FDF744FF0021F848007884
:40534000FDF73FFFF748F8490863F84888630846006B80F800A0300A096B4870F249096B8E70002406E018F80410EF48026BE01C1154641CAC42F6D305EB4500C0EBC510E2
:405380004FF47A6C0CEBC003E81C82B2E648016B79F0E0F981460121E1480078FDF711FFDC4800687FF05EF94846BDE8F0872DE9F84F0746884616461D464FF001094FF0AD
:4053C000FF0A17B1012F06D102E04FF0130A05E04FF0230A02E04FF0FF0A00BF00BFBAF1FF0F52D040F6B831CA4800687FF046F900284AD10121C9480078FDF7E2FE012198
:40540000C5480078FDF7DDFE0021C5480078FDF7D8FEC648C4498863C24808630846006B80F800A0300A096B4870BF49096B8E70002405E0A521BC48026BE01C1154641C5B
:40544000AC42F7D34FF47A7105FB01F000F57A600090E81C83B2B448826B016B79F06AFA8146032405E0B148015DE01E08F80010641CE81CA042F6D80121A9480078FDF7B0
:40548000A0FEA44800687FF0EDF84846BDE8F88F2DE9F04180460F461546012640F6B8319C4800687FF0EAF8002877D101219C480078FDF786FE012198480078FDF781FEF9
:4054C000002195480078FDF77CFE964896490863964888630620096B087093484FF47A630122016B79F036F90646002E4DD1012189480078FDF765FE002187480078FDF7ED
:4055000060FE884888490863884888630220096B0870380A8449096B48708349096B8F70002406E018F804107F48026BE01C1154641CAC42F6D305EB4500C0EBC5104FF4CC
:405540007A6C0CEBC003E81C82B27748016B79F001F90646CEB901216F480078FDF731FE00216D480078FDF72CFE6E486E4908636E4888630420096B08706B484FF47A63B6
:405580000122016B79F0E6F80646012162480078FDF717FE5F4800687FF064F83046BDE8F0812DE9F84307460E4615464FF0010840F6B831574800687FF060F8002849D152
:4055C000012157480078FDF7FCFD012153480078FDF7F7FD002150480078FDF7F2FD514851490863514888630320096B0870300A4D49096B48704C49096B8E70002405E017
:40560000A5214948026BE01C1154641CAC42F7D34FF47A7105FB01F000F57A600090E81C83B24148826B016B79F084F98046032404E03E48015DE01E3954641CE81C844204
:40564000F7D3012134480078FDF7BBFD314800687FF008F84046BDE8F8832DE9FC4706460F464FF0080A4FF00008002000900190FD0807F0070915B9B9F1000F1FD085B11D
:4056800000240BE006EBC40108226846FFF700FF8046B8F1000F00D002E0641CAC42F1D300BFB9F1000F0CD0B8F1000F09D106EBC5014A466846FFF7EBFE804601E04FF056
:4056C00001084046BDE8FC87F8B506460D46012740F6B831164800687EF0D0FF80BB002430E0144814490863144888630020096B08704FF47A6000900F48826B0123016BF6
:4057000079F018F907460C48806B0178281B401E315416E0640100208B000010890000108A0000100430001054270010042800106801002016380010AC270010043800105A
:4057400006E0641CAC42CCD3074800687EF08AFF3846F8BD10B505487AF02FFC10BD10B503487AF02AFC10BD6801002054270010AC27001038B5044660680090009D2068C9
:4057800080F3088800BFA84738BD10B572B66FF0040000F0FCF96FF0010000F0F8F94FF0FF3000F0F4F9042000F0F1F9052000F0EEF9062000F0EBF9072000F0E8F908206E
:4057C00000F0E5F9092000F0E2F90A2000F0DFF90B2000F0DCF90C2000F0D9F90D2000F0D6F90E2000F0D3F90F2000F0D0F9102000F0CDF9112000F0CAF9122000F0C7F9AD
:40580000132000F0C4F9142000F0C1F9152000F0BEF9162000F0BBF9172000F0B8F9182000F0B5F9192000F0B2F91A2000F0AFF91B2000F0ACF91C2000F0A9F91D2000F0D5
:40584000A6F91E2000F0A3F91F2000F0A0F9202000F09DF9212000F09AF9222000F097F9232000F094F9242000F091F9252000F08EF9262000F08BF9272000F088F92820B7
:4058800000F085F9292000F082F92A2000F07FF92B2000F07CF92C2000F079F92D2000F076F92E2000F073F92F2000F070F9302000F06DF9312000F06AF9322000F067F9CC
:4058C000332000F064F9342000F061F9352000F05EF9362000F05BF9372000F058F9382000F055F9392000F052F93A2000F04FF93B2000F04CF93C2000F049F93D2000F075
:4059000046F93E2000F043F9402000F040F9412000F03DF9422000F03AF9432000F037F9442000F034F9452000F031F9462000F02EF9472000F02BF9482000F028F94920AC
:4059400000F025F94A2000F022F94B2000F01FF94C2000F01CF94D2000F019F94E2000F016F9502000F013F9512000F010F96FF0040000F015F96FF0010000F011F94FF014
:40598000FF3000F00DF9042000F00AF9052000F007F9062000F004F9072000F001F9082000F0FEF8092000F0FBF80A2000F0F8F80B2000F0F5F80C2000F0F2F80D2000F023
:4059C000EFF80E2000F0ECF80F2000F0E9F8102000F0E6F8112000F0E3F8122000F0E0F8132000F0DDF8142000F0DAF8152000F0D7F8162000F0D4F8172000F0D1F81820CE
:405A000000F0CEF8192000F0CBF81A2000F0C8F81B2000F0C5F81C2000F0C2F81D2000F0BFF81E2000F0BCF81F2000F0B9F8202000F0B6F8212000F0B3F8222000F0B0F8D2
:405A4000232000F0ADF8242000F0AAF8252000F0A7F8262000F0A4F8272000F0A1F8282000F09EF8292000F09BF82A2000F098F82B2000F095F82C2000F092F82D2000F0D3
:405A80008FF82E2000F08CF82F2000F089F8302000F086F8312000F083F8322000F080F8332000F07DF8342000F07AF8352000F077F8362000F074F8382000F071F83920CB
:405AC00000F06EF83A2000F06BF83B2000F068F83C2000F065F83D2000F062F83E2000F05FF83F2000F05CF8402000F059F8412000F056F8422000F053F8432000F050F8E8
:405B0000442000F04DF8452000F04AF8462000F047F8472000F044F8482000F041F8492000F03EF84A2000F03BF84B2000F038F84C2000F035F84D2000F032F84E2000F067
:405B40002FF8502000F02CF8512000F029F862B610BD00BF00BF00BF00BF00BFBFF34F8F00BF00BF00BF1348006800F4E06012490843001D0F49086000BF00BF00BFBFF322
:405B80004F8F00BF00BF00BF00BF00BFFDE700F01F0201219140094A430942F82310704700F01F0201219140054A430942F82310704700000CED00E00000FA0580E100E0C5
:405BC00080E200E0A3480068704700B50120A2490870FFF7F7FFA14908600120A04908601EE0A0480068C0F3400078B145F255509D4908600120486040F6B83088604CF6CB
:405C0000CC40086002209449087009E0FFF7DAFF92490968401A642802D903208E4908708D4800780128DCD000BD0EB50020029001908C487438006840F480308949743912
:405C4000086000BF87487438006800F4003001900298401C0290019820B941F2883102988842EFD17F487438006800F4003010B10120019001E0002001900198012865D15F
:405C80007A48784970390860081F006840F08070091F086000BF0020009072483438006840F080506F49343908600846006800F08050009000BF6E48006840F4E0306C49AB
:405CC000086000BF6A48406800F480300028F9D06748006840F400306549086000BF6448406800F400300028F9D05E486C3800685C496C3908600846006840F400400860DF
:405D00000846006840F4A050086000BF55487438006800F000700028F8D040F205605549086050486C38006820F003004D496C3908600846006840F00200086000BF4948CA
:405D40006C38006800F00C000828F8D17BF000FC0EBD38B5FFF769FF00203E4908604649086000BF00903F483438006840F020003C49343908600846006800F020000090F5
:405D800000BF01203D49086059203C491C310860F920091D086037200521002807DA0A07140E374A00F00F031B1FD45403E00A07130E344A135400BF372000F01F020121DA
:405DC00091404209920002F1E022C2F8001100BF05202A490C390860FFF7F7FE38BD2648006870471B480068704710B52348001D006800F0010058B31F480068401C1E49FF
:405E000008600846007800F0030088B911480068401C104908601C480078401C1A49087008460078642801DB00200870F8F74FF9164890F8350018B94AF6AA200A49086061
:405E40000E48001D006820F001000C49091D086010BD0000700100207801002074010020800E474274380240003000400C5A400700700040003C02406C0100200C1400408A
:405E800018ED00E000E400E079010020300A002030B50A46562826DA012A12D1C31700EB5373DB10F74CE35C00F007050124AC4023430146C41700EB5474E410F14D2B5592
:405EC00011E0C31700EB5373DB10EE4CE35C00F007050124AC40A3430146C41700EB5474E410E84D2B5530BD30B501460022562910DA0846CB1701EB5373DB10E14CE35C74
:405F000001F007050124AC4023400BB1012300E000231A46104630BD30B501460023002915DD092913DC481EC1B20846CC1701EB9474A410D44D2C5D0A46CD1701EB957559
:405F4000AD10A1EB85056D002C4104F00303184630BDF0B504460E462046FFF7DDFF0746002C39DD092C37DC601EC4B276B337B1012F20D0022F1FD0032F24D122E0E21776
:405F800004EB92729210C04B9A5C2146E31704EB93739B10A4EB83035B0006FA03F31A432046E31704EB93739B10DFF8DCC20CF80320012509E000BFBE4201D1012500E045
:405FC000002502E000BF002500BF06E0BE4201D1012502E0002500E000252846F0BD30B502460120A94B9A4202D0A94B9A4203D1536C43F400435364012313604FF6FF7320
:40600000D3620023536231B101290FD0022917D003292AD11FE000235363936903F47F439361936943F06003936120E0002393639369DBB29361936943F4C043936116E072
:406040000023D363D36903F47F43D361D36943F06003D3610BE000231364D369DBB2D361D36943F4C043D36101E0002000BF00BF012805D1136A8D000124AC4023431362F8
:4060800030BD0146FF20824A914201D1012035E0B1F1804F01D1012030E07E4A914201D102202BE07C4A914201D1022026E07B4A914201D1022021E0744A914201D1032032
:4060C0001CE0774A914201D1032017E0754A914201D1032012E0744A914201D103200DE0724A914201D1092008E0714A914201D1092003E06F4A914200D10920704730B538
:40610000034601203E2B71D022DC3E2B6FD2DFE803F06E5557595B6E5D5F6163686F74796E6E7B7D7F6E818385878C929496989A9C9EA06E6E6E6E6E6EA2ACB1D36E6E6E94
:406140006E6E6E6E6ED86E6E6E6E6E6E6E6E6EDA592B6FD012DCA3F13F041A2CD6D2DFE804F0B6BBC046464646C2C7CCCED0D2D4D6D8DADC464646464646DEE3802B6FD0A3
:4061800012DC7C2B6DD008DC5A2B6BD0772B6AD07A2B69D07B2B2AD1D9E07D2B6FD07E2B6ED07F2BF7D1E3E0A3F18104082CADD2DFE804F0E21DE7F1F3F5FAFF0020FFE014
:4061C0000020FDE00020FBE00020F9E00020F7E00020F5E00020F3E02D4C0C6000241470EEE02B4C0C6001241470E9E06DE0E5E0274C0C6002241470E2E0254C0C600324BE
:406200001470DDE00020DBE00020D9E00020D7E00020D5E00020D3E00020D1E00020CFE01D4C0C6000241470CAE01B4C0C6001241470C5E07DE00020C2E00020C0E0002003
:40624000BEE00020BCE00020BAE00020B8E00020B6E00020B4E00F4C0C6000241470AFE088E079E067E068E06CE00A4C0C6001241470A5E0074C0C6002241470A0E070E025
:4062800074E00000D41C0020AC00001000040140000001400004004000080040000C004000400140004401400048014000180040001C004000200040FB4C0C60032414705F
:4062C0007EE000207CE000207AE0002078E0F74C0C600224147073E0F44C0C60032414706EE000206CE0F24C0C600024147067E0EF4C0C600124147062E0002060E000206A
:406300005EE000205CE000205AE0002058E0002056E0002054E0002052E0002050E0E54C0C60002414704BE0E34C0C600024147046E0002044E0002042E0E04C0C600024AA
:4063400014703DE0DD4C0C600124147038E0DC4C0C600024147033E0D94C0C60012414702EE0D74C0C600224147029E0002027E0002025E0002023E0D14C0C6003241470AA
:406380001EE0D04C0C600324147019E011E00BE005E002E0FFE7002012E0002010E0C94C0C60002414700BE0C64C0C600124147006E0C44C0C600224147001E0002000BF01
:4063C00000BF18B900240C600424147030BD7CB506460C466A4601A93046FFF790FE05460198FFF74EFE206055B1019840B12068FF2805D09DF800100198FFF7F0FD05469B
:4064000028467CBD03B585B001200490002003900598562885F06585DFE810F06705680569056A056B056C056D056E056F0570056D00A10119027105720573057405750538
:40644000760591026A03430477057A052F06E40607072A074D077007B107D109D209D309D409F2076908D509D609D709D809E1085909D909DA09DB09DE09AE0A7E0B290ED5
:40648000D410A41174121F15CA179A186A193A1A0A1BDA1B511CC91C0B1E2F1FA71F1F20D4205E2D892159222923DD24912674275F2D602D57287C29822A882B8E2C560048
:4064C0005700580059005A0000BF00BF00BF00BF069830B1012806D0022803D0052804D102E000BF00BF00BF02E00020049000BF00BF05F0F9BC06980C287CD2DFE800F00D
:406500000624417B5E7C0799B6E4FCD300BF0020009003460246014601902220FCF7AAFE022200218D20FDF735FF00221146BA20FDF730FF00221146AC20FDF72BFF0021C9
:406540000120FAF7E2FF08E10020009003460246032101902220FCF78DFE022200218D20FDF718FF00221146BA20FDF713FF00221146AC20FDF70EFF00210120FAF7C5FFF6
:40658000EBE00020009003460246032101902220FCF770FE002211468D20FDF7FBFE00221146BA20FDF7F6FE01220021AC20FDF7F1FE00210120FAF7A8FFCEE000200090FE
:4065C00003460246014601902220FCF753FE002211468D20FDF7DEFE03220021BA20FDF7D9FE00221146AC20FDF7D4FE01210846FAF78BFFB1E0ADE0002000900346024676
:40660000032101902220FCF735FE002211468D20FDF7C0FE00221146BA20FDF7BBFE00221146AC20FDF7B6FE00210120FAF76DFF93E000200090034602460146019022200B
:40664000FCF718FE012200218D20FDF7A3FE00221146BA20FDF79EFE00221146AC20FDF799FE00210120FAF750FF76E00020009003460246014601902220FCF7FBFD002298
:4066800011468D20FDF786FE00221146BA20FDF781FE00221146AC20FDF77CFE00210120FAF733FF59E03EE0000400400008004000400140004401400048014000180040B6
:4066C000000C0040000401402220FEF7D2F8012200218D20FDF75EFE00221146BA20FDF759FE00221146AC20FDF754FE00210120FAF70BFF31E0FFE72220FEF7BAF802225D
:4067000000218D20FDF746FE00221146BA20FDF741FE00221146AC20FDF73CFE00210120FAF7F3FE19E02220FEF7A3F8002211468D20FDF72FFE00221146BA20FDF72AFEB5
:4067400000221146AC20FDF725FE00210120FAF7DCFE02E00020049000BF00BFC9E606980C286FD2DFE800F006166E6E6E25073443525B6400BF00200090034602460146C2
:4067800001907020FCF776FD022200218E20FDF701FE5AE00020009003460246032101907020FCF767FD022200218E20FDF7F2FD4BE00020009003460246032101907020CE
:4067C000FCF758FD002211468E20FDF7E3FD3CE00020009003460246014601907020FCF749FD012200218E20FDF7D4FD2DE00020009003460246014601907020FCF73AFDC1
:40680000002211468E20FDF7C5FD1EE07020FEF730F8012200218E20FDF7BCFD15E07020FEF727F8022200218E20FDF7B3FD0CE07020FEF71EF8002211468E20FDF7AAFDB8
:4068400003E0FFE70020049000BF00BF51E606980C286FD2DFE800F006166E6E6E25073443525B6400BF0020009003460246014601903E20FCF7FEFC022200218F20FDF7F7
:4068800089FD5AE00020009003460246032101903E20FCF7EFFC022200218F20FDF77AFD4BE00020009003460246032101903E20FCF7E0FC002211468F20FDF76BFD3CE099
:4068C0000020009003460246014601903E20FCF7D1FC012200218F20FDF75CFD2DE00020009003460246014601903E20FCF7C2FC002211468F20FDF74DFD1EE03E20FDF736
:40690000B8FF012200218F20FDF744FD15E03E20FDF7AFFF022200218F20FDF73BFD0CE03E20FDF7A6FF002211468F20FDF732FD03E0FFE70020049000BF00BFD9E50698DE
:406940000C287DD2DFE800F0061FCFCF374F07678199ABBD00BF0020009003460246014601906720FCF786FC022200219020FDF711FD00221146BC20FDF70CFD0021032043
:40698000FAF7C3FDB2E00020009003460246032101906720FCF76EFC022200219020FDF7F9FC00221146BC20FDF7F4FC00210320FAF7ABFD9AE000200090034602460146C4
:4069C00001906720FCF756FC002211469020FDF7E1FC03220021BC20FDF7DCFC01210320FAF793FD82E00020009003460246032101906720FCF73EFC002211469020FDF763
:406A0000C9FC00221146BC20FDF7C4FC00210320FAF77BFD6AE00020009003460246014601906720FCF726FC012200219020FDF7B1FC00221146BC20FDF7ACFC002100E055
:406A400051E00320FAF761FD50E00020009003460246014601906720FCF70CFC002211469020FDF797FC00221146BC20FDF792FC00210320FAF749FD38E06720FDF7F9FE1C
:406A8000012200219020FDF785FC00221146BC20FDF780FC00210320FAF737FD26E06720FDF7E7FE022200219020FDF773FC00221146BC20FDF76EFC00210320FAF725FD77
:406AC00014E06720FDF7D5FE002211469020FDF761FC00221146BC20FDF75CFC00210320FAF713FD02E00020049000BF00BF00E506980C287ED2DFE800F0061FCFCF374FD9
:406B000007678199ABBD00BF0020009003460246014601906B20FCF7ADFB022200219120FDF738FC00221146BC20FDF733FC00210320FAF7EAFCB2E00020009003460246E3
:406B4000032101906B20FCF795FB022200219120FDF720FC00221146BC20FDF71BFC00210320FAF7D2FC9AE00020009003460246014601906B20FCF77DFB00221146912036
:406B8000FDF708FC03220021BC20FDF703FC01210320FAF7BAFC82E00020009003460246032101906B20FCF765FB002211469120FDF7F0FB00221146BC20FDF7EBFB00214D
:406BC0000320FAF7A2FC6AE00020009003460246014601906B20FCF74DFB012200219120FDF7D8FB00221146BC20FDF7D3FB0021032000E050E0FAF788FC50E0002000903E
:406C000003460246014601906B20FCF733FB002211469120FDF7BEFB00221146BC20FDF7B9FB00210320FAF770FC38E06B20FDF720FE012200219120FDF7ACFB002211460C
:406C4000BC20FDF7A7FB00210320FAF75EFC26E06B20FDF70EFE022200219120FDF79AFB00221146BC20FDF795FB00210320FAF74CFC14E06B20FDF7FCFD00221146912017
:406C8000FDF788FB00221146BC20FDF783FB00210320FAF73AFC02E00020049000BF00BF27E406980C287CD2DFE800F00624417B5E7C0799B6D3EAFE00BF002000900346AC
:406CC0000246014601902520FCF7D4FA022200219220FDF75FFB00221146BA20FDF75AFB00221146AC20FDF755FB00210120FAF70CFCF8E0002000900346024603210190FB
:406D00002520FCF7B7FA022200219220FDF742FB00221146BA20FDF73DFB00221146AC20FDF738FB00210120FAF7EFFBDBE00020009003460246032101902520FCF79AFABD
:406D4000002211469220FDF725FB00221146BA20FDF720FB01220021AC20FDF71BFB00210120FAF7D2FBBEE00020009003460246014601902520FCF77DFA002211469220C7
:406D8000FDF708FB03220021BA20FDF703FB00221146AC20FDF7FEFA01210846FAF7B5FBA1E09DE00020009003460246032101902520FCF75FFA002211469220FDF7EAFA00
:406DC00000221146BA20FDF7E5FA00221146AC20FDF7E0FA00210120FAF797FB83E00020009003460246014601902520FCF742FA012200219220FDF7CDFA00221146BA20A1
:406E0000FDF7C8FA00221146AC20FDF7C3FA00210120FAF77AFB66E00020009003460246014601902520FCF725FA002211469220FDF7B0FA00221146BA20FDF7ABFA002271
:406E40001146AC20FDF7A6FA00210120FAF75DFB49E02520FDF70DFD012200219220FDF799FA00221146BA20FDF794FA00221146AC20FDF78FFA00210120FAF746FB32E0CA
:406E80002520FDF7F6FC022200219220FDF782FA00221146BA20FDF77DFA00221146AC20FDF778FA002100E003E00120FAF72DFB19E02520FDF7DDFC002211469220FDF78F
:406EC00069FA00221146BA20FDF764FA00221146AC20FDF75FFA00210120FAF716FB02E00020049000BF00BF38E400BF00BF00BF00BF00BF00BF00BF00BF00BF00BF00BF4F
:406F000000BF00BF00BF00BF00BF0020049025E406980D284CD005DC58B101280AD00C287ED126E00E2852D00F2866D0102877D18AE000BF00200090034602460121019012
:406F40002920FCF797F90020009003460246012101904F20FCF78EF901210920FEF7F9FF04990840049000221146EC20FDF712FA81E0002000900346024601210190292094
:406F8000FCF778F90020009003460246012101904F20FCF76FF901210920FEF7DAFF04990840049001220021EC20FDF7F3F962E00020009003460246012101902920FCF77B
:406FC00059F901220021EC20FDF7E4F953E00020009003460246012101904F20FCF74AF903210920FEF7B5FF04990840049001220021EC20FDF7CEF93DE003A92920FFF7D0
:40700000E6F90020039903460246CDE9001002212920FCF72FF9012000210B460A4600E026E0CDE9001001464F20FCF723F902210920FEF78EFF04990840049001220021F8
:40704000EC20FDF7A7F916E003A92920FFF7BFF90020039903460246CDE9001002212920FCF708F901220021EC20FDF793F902E00020049000BF00BF60E406980D284CD04D
:4070800005DC58B101280AD00C287DD126E00E2852D00F2866D0102876D18AE000BF0020009003460246012101902A20FCF7E2F80020009003460246012101904F20FCF78D
:4070C000D9F801210920FEF744FF04990840049000221146EB20FDF75DF981E00020009003460246012101902A20FCF7C3F80020009003460246012101904F20FCF7BAF8A0
:4071000001210920FEF725FF04990840049001220021EB20FDF73EF962E00020009003460246012101902A20FCF7A4F801220021EB20FDF72FF953E000200090034602460A
:40714000012101904F20FCF795F803210920FEF700FF04990840049001220021EB20FDF719F93DE003A92A20FFF731F90020039903460246CDE9001002212A20FCF77AF846
:40718000012000210B4600E027E00A46CDE9001001464F20FCF76EF802210920FEF7D9FE04990840049001220021EB20FDF7F2F816E003A92A20FFF70AF900200399034688
:4071C0000246CDE9001002212A20FCF753F801220021EB20FDF7DEF802E00020049000BF00BF84E4069820B1012803D00C2817D10BE000BF00221146D220FDF7CBF80022CC
:407200001146F720FDF7C6F80DE000221146D220FDF7C0F801220021F720FDF7BBF802E00020049000BF00BF61E4069820B1012803D00C2817D10BE000BF00221146D32032
:40724000FDF7A8F800221146F820FDF7A3F80DE000221146D320FDF79DF801220021F820FDF798F802E00020049000BF00BF3EE4069820B1012803D00C2817D10BE000BF31
:4072800000221146D420FDF785F800221146F920FDF780F80DE000221146D420FDF77AF801220021F920FDF775F802E00020049000BF00BF1BE4069820B1012803D00C28C2
:4072C00017D10BE000BF00221146D520FDF762F800221146FA20FDF75DF80DE000221146D520FDF757F801220021FA20FDF752F802E00020049000BF00BFD1E4069830B1E2
:40730000012805D00C2812D00F2833D11EE000BF0020009003460246012101908820FBF7A9FF00221146F520FDF734F825E00020009003460246012101908820FBF79AFF31
:4073400001220021F520FDF725F816E003A98820FFF73DF80020039903460246CDE9001002218820FBF786FF01220021F520FDF711F802E00020049000BF00BF90E406985D
:4073800030B1012805D00C2812D00F2833D11EE000BF0020009003460246012101908320FBF768FF00221146F620FCF7F3FF25E00020009003460246012101908320FBF7EE
:4073C00059FF01220021F620FCF7E4FF16E003A98320FEF7FCFF0020039903460246CDE9001002218320FBF745FF01220021F620FCF7D0FF02E00020049000BF00BF4FE45E
:4074000006980C286ED2DFE800F006166D6D6D25073443525B6400BF0020009003460246014601902D20FBF725FF022200219320FCF7B0FF59E000200090034602460321F9
:4074400001902D20FBF716FF022200219320FCF7A1FF4AE00020009003460246032101902D20FBF707FF002211469320FCF792FF3BE00020009003460246014601902D2006
:40748000FBF7F8FE012200219320FCF783FF2CE00020009003460246014601902D20FBF7E9FE002211469320FCF774FF1DE02D20FDF7DFF9012200219320FCF76BFF14E03D
:4074C0002D20FDF7D6F9022200219320FCF762FF0BE02D20FDF7CDF9002211469320FCF759FF02E00020049000BF00BFFCE406980C286FD2DFE800F006166E6E6E25073443
:4075000043525B6400BF0020009003460246014601903020FBF7AEFE022200219420FCF739FF5AE00020009003460246032101903020FBF79FFE022200219420FCF72AFFE9
:407540004BE00020009003460246032101903020FBF790FE002211469420FCF71BFF3CE00020009003460246014601903020FBF781FE012200219420FCF70CFF2DE00020C7
:40758000009003460246014601903020FBF772FE002211469420FCF7FDFE1EE03020FDF768F9012200219420FCF7F4FE15E03020FDF75FF9022200219420FCF7EBFE0CE033
:4075C0003020FDF756F9002211469420FCF7E2FE03E0FFE70020049000BF00BF84E406980C286FD2DFE800F006166E6E6E25073443525B6400BF002000900346024601466A
:4076000001902F20FBF736FE022200219520FCF7C1FE5AE00020009003460246032101902F20FBF727FE022200219520FCF7B2FE4BE00020009003460246032101902F20F5
:40764000FBF718FE002211469520FCF7A3FE3CE00020009003460246014601902F20FBF709FE012200219520FCF794FE2DE00020009003460246014601902F20FBF7FAFDE7
:40768000002211469520FCF785FE1EE02F20FDF7F0F8012200219520FCF77CFE15E02F20FDF7E7F8022200219520FCF773FE0CE02F20FDF7DEF8002211469520FCF76AFE94
:4076C00003E0FFE70020049000BF00BF0CE406980C286FD2DFE800F006166E6E6E25073443525B6400BF0020009003460246014601902E20FBF7BEFD022200219620FCF7FA
:4077000049FE5AE00020009003460246032101902E20FBF7AFFD022200219620FCF73AFE4BE00020009003460246032101902E20FBF7A0FD002211469620FCF72BFE3CE05B
:407740000020009003460246014601902E20FBF791FD012200219620FCF71CFE2DE00020009003460246014601902E20FBF782FD002211469620FCF70DFE1EE02E20FDF7C9
:4077800078F8012200219620FCF704FE15E02E20FDF76FF8022200219620FCF7FBFD0CE02E20FDF766F8002211469620FCF7F2FD03E0FFE70020049000BF00BF5CE400BF4F
:4077C00000BF00BF00BF00BF00BF00BF00BF00BF00BF002004904FE406980E285AD005DC58B10C2828D00D287DD144E00F2867D0102879D0112876D19EE00020009003464A
:407800000246012101907B20FBF734FD0020009003460246012101908720FBF72BFD01210620FEF796FB04990840049000221146E620FCF7AFFD9DE00020009003460246B7
:40784000012101907B20FBF715FD0020009003460246012101908720FBF70CFD01210620FEF777FB04990840049001220021E620FCF790FD7EE0002000900346024601216D
:4078800001907B20FBF7F6FC01220021E620FCF781FD6FE00020009003460246012101908720FBF7E7FC03210620FEF752FB04990840049001220021E620FCF76BFD59E05B
:4078C00003A97B20FEF783FD0020039903460246CDE9001002217B20FBF7CCFC012000210B460A4601E042E012E0CDE9001001468720FBF7BFFC02210620FEF72AFB049908
:407900000840049001220021E620FCF743FD31E003A97B20FEF75BFD0020039903460246CDE9001002217B20FBF7A4FC01220021E620FCF72FFD1DE003A98720FEF747FDF4
:407940000020039903460246CDE9001002218720FBF790FC03210620FEF7FBFA04990840049001220021E620FCF714FD02E00020049000BF00BF34E406980E285AD005DCA6
:4079800058B10C2828D00D287DD144E00F2867D0102879D0112876D19EE00020009003460246012101907C20FBF764FC0020009003460246012101908720FBF75BFC012116
:4079C0000620FEF7C6FA04990840049000221146E520FCF7DFFC9DE00020009003460246012101907C20FBF745FC0020009003460246012101908720FBF73CFC012106209A
:407A0000FEF7A7FA04990840049001220021E520FCF7C0FC7EE00020009003460246012101907C20FBF726FC01220021E520FCF7B1FC6FE000200090034602460121019011
:407A40008720FBF717FC03210620FEF782FA04990840049001220021E520FCF79BFC59E003A97C20FEF7B3FC0020039903460246CDE9001002217C20FBF7FCFB0120002131
:407A80000B460A4601E042E012E0CDE9001001468720FBF7EFFB02210620FEF75AFA04990840049001220021E520FCF773FC31E003A97C20FEF78BFC0020039903460246C8
:407AC000CDE9001002217C20FBF7D4FB01220021E520FCF75FFC1DE003A98720FEF777FC0020039903460246CDE9001002218720FBF7C0FB03210620FEF72BFA049908401E
:407B0000049001220021E520FCF744FC02E00020049000BF00BF31E4069811286FD2DFE800F0096FA16E6ED30AFDFCFBFAF93CF8F7F6F50000BF0020009003460246014627
:407B400001903A20FBF796FB0020009003460246012101904020FBF78DFB0020009003460246012101905C20FBF784FB01210820FEF7EFF90499084004900222002197204C
:407B8000FCF708FC00221146AE20FCF703FC00221146E920FCF7FEFB67E20020009003460246014601903A20FBF764FB0020009003460246012101904020FBF75BFB00205E
:407BC000009003460246012101905C20FBF752FB01210820FEF7BDF9049908400490022200219720FCF7D6FB00221146AE20FCF7D1FB01220021E920FCF7CCFB35E231E291
:407C00000020009003460246032101903A20FBF731FB0020009003460246012101904020FBF728FB0020009003460246012101905C20FBF71FFB01210820FEF78AF9049992
:407C400008400490022200219720FCF7A3FB00221146AE20FCF79EFB00221146E920FCF799FB02E20020009003460246032101903A20FBF7FFFA002000900346024601213D
:407C800001904020FBF7F6FA0020009003460246012101905C20FBF7EDFA01210820FEF758F9049908400490002211469720FCF771FB01220021AE20FCF76CFB002211462B
:407CC000E920FCF767FBD0E10020009003460246032101903A20FBF7CDFA0020009003460246012101904020FBF7C4FA0020009003460246012101905C20FBF7BBFA01212F
:407D00000820FEF726F90499084008E083E14AE120E1FDE0D0E0A3E076E043E010E00490002211469720FCF735FB00221146AE20FCF730FB00221146E920FCF72BFB94E1D5
:407D40000020009003460246014601903A20FBF791FA0020009003460246012101904020FBF788FA0020009003460246012101905C20FBF77FFA01210820FEF7EAF80499B2
:407D800008400490012200219720FCF703FB00221146AE20FCF7FEFA00221146E920FCF7F9FA62E10020009003460246014601903A20FBF75FFA00200090034602460121FD
:407DC00001904020FBF756FA0020009003460246012101905C20FBF74DFA01210820FEF7B8F8049908400490002211469720FCF7D1FA00221146AE20FCF7CCFA00221146D8
:407E0000E920FCF7C7FA30E13A20FCF732FD0020009003460246012101904020FBF72AFA0020009003460246012101905C20FBF721FA01210820FEF78CF8049908400490D5
:407E4000012200219720FCF7A5FA00221146AE20FCF7A0FA00221146E920FCF79BFA04E13A20FCF706FD0020009003460246012101904020FBF7FEF90020009003460246E4
:407E8000012101905C20FBF7F5F901210820FEF760F8049908400490022200219720FCF779FA00221146AE20FCF774FA00221146E920FCF76FFAD8E03A20FCF7DAFC0020C0
:407EC000009003460246012101904020FBF7D2F90020009003460246012101905C20FBF7C9F901210820FEF734F8049908400490002211469720FCF74DFA00221146AE20D8
:407F0000FCF748FA00221146E920FCF743FAACE00020009003460246014601903A20FBF7A9F90020009003460246012101904020FBF7A0F9022200219720FCF72BFA0022B2
:407F40001146AE20FCF726FA01220021E920FCF721FA8AE00020009003460246014601903A20FBF787F90020009003460246012101905C20FBF77EF903210820FDF7E9FF1E
:407F8000049908400490022200219720FCF702FA00221146AE20FCF7FDF901220021E920FCF7F8F961E00020009003460246014601903A20FBF75EF903A94020FEF707FAFD
:407FC0000020039903460246CDE9001002214020FBF750F9012000210B460A46CDE9001001465C20FBF746F902210820FDF7B1FF049908400490022200219720FCF7CAF9F9
:4080000000221146AE20FCF7C5F901220021E920FCF7C0F929E00020009003460246014601903A20FBF726F903A94020FEF7CFF90020039903460246CDE900100221402063
:40804000FBF718F9022200219720FCF7A3F900221146AE20FCF79EF901220021E920FCF799F902E00020049000BF00BF83E4069811286FD2DFE800F0096FA16E6ED30AFEB5
:40808000FDFCFBFA3CF9F8F7F60000BF0020009003460246014601906C20FBF7EBF80020009003460246012101903F20FBF7E2F80020009003460246012101905C20FBF7FE
:4080C000D9F801210820FDF744FF049908400490022200219820FCF75DF900221146AE20FCF758F900221146EA20FCF753F967E20020009003460246014601906C20FBF742
:40810000B9F80020009003460246012101903F20FBF7B0F80020009003460246012101905C20FBF7A7F801210820FDF712FF049908400490022200219820FCF72BF90022A2
:408140001146AE20FCF726F901220021EA20FCF721F935E231E20020009003460246032101906C20FBF786F80020009003460246012101903F20FBF77DF80020009003469E
:408180000246012101905C20FBF774F801210820FDF7DFFE049908400490022200219820FCF7F8F800221146AE20FCF7F3F800221146EA20FCF7EEF802E200200090034618
:4081C0000246032101906C20FBF754F80020009003460246012101903F20FBF74BF80020009003460246012101905C20FBF742F801210820FDF7ADFE049908400490002210
:4082000011469820FCF7C6F801220021AE20FCF7C1F800221146EA20FCF7BCF8D0E10020009003460246032101906C20FBF722F80020009003460246012101903F20FBF712
:4082400019F80020009003460246012101905C20FBF710F801210820FDF77BFE04990840049008E082E149E11FE1FCE0CFE0A2E075E042E00FE0002211469820FCF78AF8C5
:4082800000221146AE20FCF785F800221146EA20FCF780F894E10020009003460246014601906C20FAF7E6FF0020009003460246012101903F20FAF7DDFF00200090034610
:4082C0000246012101905C20FAF7D4FF01210820FDF73FFE049908400490012200219820FCF758F800221146AE20FCF753F800221146EA20FCF74EF862E100200090034693
:408300000246014601906C20FAF7B4FF0020009003460246012101903F20FAF7ABFF0020009003460246012101905C20FAF7A2FF01210820FDF70DFE049908400490002219
:4083400011469820FCF726F800221146AE20FCF721F800221146EA20FCF71CF830E16C20FCF787FA0020009003460246012101903F20FAF77FFF00200090034602460121CA
:4083800001905C20FAF776FF01210820FDF7E1FD049908400490012200219820FBF7FAFF00221146AE20FBF7F5FF00221146EA20FBF7F0FF04E16C20FCF75BFA00200090D4
:4083C00003460246012101903F20FAF753FF0020009003460246012101905C20FAF74AFF01210820FDF7B5FD049908400490022200219820FBF7CEFF00221146AE20FBF78F
:40840000C9FF00221146EA20FBF7C4FFD8E06C20FCF72FFA0020009003460246012101903F20FAF727FF0020009003460246012101905C20FAF71EFF01210820FDF789FD30
:40844000049908400490002211469820FBF7A2FF00221146AE20FBF79DFF00221146EA20FBF798FFACE00020009003460246014601906C20FAF7FEFE00200090034602467F
:40848000012101903F20FAF7F5FE022200219820FBF780FF00221146AE20FBF77BFF01220021EA20FBF776FF8AE00020009003460246014601906C20FAF7DCFE0020009066
:4084C00003460246012101905C20FAF7D3FE03210820FDF73EFD049908400490022200219820FBF757FF00221146AE20FBF752FF01220021EA20FBF74DFF61E000200090BA
:4085000003460246014601906C20FAF7B3FE03A93F20FDF75CFF0020039903460246CDE9001002213F20FAF7A5FE012000210B460A46CDE9001001465C20FAF79BFE022108
:408540000820FDF706FD049908400490022200219820FBF71FFF00221146AE20FBF71AFF01220021EA20FBF715FF29E00020009003460246014601906C20FAF77BFE03A9EC
:408580003F20FDF724FF0020039903460246CDE9001002213F20FAF76DFE022200219820FBF7F8FE00221146AE20FBF7F3FE01220021EA20FBF7EEFE02E00020049000BFC4
:4085C00000BF53E506980E285AD005DC58B10C2828D00D287DD144E00F2867D0102879D0112876D19EE00020009003460246012101901720FAF73EFE002000900346024643
:40860000012101908620FAF735FE01210520FDF7A0FC04990840049000221146E420FBF7B9FE9DE00020009003460246012101901720FAF71FFE002000900346024601212E
:4086400001908620FAF716FE01210520FDF781FC04990840049001220021E420FBF79AFE7EE00020009003460246012101901720FAF700FE01220021E420FBF78BFE6FE031
:408680000020009003460246012101908620FAF7F1FD03210520FDF75CFC04990840049001220021E420FBF775FE59E003A91720FDF78DFE0020039903460246CDE90010D8
:4086C00002211720FAF7D6FD012000210B460A4601E042E012E0CDE9001001468620FAF7C9FD02210520FDF734FC04990840049001220021E420FBF74DFE31E003A91720BC
:40870000FDF765FE0020039903460246CDE9001002211720FAF7AEFD01220021E420FBF739FE1DE003A98620FDF751FE0020039903460246CDE9001002218620FAF79AFD72
:4087400003210520FDF705FC04990840049001220021E420FBF71EFE02E00020049000BF00BF83E406980E285AD005DC58B10C2828D00D287DD144E00F2867D0102879D0C7
:40878000112876D19EE00020009003460246012101901820FAF76EFD0020009003460246012101908620FAF765FD01210520FDF7D0FB04990840049000221146E320FBF759
:4087C000E9FD9DE00020009003460246012101901820FAF74FFD0020009003460246012101908620FAF746FD01210520FDF7B1FB04990840049001220021E320FBF7CAFD7F
:408800007EE00020009003460246012101901820FAF730FD01220021E320FBF7BBFD6FE00020009003460246012101908620FAF721FD03210520FDF78CFB0499084004906A
:4088400001220021E320FBF7A5FD59E003A91820FDF7BDFD0020039903460246CDE9001002211820FAF706FD012000210B460A4601E042E012E0CDE9001001468620FAF774
:40888000F9FC02210520FDF764FB04990840049001220021E320FBF77DFD31E003A91820FDF795FD0020039903460246CDE9001002211820FAF7DEFC01220021E320FBF70F
:4088C00069FD1DE003A98620FDF781FD0020039903460246CDE9001002218620FAF7CAFC03210520FDF735FB04990840049001220021E320FBF74EFD02E00020049000BFFF
:4089000000BF5EE6069811286FD2DFE800F0096FA16E6ED30AFDFCFBFAF93CF8F7F6F50000BF0020009003460246014601906E20FAF7A0FC002000900346024601210190AF
:408940008120FAF797FC0020009003460246012101903B20FAF78EFC01210720FDF7F9FA049908400490022200219920FBF712FD00221146AE20FBF70DFD00221146E7209D
:40898000FBF708FD67E20020009003460246014601906E20FAF76EFC0020009003460246012101908120FAF765FC0020009003460246012101903B20FAF75CFC01210720AD
:4089C000FDF7C7FA049908400490022200219920FBF7E0FC00221146AE20FBF7DBFC01220021E720FBF7D6FC35E231E20020009003460246032101906E20FAF73BFC002068
:408A0000009003460246012101908120FAF732FC0020009003460246012101903B20FAF729FC01210720FDF794FA049908400490022200219920FBF7ADFC00221146AE2019
:408A4000FBF7A8FC00221146E720FBF7A3FC02E20020009003460246032101906E20FAF709FC0020009003460246012101908120FAF700FC0020009003460246012101907B
:408A80003B20FAF7F7FB01210720FDF762FA049908400490002211469920FBF77BFC01220021AE20FBF776FC00221146E720FBF771FCD0E1002000900346024603210190CF
:408AC0006E20FAF7D7FB0020009003460246012101908120FAF7CEFB0020009003460246012101903B20FAF7C5FB01210720FDF730FA0499084008E083E14AE120E1FDE035
:408B0000D0E0A3E076E043E010E00490002211469920FBF73FFC00221146AE20FBF73AFC00221146E720FBF735FC94E10020009003460246014601906E20FAF79BFB0020D1
:408B4000009003460246012101908120FAF792FB0020009003460246012101903B20FAF789FB01210720FDF7F4F9049908400490012200219920FBF70DFC00221146AE205C
:408B8000FBF708FC00221146E720FBF703FC62E10020009003460246014601906E20FAF769FB0020009003460246012101908120FAF760FB0020009003460246012101903A
:408BC0003B20FAF757FB01210720FDF7C2F9049908400490002211469920FBF7DBFB00221146AE20FBF7D6FB00221146E720FBF7D1FB30E16E20FBF73CFE00200090034660
:408C00000246012101908120FAF734FB0020009003460246012101903B20FAF72BFB01210720FDF796F9049908400490012200219920FBF7AFFB00221146AE20FBF7AAFB56
:408C400000221146E720FBF7A5FB04E16E20FBF710FE0020009003460246012101908120FAF708FB0020009003460246012101903B20FAF7FFFA01210720FDF76AF9049970
:408C800008400490022200219920FBF783FB00221146AE20FBF77EFB00221146E720FBF779FBD8E06E20FBF7E4FD0020009003460246012101908120FAF7DCFA00200090AD
:408CC00003460246012101903B20FAF7D3FA01210720FDF73EF9049908400490002211469920FBF757FB00221146AE20FBF752FB00221146E720FBF74DFBACE00020009038
:408D000003460246014601906E20FAF7B3FA0020009003460246012101908120FAF7AAFA022200219920FBF735FB00221146AE20FBF730FB01220021E720FBF72BFB8AE023
:408D40000020009003460246014601906E20FAF791FA0020009003460246012101903B20FAF788FA03210720FDF7F3F8049908400490022200219920FBF70CFB00221146FB
:408D8000AE20FBF707FB01220021E720FBF702FB61E00020009003460246014601906E20FAF768FA03A98120FDF711FB0020039903460246CDE9001002218120FAF75AFA13
:408DC000012000210B460A46CDE9001001463B20FAF750FA02210720FDF7BBF8049908400490022200219920FBF7D4FA00221146AE20FBF7CFFA01220021E720FBF7CAFAC2
:408E000029E00020009003460246014601906E20FAF730FA03A98120FDF7D9FA0020039903460246CDE9001002218120FAF722FA022200219920FBF7ADFA00221146AE2091
:408E4000FBF7A8FA01220021E720FBF7A3FA02E00020049000BF00BF83E4069811286FD2DFE800F0096FA16E6ED30AFEFDFCFBFA3CF9F8F7F60000BF002000900346024662
:408E8000014601906820FAF7F5F90020009003460246012101907D20FAF7ECF90020009003460246012101903B20FAF7E3F901210720FDF74EF804990840049002220021AF
:408EC0009A20FBF767FA00221146AE20FBF762FA00221146E820FBF75DFA67E20020009003460246014601906820FAF7C3F90020009003460246012101907D20FAF7BAF93A
:408F00000020009003460246012101903B20FAF7B1F901210720FDF71CF8049908400490022200219A20FBF735FA00221146AE20FBF730FA01220021E820FBF72BFA35E280
:408F400031E20020009003460246032101906820FAF790F90020009003460246012101907D20FAF787F90020009003460246012101903B20FAF77EF901210720FCF7E9FF09
:408F8000049908400490022200219A20FBF702FA00221146AE20FBF7FDF900221146E820FBF7F8F902E20020009003460246032101906820FAF75EF90020009003460246CD
:408FC000012101907D20FAF755F90020009003460246012101903B20FAF74CF901210720FCF7B7FF049908400490002211469A20FBF7D0F901220021AE20FBF7CBF900221A
:409000001146E820FBF7C6F9D0E10020009003460246032101906820FAF72CF90020009003460246012101907D20FAF723F90020009003460246012101903B20FAF71AF9EA
:4090400001210720FCF785FF04990840049008E082E149E11FE1FCE0CFE0A2E075E042E00FE0002211469A20FBF794F900221146AE20FBF78FF900221146E820FBF78AF966
:4090800094E10020009003460246014601906820FAF7F0F80020009003460246012101907D20FAF7E7F80020009003460246012101903B20FAF7DEF801210720FCF749FFC6
:4090C000049908400490012200219A20FBF762F900221146AE20FBF75DF900221146E820FBF758F962E10020009003460246014601906820FAF7BEF800200090034602468D
:40910000012101907D20FAF7B5F80020009003460246012101903B20FAF7ACF801210720FCF717FF049908400490002211469A20FBF730F900221146AE20FBF72BF90022C5
:409140001146E820FBF726F930E16820FBF791FB0020009003460246012101907D20FAF789F80020009003460246012101903B20FAF780F801210720FCF7EBFE04990840A3
:409180000490012200219A20FBF704F900221146AE20FBF7FFF800221146E820FBF7FAF804E16820FBF765FB0020009003460246012101907D20FAF75DF80020009003460A
:4091C0000246012101903B20FAF754F801210720FCF7BFFE049908400490022200219A20FBF7D8F800221146AE20FBF7D3F800221146E820FBF7CEF8D8E06820FBF739FB06
:409200000020009003460246012101907D20FAF731F80020009003460246012101903B20FAF728F801210720FCF793FE049908400490002211469A20FBF7ACF8002211469B
:40924000AE20FBF7A7F800221146E820FBF7A2F8ACE00020009003460246014601906820FAF708F80020009003460246012101907D20F9F7FFFF022200219A20FBF78AF872
:4092800000221146AE20FBF785F801220021E820FBF780F88AE00020009003460246014601906820F9F7E6FF0020009003460246012101903B20F9F7DDFF03210720FCF709
:4092C00048FE049908400490022200219A20FBF761F800221146AE20FBF75CF801220021E820FBF757F861E00020009003460246014601906820F9F7BDFF03A97D20FDF780
:4093000066F80020039903460246CDE9001002217D20F9F7AFFF012000210B460A46CDE9001001463B20F9F7A5FF02210720FCF710FE049908400490022200219A20FBF7CA
:4093400029F800221146AE20FBF724F801220021E820FBF71FF829E00020009003460246014601906820F9F785FF03A97D20FDF72EF80020039903460246CDE9001002216B
:409380007D20F9F777FF022200219A20FBF702F800221146AE20FAF7FDFF01220021E820FAF7F8FF02E00020049000BF00BF53E506980E285AD005DC58B10C2828D00D28C2
:4093C0007DD144E00F2867D0102879D0112876D19EE00020009003460246012101902720F9F748FF0020009003460246012101900C20F9F73FFF01210420FCF7AAFD0499D1
:409400000840049000221146E220FAF7C3FF9DE00020009003460246012101902720F9F729FF0020009003460246012101900C20F9F720FF01210420FCF78BFD049908407D
:40944000049001220021E220FAF7A4FF7EE00020009003460246012101902720F9F70AFF01220021E220FAF795FF6FE00020009003460246012101900C20F9F7FBFE0321A5
:409480000420FCF766FD04990840049001220021E220FAF77FFF59E003A92720FCF797FF0020039903460246CDE9001002212720F9F7E0FE012000210B460A4601E042E01E
:4094C00012E0CDE9001001460C20F9F7D3FE02210420FCF73EFD04990840049001220021E220FAF757FF31E003A92720FCF76FFF0020039903460246CDE900100221272023
:40950000F9F7B8FE01220021E220FAF743FF1DE003A90C20FCF75BFF0020039903460246CDE9001002210C20F9F7A4FE03210420FCF70FFD04990840049001220021E220F0
:40954000FAF728FF02E00020049000BF00BF83E406980E285AD005DC58B10C2828D00D287DD144E00F2867D0102879D0112876D19EE0002000900346024601210190282074
:40958000F9F778FE0020009003460246012101900C20F9F76FFE01210420FCF7DAFC04990840049000221146E120FAF7F3FE9DE00020009003460246012101902820F9F73B
:4095C00059FE0020009003460246012101900C20F9F750FE01210420FCF7BBFC04990840049001220021E120FAF7D4FE7EE00020009003460246012101902820F9F73AFE83
:4096000001220021E120FAF7C5FE6FE00020009003460246012101900C20F9F72BFE03210420FCF796FC04990840049001220021E120FAF7AFFE59E003A92820FCF7C7FE9B
:409640000020039903460246CDE9001002212820F9F710FE012000210B460A4601E042E012E0CDE9001001460C20F9F703FE02210420FCF76EFC049908400490012200210B
:40968000E120FAF787FE31E003A92820FCF79FFE0020039903460246CDE9001002212820F9F7E8FD01220021E120FAF773FE1DE003A90C20FCF78BFE002003990346024606
:4096C000CDE9001002210C20F9F7D4FD03210420FCF73FFC04990840049001220021E120FAF758FE02E00020049000BF00BF5EE606980E285AD005DC58B10C2828D00D2878
:409700007DD144E00F2867D0102879D0112876D19EE00020009003460246012101905820F9F7A8FD0020009003460246012101900B20F9F79FFD01210320FCF70AFC049943
:409740000840049000221146DF20FAF723FE9DE00020009003460246012101905820F9F789FD0020009003460246012101900B20F9F780FD01210320FCF7EBFB0499084095
:40978000049001220021DF20FAF704FE7EE00020009003460246012101905820F9F76AFD01220021DF20FAF7F5FD6FE00020009003460246012101900B20F9F75BFD0321BE
:4097C0000846FCF7C6FB04990840049001220021DF20FAF7DFFD59E003A95820FCF7F7FD0020039903460246CDE9001002215820F9F740FD012000210B460A4601E042E0D9
:4098000012E0CDE9001001460B20F9F733FD02210320FCF79EFB04990840049001220021DF20FAF7B7FD31E003A95820FCF7CFFD0020039903460246CDE900100221582009
:40984000F9F718FD01220021DF20FAF7A3FD1DE003A90B20FCF7BBFD0020039903460246CDE9001002210B20F9F704FD03210846FCF76FFB04990840049001220021DF20B3
:40988000FAF788FD02E00020049000BF00BF8EE506980E285AD005DC58B10C2828D00D287DD144E00F2867D0102879D0112876D19EE0002000900346024601210190572098
:4098C000F9F7D8FC0020009003460246012101900B20F9F7CFFC01210320FCF73AFB04990840049000221146E020FAF753FD9DE00020009003460246012101905720F9F752
:40990000B9FC0020009003460246012101900B20F9F7B0FC01210320FCF71BFB04990840049001220021E020FAF734FD7EE00020009003460246012101905720F9F79AFC3B
:4099400001220021E020FAF725FD6FE00020009003460246012101900B20F9F78BFC03210846FCF7F6FA04990840049001220021E020FAF70FFD59E003A95720FCF727FD29
:409980000020039903460246CDE9001002215720F9F770FC012000210B460A4601E042E012E0CDE9001001460B20F9F763FC02210320FCF7CEFA0499084004900122002181
:4099C000E020FAF7E7FC31E003A95720FCF7FFFC0020039903460246CDE9001002215720F9F748FC01220021E020FAF7D3FC1DE003A90B20FCF7EBFC002003990346024691
:409A0000CDE9001002210B20F9F734FC03210846FCF79FFA04990840049001220021E020FAF7B8FC02E00020049000BF00BFBEE406980E285AD005DC58B10C2828D00D2893
:409A40007DD144E00F2867D0102879D0112876D19EE00020009003460246012101907720F9F708FC0020009003460246012101900A20F9F7FFFB01210220FCF76AFA0499C8
:409A80000840049000221146DE20FAF783FC9DE00020009003460246012101907720F9F7E9FB0020009003460246012101900A20F9F7E0FB01210220FCF74BFA04990840BD
:409AC000049001220021DE20FAF764FC7EE00020009003460246012101907720F9F7CAFB01220021DE20FAF755FC6FE00020009003460246012101900A20F9F7BBFB0321E6
:409B00000220FCF726FA04990840049001220021DE20FAF73FFC59E003A97720FCF757FC0020039903460246CDE9001002217720F9F7A0FB012000210B460A4601E042E009
:409B400012E0CDE9001001460A20F9F793FB02210846FCF7FEF904990840049001220021DE20FAF717FC31E003A97720FCF72FFC0020039903460246CDE9001002217720E5
:409B8000F9F778FB01220021DE20FAF703FC1DE003A90A20FCF71BFC0020039903460246CDE9001002210A20F9F764FB03210220FCF7CFF904990840049001220021DE20C8
:409BC000FAF7E8FB02E00020049000BF00BFBEE406980C286ED2DFE800F006166D6D6D25073443525B6400BF0020009003460246014601900120F9F73DFB022200219B20DA
:409C0000FAF7C8FB59E00020009003460246032101900120F9F72EFB022200219B20FAF7B9FB4AE00020009003460246032101900120F9F71FFB002211469B20FAF7AAFB4D
:409C40003BE00020009003460246014601900120F9F710FB012200219B20FAF79BFB2CE00020009003460246014601900120F9F701FB002211469B20FAF78CFB1DE0012012
:409C8000FAF7F7FD012200219B20FAF783FB14E00120FAF7EEFD022200219B20FAF77AFB0BE00120FAF7E5FD002211469B20FAF771FB02E00020049000BF00BF47E40698AD
:409CC0000C286FD2DFE800F006166E6E6E25073443525B6400BF0020009003460246014601900220F9F7C6FA022200219C20FAF751FB5AE000200090034602460321019006
:409D00000220F9F7B7FA022200219C20FAF742FB4BE00020009003460246032101900220F9F7A8FA002211469C20FAF733FB3CE00020009003460246014601900220F9F7C1
:409D400099FA012200219C20FAF724FB2DE00020009003460246014601900220F9F78AFA002211469C20FAF715FB1EE00220FAF780FD012200219C20FAF70CFB15E00220B1
:409D8000FAF777FD022200219C20FAF703FB0CE00220FAF76EFD002211469C20FAF7FAFA03E0FFE70020049000BF00BF9FE406980C287CD2DFE800F00624415E7C9907B6DA
:409DC000D3F3F1F000BF0020009003460246014601902320F9F74EFA022200219D20FAF7D9FA00221146BB20FAF7D4FA00221146AC20FAF7CFFA00210220F7F786FB16E1E8
:409E00000020009003460246032101902320F9F731FA022200219D20FAF7BCFA00221146BB20FAF7B7FA00221146AC20FAF7B2FA00210220F7F769FBF9E0002000900346E6
:409E40000246032101902320F9F714FA002211469D20FAF79FFA00221146BB20FAF79AFA01220021AC20FAF795FA00210220F7F74CFBDCE000200090034602460321019051
:409E80002320F9F7F7F9042200219D20FAF782FA00221146BB20FAF77DFA00221146AC20FAF778FA00210220F7F72FFBBFE0BBE00020009003460246014601902320F9F7C9
:409EC000D9F9002211469D20FAF764FA03220021BB20FAF75FFA00221146AC20FAF75AFA01210220F7F711FBA1E00020009003460246032101902320F9F7BCF90022114600
:409F00009D20FAF747FA00221146BB20FAF742FA00221146AC20FAF73DFA00210220F7F7F4FA84E00020009003460246014601902320F9F79FF9012200219D20FAF72AFAC7
:409F400000221146BB20FAF725FA00221146AC20FAF720FA00210220F7F7D7FA67E00020009003460246014601902320F9F782F9002211469D20FAF70DFA00221146BB209B
:409F8000FAF708FA00221146AC20FAF703FA00210220F7F7BAFA4AE02FE017E0FFE72320FAF767FC012200219D20FAF7F3F900221146BB20FAF7EEF900221146AC20FAF7A9
:409FC000E9F900210220F7F7A0FA30E02320FAF750FC022200219D20FAF7DCF900221146BB20FAF7D7F900221146AC20FAF7D2F900210220F7F789FA19E02320FAF739FC30
:40A00000002211469D20FAF7C5F900221146BB20FAF7C0F900221146AC20FAF7BBF900210220F7F772FA02E00020049000BF00BF2DE406980C287CD2DFE800F00624417BD4
:40A040005E7C0799B6D3EAFE00BF0020009003460246014601902420F9F70CF9022200219E20FAF797F900221146BB20FAF792F900221146AC20FAF78DF900210220F7F7A3
:40A0800044FAF8E00020009003460246032101902420F9F7EFF8022200219E20FAF77AF900221146BB20FAF775F900221146AC20FAF770F900210220F7F727FADBE0002093
:40A0C000009003460246032101902420F9F7D2F8002211469E20FAF75DF900221146BB20FAF758F901220021AC20FAF753F900210220F7F70AFABEE0002000900346024617
:40A10000014601902420F9F7B5F8002211469E20FAF740F903220021BB20FAF73BF900221146AC20FAF736F901210220F7F7EDF9A1E09DE00020009003460246032101904E
:40A140002420F9F797F8002211469E20FAF722F900221146BB20FAF71DF900221146AC20FAF718F900210220F7F7CFF983E00020009003460246014601902420F9F77AF81C
:40A18000012200219E20FAF705F900221146BB20FAF700F900221146AC20FAF7FBF800210220F7F7B2F966E00020009003460246014601902420F9F75DF8002211469E204C
:40A1C000FAF7E8F800221146BB20FAF7E3F800221146AC20FAF7DEF800210220F7F795F949E02420FAF745FB012200219E20FAF7D1F800221146BB20FAF7CCF800221146C7
:40A20000AC20FAF7C7F800210220F7F77EF932E02420FAF72EFB022200219E20FAF7BAF800221146BB20FAF7B5F800221146AC20FAF7B0F8002100E003E00220F7F765F9C2
:40A2400019E02420FAF715FB002211469E20FAF7A1F800221146BB20FAF79CF800221146AC20FAF797F800210220F7F74EF902E00020049000BF00BFA9E406980C286FD215
:40A28000DFE800F006166E6E6E25073443525B6400BF0020009003460246014601904C20F8F7E8FF022200219F20FAF773F85AE00020009003460246032101904C20F8F7C8
:40A2C000D9FF022200219F20FAF764F84BE00020009003460246032101904C20F8F7CAFF002211469F20FAF755F83CE00020009003460246014601904C20F8F7BBFF01220D
:40A3000000219F20FAF746F82DE00020009003460246014601904C20F8F7ACFF002211469F20FAF737F81EE04C20FAF7A2FA012200219F20FAF72EF815E04C20FAF799FA94
:40A34000022200219F20FAF725F80CE04C20FAF790FA002211469F20FAF71CF803E0FFE70020049000BF00BF31E406980C286FD2DFE800F006166E6E6E25073443525B64C7
:40A3800000BF0020009003460246014601905020F8F770FF02220021A020F9F7FBFF5AE00020009003460246032101905020F8F761FF02220021A020F9F7ECFF4BE00020EE
:40A3C000009003460246032101905020F8F752FF00221146A020F9F7DDFF3CE00020009003460246014601905020F8F743FF01220021A020F9F7CEFF2DE000200090034635
:40A400000246014601905020F8F734FF00221146A020F9F7BFFF1EE05020FAF72AFA01220021A020F9F7B6FF15E05020FAF721FA02220021A020F9F7ADFF0CE05020FAF7F8
:40A4400018FA00221146A020F9F7A4FF03E0FFE70020049000BF00BF30E406980C287DD2DFE800F0061B2FABAB4307576B818F9D00BF00200090034602460146019021209F
:40A48000F8F7F8FE02220021A120F9F783FF00221146AC20F9F77EFF92E00020009003460246032101902120F8F7E4FE02220021A120F9F76FFF00221146AC20F9F76AFF11
:40A4C0007EE00020009003460246032101902120F8F7D0FE00221146A120F9F75BFF01220021AC20F9F756FF6AE00020009003460246032101902120F8F7BCFE002211468E
:40A50000A120F9F747FF00221146AC20F9F742FF56E00020009003460246014601902120F8F7A8FE01220021A120F9F733FF00221146AC20F9F72EFF42E0002000900346E5
:40A540000246014601902120F8F794FE00221146A120F9F71FFF0022114600E02DE0AC20F9F718FF2CE02120FAF783F901220021A120F9F70FFF00221146AC20F9F70AFF7D
:40A580001EE02120FAF775F902220021A120F9F701FF00221146AC20F9F7FCFE10E02120FAF767F900221146A120F9F7F3FE00221146AC20F9F7EEFE02E00020049000BFC5
:40A5C00000BF35E506980C287ED2DFE800F0061B2FABAB4307576B818F9D00BF0020009003460246014601904B20F8F743FE02220021A220F9F7CEFE00221146AC20F9F7DF
:40A60000C9FE92E00020009003460246032101904B20F8F72FFE02220021A220F9F7BAFE00221146AC20F9F7B5FE7EE00020009003460246032101904B20F8F71BFE0022E4
:40A640001146A220F9F7A6FE01220021AC20F9F7A1FE6AE00020009003460246032101904B20F8F707FE00221146A220F9F792FE00221146AC20F9F78DFE56E0002000908E
:40A6800003460246014601904B20F8F7F3FD01220021A220F9F77EFE00221146AC20F9F779FE42E00020009003460246014601904B20F8F7DFFD00221146A220F9F76AFEC5
:40A6C00000221146AC2000E02CE0F9F763FE2CE04B20FAF7CEF801220021A220F9F75AFE00221146AC20F9F755FE1EE04B20FAF7C0F802220021A220F9F74CFE0022114608
:40A70000AC20F9F747FE10E04B20FAF7B2F800221146A220F9F73EFE00221146AC20F9F739FE02E00020049000BF00BF80E406980E285AD005DC58B10C2828D00D287DD140
:40A7400044E00F2867D0102879D0112876D19EE00020009003460246012101904620F8F789FD0020009003460246012101900920F8F780FD01210846FBF7EBFB0499084043
:40A78000049000221146DC20F9F704FE9DE00020009003460246012101904620F8F76AFD0020009003460246012101900920F8F761FD01210846FBF7CCFB04990840049065
:40A7C00001220021DC20F9F7E5FD7EE00020009003460246012101904620F8F74BFD01220021DC20F9F7D6FD6FE00020009003460246012101900920F8F73CFD032101207C
:40A80000FBF7A7FB04990840049001220021DC20F9F7C0FD59E003A94620FBF7D8FD0020039903460246CDE9001002214620F8F721FD012000210B460A4601E042E012E08B
:40A84000CDE9001001460920F8F714FD02210120FBF77FFB04990840049001220021DC20F9F798FD31E003A94620FBF7B0FD0020039903460246CDE9001002214620F8F767
:40A88000F9FC01220021DC20F9F784FD1DE003A90920FBF79CFD0020039903460246CDE9001002210920F8F7E5FC03210120FBF750FB04990840049001220021DC20F9F73B
:40A8C00069FD02E00020049000BF00BFD4E406980E285AD005DC58B10C2828D00D287DD144E00F2867D0102879D0112876D19EE00020009003460246012101907A20F8F701
:40A90000B9FC0020009003460246012101900A20F8F7B0FC01210220FBF71BFB04990840049000221146DD20F9F734FD9DE00020009003460246012101907A20F8F79AFCBD
:40A940000020009003460246012101900A20F8F791FC01210220FBF7FCFA04990840049001220021DD20F9F715FD7EE00020009003460246012101907A20F8F77BFC0122E0
:40A980000021DD20F9F706FD6FE00020009003460246012101900A20F8F76CFC03210220FBF7D7FA04990840049001220021DD20F9F7F0FC59E003A97A20FBF708FD00208D
:40A9C000039903460246CDE9001002217A20F8F751FC012000210B460A4601E042E012E0CDE9001001460A20F8F744FC02210846FBF7AFFA04990840049001220021DD2067
:40AA0000F9F7C8FC31E003A97A20FBF7E0FC0020039903460246CDE9001002217A20F8F729FC01220021DD20F9F7B4FC1DE003A90A20FBF7CCFC0020039903460246CDE9E8
:40AA4000001002210A20F8F715FC03210220FBF780FA04990840049001220021DD20F9F799FC02E00020049000BF00BF04E406980D287CD2DFE800F007567F7BA6CD08F9E9
:40AA8000F7F6F5F42F0000BF0020009003460246014601904920F8F7EDFB02220021A320F9F778FC00221146B920F9F773FC00221146AD20F9F76EFC00221146CD20F9F766
:40AAC00069FC00210846F6F720FD00221146ED20F9F760FC7DE10020009003460246014601904920F8F7C6FB02220021A320F9F751FC00221146B920F9F74CFC00221146CE
:40AB0000AD20F9F747FC00221146CD20F9F742FC00210846F6F7F9FC01220021ED20F9F739FC56E10020009003460246032101904920F8F79FFB02220021A320F9F72AFC7D
:40AB400000221146B920F9F725FC00221146AD20F9F720FC00221146CD20F9F71BFC00210846F6F7D2FC00221146ED2000E02DE1F9F710FC2DE100200090034602460321A6
:40AB800001904920F8F776FB00221146A320F9F701FC00221146B920F9F7FCFB01220021AD20F9F7F7FB00221146CD20F9F7F2FB00210846F6F7A9FC00221146ED20F9F72C
:40ABC000E9FB06E10020009003460246014601904920F8F74FFB00221146A320F9F7DAFB03220021B920F9F7D5FB00221146AD20F9F7D0FB00221146CD20F9F7CBFB0121B0
:40AC00000020F6F782FC00221146ED20F9F7C2FBDFE00020009003460246032101904920F8F728FB00221146A320F9F7B3FB00221146B920F9F7AEFB00221146AD20F9F72B
:40AC4000A9FB00221146CD20F9F7A4FB00210846F6F75BFC00221146ED20F9F79BFBB8E093E071E04FE027E0FFE70020009003460246014601904920F8F7FCFA0122002159
:40AC8000A320F9F787FB00221146B920F9F782FB00221146AD20F9F77DFB00221146CD20F9F778FB00210846F6F72FFC00221146ED20F9F76FFB8CE0002000900346024615
:40ACC000014601904920F8F7D5FA00221146A320F9F760FB00221146B920F9F75BFB00221146AD20F9F756FB00221146CD20F9F751FB00210846F6F708FC00221146ED2027
:40AD0000F9F748FB65E04920F9F7B3FD01220021A320F9F73FFB00221146B920F9F73AFB00221146AD20F9F735FB00221146CD20F9F730FB00210846F6F7E7FB002211464C
:40AD4000ED20F9F727FB44E04920F9F792FD02220021A320F9F71EFB00221146B920F9F719FB00221146AD20F9F714FB00221146CD20F9F70FFB00210846F6F7C6FB00225D
:40AD80001146ED20F9F706FB23E04920F9F771FD00221146A320F9F7FDFA00221146B920F9F7F8FA00221146AD20F9F7F3FA00221146CD20F9F7EEFA00210846F6F7A5FBC0
:40ADC00000221146ED20F9F7E5FA02E00020049000BF00BFAAE406980D287CD2DFE800F007567F7BA6CD08F9F7F6F5F42F0000BF0020009003460246014601906F20F8F75E
:40AE000039FA02220021A420F9F7C4FA00221146B920F9F7BFFA00221146AD20F9F7BAFA00221146CE20F9F7B5FA00210846F6F76CFB00221146EE20F9F7ACFA7DE10020DF
:40AE4000009003460246014601906F20F8F712FA02220021A420F9F79DFA00221146B920F9F798FA00221146AD20F9F793FA00221146CE20F9F78EFA00210846F6F745FBAD
:40AE800001220021EE20F9F785FA56E10020009003460246032101906F20F8F7EBF902220021A420F9F776FA00221146B920F9F771FA00221146AD20F9F76CFA0022114617
:40AEC000CE20F9F767FA00210846F6F71EFB00221146EE2000E02DE1F9F75CFA2DE10020009003460246032101906F20F8F7C2F900221146A420F9F74DFA00221146B920E0
:40AF0000F9F748FA01220021AD20F9F743FA00221146CE20F9F73EFA00210846F6F7F5FA00221146EE20F9F735FA06E10020009003460246014601906F20F8F79BF90022ED
:40AF40001146A420F9F726FA03220021B920F9F721FA00221146AD20F9F71CFA00221146CE20F9F717FA01210020F6F7CEFA00221146EE20F9F70EFADFE00020009003469A
:40AF80000246032101906F20F8F774F900221146A420F9F7FFF900221146B920F9F7FAF900221146AD20F9F7F5F900221146CE20F9F7F0F900210846F6F7A7FA0022114675
:40AFC000EE20F9F7E7F9B8E093E071E04FE027E0FFE70020009003460246014601906F20F8F748F901220021A420F9F7D3F900221146B920F9F7CEF900221146AD20F9F720
:40B00000C9F900221146CE20F9F7C4F900210846F6F77BFA00221146EE20F9F7BBF98CE00020009003460246014601906F20F8F721F900221146A420F9F7ACF900221146D6
:40B04000B920F9F7A7F900221146AD20F9F7A2F900221146CE20F9F79DF900210846F6F754FA00221146EE20F9F794F965E06F20F9F7FFFB01220021A420F9F78BF900229F
:40B080001146B920F9F786F900221146AD20F9F781F900221146CE20F9F77CF900210846F6F733FA00221146EE20F9F773F944E06F20F9F7DEFB02220021A420F9F76AF931
:40B0C00000221146B920F9F765F900221146AD20F9F760F900221146CE20F9F75BF900210846F6F712FA00221146EE20F9F752F923E06F20F9F7BDFB00221146A420F9F7E5
:40B1000049F900221146B920F9F744F900221146AD20F9F73FF900221146CE20F9F73AF900210846F6F7F1F900221146EE20F9F731F902E00020049000BF00BF96E4069843
:40B140000D287DD2DFE800F0073AD9D9D953086C87A0B3C6210000BF0020009003460246014601905A20F8F785F802220021A520F9F710F900221146CF20F9F70BF9002201
:40B180001146EF20F9F706F9BAE00020009003460246014601905A20F8F76CF802220021A520F9F7F7F800221146CF20F9F7F2F801220021EF20F9F7EDF8A1E00020009036
:40B1C00003460246032101905A20F8F753F802220021A520F9F7DEF800221146CF20F9F7D9F800221146EF20F9F7D4F888E00020009003460246032101905A20F8F73AF81F
:40B2000000221146A520F9F7C5F800221146CF20F9F7C0F800221146EF20F9F7BBF86FE00020009003460246014601905A20F8F721F801220021A520F9F7ACF8002200E05F
:40B240005BE01146CF20F9F7A5F800221146EF20F9F7A0F854E00020009003460246014601905A20F8F706F800221146A520F9F791F800221146CF20F9F78CF800221146F0
:40B28000EF20F9F787F83BE05A20F9F7F2FA01220021A520F9F77EF800221146CF20F9F779F800221146EF20F9F774F828E05A20F9F7DFFA02220021A520F9F76BF80022B9
:40B2C0001146CF20F9F766F800221146EF20F9F761F815E05A20F9F7CCFA00221146A520F9F758F800221146CF20F9F753F800221146EF20F9F74EF802E00020049000BF90
:40B3000000BF67E506980D287ED2DFE800F0073AD9D9D953086C87A0B3C6210000BF0020009003460246014601905620F7F7A2FF02220021A620F9F72DF800221146D0206E
:40B34000F9F728F800221146F020F9F723F8BAE00020009003460246014601905620F7F789FF02220021A620F9F714F800221146D020F9F70FF801220021F020F9F70AF8DD
:40B38000A1E00020009003460246032101905620F7F770FF02220021A620F8F7FBFF00221146D020F8F7F6FF00221146F020F8F7F1FF88E00020009003460246032101903C
:40B3C0005620F7F757FF00221146A620F8F7E2FF00221146D020F8F7DDFF00221146F020F8F7D8FF6FE00020009003460246014601905620F7F73EFF01220021A620F8F7FF
:40B40000C9FF0022114600E05AE0D020F8F7C2FF00221146F020F8F7BDFF54E00020009003460246014601905620F7F723FF00221146A620F8F7AEFF00221146D020F8F7D7
:40B44000A9FF00221146F020F8F7A4FF3BE05620F9F70FFA01220021A620F8F79BFF00221146D020F8F796FF00221146F020F8F791FF28E05620F9F7FCF902220021A62089
:40B48000F8F788FF00221146D020F8F783FF00221146F020F8F77EFF15E05620F9F7E9F900221146A620F8F775FF00221146D020F8F770FF00221146F020F8F76BFF02E0DD
:40B4C0000020049000BF00BF29E206980D287DD2DFE800F007427C7D7C5F089AB7D4EBFE250000BF0020009003460246014601900320F7F7BFFE00200090034602460121D5
:40B5000001900D20F7F7B6FE02220021A720F8F741FF00221146F120F8F73CFFF8E00020009003460246014601900320F7F7A2FE0020009003460246012101900D20F7F70B
:40B5400099FE02220021A720F8F724FF01220021F120F8F71FFFDBE00020009003460246032101900846F7F785FE0020009003460246012101900D20F7F77CFE0222002176
:40B58000A720F8F707FF00221146F120F8F702FFBEE00020009003460246032101900846F7F768FE0020009003460246012101900D20F7F75FFE00221146A720F8F7EAFE9C
:40B5C00000221146F120F8F7E5FEA1E09DE00020009003460246032101900846F7F74AFE0020009003460246012101900D20F7F741FE04220021A720F8F7CCFE00221146E9
:40B60000F120F8F7C7FE83E00020009003460246014601900320F7F72DFE0020009003460246012101900D20F7F724FE01220021A720F8F7AFFE00221146F120F8F7AAFE94
:40B6400066E00020009003460246014601900320F7F710FE0020009003460246012101900D20F7F707FE00221146A720F8F792FE00221146F120F8F78DFE49E00320F9F739
:40B68000F8F80020009003460246012101900D20F7F7F0FD01220021A720F8F77BFE00221146F120F8F776FE32E00320F9F7E1F80020009003460246012101900D20F7F731
:40B6C000D9FD02220021A720F8F764FE002200E004E01146F120F8F75DFE19E00320F9F7C8F80020009003460246012101900D20F7F7C0FD00221146A720F8F74BFE00224D
:40B700001146F120F8F746FE02E00020049000BF00BFE9E306980D287DD2DFE800F00742FCFCFC5F087D9AB7CEE5250000BF0020009003460246014601905520F7F79AFD99
:40B740000020009003460246012101901D20F7F791FD02220021A820F8F71CFE00221146F220F8F717FED9E00020009003460246014601905520F7F77DFD002000900346CF
:40B780000246012101901D20F7F774FD02220021A820F8F7FFFD01220021F220F8F7FAFDBCE00020009003460246032101905520F7F760FD00200090034602460121019078
:40B7C0001D20F7F757FD02220021A820F8F7E2FD00221146F220F8F7DDFD9FE00020009003460246032101905520F7F743FD0020009003460246012101901D20F7F73AFD2D
:40B8000000221146A820F8F7C5FD00221146F220F8F7C0FD82E07EE00020009003460246014601905520F7F725FD0020009003460246012101901D20F7F71CFD0122002105
:40B84000A820F8F7A7FD00221146F220F8F7A2FD64E00020009003460246014601905520F7F708FD0020009003460246012101901D20F7F7FFFC00221146A820F8F78AFDBE
:40B8800000221146F220F8F785FD47E05520F8F7F0FF0020009003460246012101901D20F7F7E8FC01220021A820F8F773FD00221146F220F8F76EFD30E05520F8F7D9FF73
:40B8C0000020009003460246012101901D20F7F7D1FC02220021A820F8F75CFD00221146F220F8F757FD19E05520F8F7C2FF0020009003460246012101901D20F7F7BAFC46
:40B9000000221146A820F8F745FD00221146F220F8F740FD02E00020049000BF00BFE3E206980D287DD2DFE800F00742FCFCFC5F087D9AB7CEE5250000BF0020009003462A
:40B940000246014601905920F7F794FC0020009003460246012101904D20F7F78BFC02220021A920F8F716FD00221146F320F8F711FDD9E00020009003460246014601906F
:40B980005920F7F777FC0020009003460246012101904D20F7F76EFC02220021A920F8F7F9FC01220021F320F8F7F4FCBCE00020009003460246032101905920F7F75AFC7D
:40B9C0000020009003460246012101904D20F7F751FC02220021A920F8F7DCFC00221146F320F8F7D7FC9FE00020009003460246032101905920F7F73DFC0020009003467A
:40BA00000246012101904D20F7F734FC00221146A920F8F7BFFC00221146F320F8F7BAFC82E07EE00020009003460246014601905920F7F71FFC00200090034602460121A5
:40BA400001904D20F7F716FC01220021A920F8F7A1FC00221146F320F8F79CFC64E00020009003460246014601905920F7F702FC0020009003460246012101904D20F7F70B
:40BA8000F9FB00221146A920F8F784FC00221146F320F8F77FFC47E05920F8F7EAFE0020009003460246012101904D20F7F7E2FB01220021A920F8F76DFC00221146F32057
:40BAC000F8F768FC30E05920F8F7D3FE0020009003460246012101904D20F7F7CBFB02220021A920F8F756FC00221146F320F8F751FC19E05920F8F7BCFE0020009003466A
:40BB00000246012101904D20F7F7B4FB00221146A920F8F73FFC00221146F320F8F73AFC02E00020049000BF00BFDDE106980D287DD2DFE800F00742FCFCFC5F087D9AB7C6
:40BB4000CEE5250000BF0020009003460246014601905420F7F78EFB0020009003460246012101902020F7F785FB02220021AA20F8F710FC00221146F420F8F70BFCD9E042
:40BB80000020009003460246014601905420F7F771FB0020009003460246012101902020F7F768FB02220021AA20F8F7F3FB01220021F420F8F7EEFBBCE000200090034668
:40BBC0000246032101905420F7F754FB0020009003460246012101902020F7F74BFB02220021AA20F8F7D6FB00221146F420F8F7D1FB9FE0002000900346024603210190A3
:40BC00005420F7F737FB0020009003460246012101902020F7F72EFB00221146AA20F8F7B9FB00221146F420F8F7B4FB82E07EE00020009003460246014601905420F7F7D9
:40BC400019FB0020009003460246012101902020F7F710FB01220021AA20F8F79BFB00221146F420F8F796FB64E00020009003460246014601905420F7F7FCFA002000907E
:40BC800003460246012101902020F7F7F3FA00221146AA20F8F77EFB00221146F420F8F779FB47E05420F8F7E4FD0020009003460246012101902020F7F7DCFA01220021E3
:40BCC000AA20F8F767FB00221146F420F8F762FB30E05420F8F7CDFD0020009003460246012101902020F7F7C5FA02220021AA20F8F750FB00221146F420F8F74BFB19E02E
:40BD00005420F8F7B6FD0020009003460246012101902020F7F7AEFA00221146AA20F8F739FB00221146F420F8F734FB02E00020049000BF00BFD7E006980E285AD005DC68
:40BD400058B10C2828D00D287DD144E00F2867D0102879D0112876D19EE00020009003460246012101904720F7F784FA0020009003460246012101900920F7F77BFA012191
:40BD80000846FAF7E6F804990840049000221146DB20F8F7FFFA9DE00020009003460246012101904720F7F765FA0020009003460246012101900920F7F75CFA012108469B
:40BDC000FAF7C7F804990840049001220021DB20F8F7E0FA7EE00020009003460246012101904720F7F746FA01220021DB20F8F7D1FA6FE0002000900346024601210190EF
:40BE00000920F7F737FA03210120FAF7A2F804990840049001220021DB20F8F7BBFA59E003A94720FAF7D3FA0020039903460246CDE9001002214720F7F71CFA01200021A1
:40BE40000B460A4601E042E012E0CDE9001001460920F7F70FFA02210120FAF77AF804990840049001220021DB20F8F793FA31E003A94720FAF7ABFA00200399034602461D
:40BE8000CDE9001002214720F7F7F4F901220021DB20F8F77FFA1DE003A90920FAF797FA0020039903460246CDE9001002210920F7F7E0F903210120FAF74BF804990840D8
:40BEC000049001220021DB20F8F764FA02E00020049000BF00BF07E000BF00BF0020049002E00020049000BF00BF049801282BD10698122827D2DFE800F0090C0D0E0F1049
:40BF000011121314151617180A191A0B00BF00BF19E000BF00BF00BF00BF00BF00BF00BF00BF00BF00BF00BF00BF00BF00BF0598F9F7DAFF10B10020049003E001210598AF
:40BF4000F9F7A6FF00BF00BF049807B000BD10B5F7F735F9A8B1F8F7B2FC6AF076FF002404E0E0B20021FAF74DFA641C562CF8D3F84800210160416001818172F6480180A1
:40BF8000817010BD01460020A1F117023A2A5ED2DFE802F01D1F21232527292B5D5D5D5D5D5D5D5D5D5D5D5D5D5D5D2D2F31333537393B3D3F4143455D5D5D5D5D5D5D5D04
:40BFC0005D47494B4D4F515D5D535557595B29203EE02A203CE0D2203AE0D32038E0D42036E0D52034E0882032E0832030E07B202EE07C202CE040202AE03F2028E01720F2
:40C0000026E0182024E0812022E07D2020E027201EE028201CE058201AE0572018E0772016E0462014E07A2012E0CD2010E0CE200EE0CF200CE0D0200AE00D2008E01D20E1
:40C0400006E04D2004E0202002E0472000E000BF00BF70472DE9F04105460E4600272846FFF790FF04462CB131462046F7F7A9F800B901273846BDE8F081FCB50646304670
:40C08000FFF780FF07466A4601A9FAF738F805460024002D51D0019800284ED0B5EEC00AF1EE10FA04D2DFEDAD0AB0EE600A0AE0DFEDAB0AB4EEE00AF1EE10FA03DBDFED66
:40C0C000A80AB0EE600ADFEDA60AB4EE600AF1EE10FA03D10198C06A441C0FE00198C06A00EE900AF8EE600A9FED9E1A20EE011A60EE810AFCEEE00A10EE904AB4F5803F3A
:40C1000001D34FF6FF7401259DF8000030B1012807D0022808D003280CD108E0019844630AE00198846307E00198C46304E00198046401E0002500BF00E000252846FCBDBE
:40C14000FCB506463046FFF71DFF07466A4601A9F9F7D5FF0546EDB10198D8B1B5EEC00AF1EE10FA0FDDDFED800A80EE801AFCEEC10A10EE904A4FF6FE70844200D90446FB
:40C180000198C46203E04FF6FE700199C8620020019948622846FCBD7CB5044600252046FFF7F0FE06466A4601A9F9F7A8FF002855D00198002852D06C490198884201D19A
:40C1C00001254CE00198B0F1804F01D1022546E067490198884201D1032540E065490198884201D104253AE063490198884201D1052534E061490198884201D106252EE03B
:40C200005F490198884201D1072528E05D490198884201D1082522E05B490198884201D109251CE059490198884201D10A2516E057490198884201D10B2510E055490198B8
:40C24000884201D10C250AE053490198884201D10D2504E051490198884200D10E2528467CBD01460020352934D014DC30292CD008DC172922D0182921D02E2921D02F2982
:40C2800037D11FE031291FD0322920D033291FD034292ED11FE03A2925D008DC36291CD037291BD038291CD0392922D118E044291CD0452918D050291BD118E000BF4F2097
:40C2C00018E000BF872015E000BF5C2012E000BF86200FE000BF3B200CE000BF0C2009E000BF0B2006E000BF0A2003E000BF092000E000BF00BF70472DE9F04105460E4611
:40C3000000272846FFF7ADFF04462CB131462046F6F757FF00B901273846BDE8F081FCB506463046FFF79DFF07466A4601A9F9F7E6FE05460024002D78D00198002875D0A0
:40C34000B5EEC00AF1EE10FA2AD2DFED040AB0EE600A30E0D41C0020AC000010000000000000C8420AD7233C00247449000001400004004000080040000C00400010004019
:40C38000001400400004014000400140004401400048014000180040001C0040002000405FED110AB4EEE00AF1EE10FA03DB5FED140AB0EE600A5FED160AB4EE600AF1EEBE
:40C3C00010FA03D10198C06A441C0FE00198C06A00EE900AF8EE600A1FED1E1A20EE011A60EE810AFCEEE00A10EE904AB4F5803F01D34FF6FF7401259DF8000030B1012807
:40C4000007D0022808D003280DD109E0019844630BE00198846308E00198C46305E005E00198046401E0002500BF00E000252846FCBDFCB506463046FFF713FF07466A46AA
:40C4400001A9F9F75CFE0546EDB10198D8B1B5EEC00AF1EE10FA0FDD5FED3D0A80EE801AFCEEC10A10EE904A4FF6FE70844200D904460198C46203E04FF6FE700199C8629E
:40C480000020019948622846FCBD7CB5044600252046FFF7E6FE06466A4601A9F9F72FFE002855D00198002852D0FB490198884201D101254CE00198B0F1804F01D1022551
:40C4C00046E0F6490198884201D1032540E0F4490198884201D104253AE0F2490198884201D1052534E0F0490198884201D106252EE0EE490198884201D1072528E0EC497B
:40C500000198884201D1082522E0EA490198884201D109251CE0E8490198884201D10A2516E0E6490198884201D10B2510E0E4490198884201D10C250AE0E24901988842EB
:40C5400001D10D2504E0E0490198884200D10E2528467CBD014600203C2953D024DC242940D010DC132935D006DC0A292CD00B292CD00C2964D12BE014292DD015292DD0F8
:40C5800023295DD12CE0312934D006DC29292BD02A292BD0302953D12AE034292CD035292CD03B294CD12BE0A1F13D02132A47D2DFE802F02A2C2E30323446464636383AE0
:40C5C0003C46463E4042440022203AE0702038E03E2036E0672034E06B2032E0252030E02D202EE030202CE02F202AE02E2028E03A2026E06C2024E06E2022E0682020E0FC
:40C6000001201EE002201CE023201AE0242018E04C2016E0502014E0212012E04B2010E049200EE06F200CE05A200AE0562008E0032006E0552004E0592002E0542000E04B
:40C6400000BF00BF704770B504464FF0FF353D2C1CD008DC0A2C14D0132C1DD0142C1CD0152C1FD10CE03E2C11D0462C02D0472C18D100E000BF0020F4F737FF054612E0D3
:40C6800000BF0120F4F731FF05460CE000BF0220F4F72BFF054606E000BF0320F4F725FF054600E000BF00BF284670BD70B504464FF0FF35562C72D2DFE804F072737475BB
:40C6C000767778797A7B7C7D7E7F8081828384858687888997A5EDECEBEAE9E8E7E6E5E4E3E2E1E0DFDEDDDCDBDAD9D8D7D6D5D4D3D2D1D0CFCECDCCCBCAC9C8C7C6C5C483
:40C70000C3C2C1C0BFBEBDBCBBBAB9B8B72B394755636E4890ED1B0AB8EE400ADFED6C0A20EE200ABCEEC00A10EE105A84E3674890ED0C0AB8EE400ADFED650A20EE200A53
:40C74000BCEEC00A10EE105A76E3604890ED1C0AB8EE400ADFED5E0A20EE200ABCEEC00A10EE105A68E3594890ED2B0AB8EE400ADFED570A20EE200ABCEEC00A10EE105A32
:40C780005AE3524890ED0B0AB8EE400ADFED500A20EE200ABCEEC00A10EE105A4CE34AE300BF00BF00BF00BF00BF00BF00BF00BF00BF00BF00BF00BF00BF00BF00BF00BF9A
:40C7C00000BF00BF00BF00BF00BF00BF34E33F4890ED2A0AB8EE400ADFED3E0A20EE200ABCEEC00A10EE105A26E3384890ED2A0AB8EE400ADFED370A20EE200ABCEEC00A75
:40C8000010EE105A18E3F6F74FF9012866D12F4890ED3A0AB8EE400ADFED2F0A20EE200ABCEEC00A10EE105A65E0EBE2CAE2A9E288E267E2FEE2FCE244E21EE2FDE1DCE144
:40C84000CDE1BEE1F4E2F2E2F0E2EEE2ECE2EAE2E8E2E6E2E4E2A6E197E188E179E16AE15BE14CE13DE12EE11FE110E101E1F2E0F0E0EEE0ECE0EAE0E8E0E6E0E4E0E2E09D
:40C88000E0E0DEE0DCE0DAE0D8E0D6E0D4E0B3E092E071E050E02FE0000001400004004000080040000C00400010004000140040000401400040014000440140004801403C
:40C8C00000180040001C004000200040B416002000804944291C15459AA94145F74890ED3A0AB8EE400ADFEDF60A20EE200ABCEEC00A10EE105A9FE2F6F7D6F801280DD1B2
:40C90000EE4890ED3B0AB8EE400A5FED0D0A20EE200ABCEEC00A10EE105A0CE0E74890ED3B0AB8EE400ADFEDE60A20EE200ABCEEC00A10EE105A7FE2F6F7B6F801280DD1F8
:40C94000DE4890ED3C0AB8EE400A5FED1D0A20EE200ABCEEC00A10EE105A0CE0D74890ED3C0AB8EE400ADFEDD60A20EE200ABCEEC00A10EE105A5FE2F6F796F801280DD116
:40C98000CE4890ED3D0AB8EE400A5FED2D0A20EE200ABCEEC00A10EE105A0CE0C74890ED3D0AB8EE400ADFEDC60A20EE200ABCEEC00A10EE105A3FE2F6F776F801280DD134
:40C9C000BE4890ED380AB8EE400A5FED3D0A20EE200ABCEEC00A10EE105A0CE0B74890ED380AB8EE400ADFEDB60A20EE200ABCEEC00A10EE105A1FE2F6F756F801280DD15E
:40CA0000AE4890ED390AB8EE400A5FED4D0A20EE200ABCEEC00A10EE105A0CE0A74890ED390AB8EE400ADFEDA60A20EE200ABCEEC00A10EE105AFFE100BF00BF00BF00BFA2
:40CA400000BF00BF00BF00BF00BF00BF00BF00BF00BF00BFF0E1994890ED290AB8EE400A5FED640A20EE200ABCEEC00A10EE105AE2E1924890ED290AB8EE400A5FED6B0A22
:40CA800020EE200ABCEEC00A10EE105AD4E18B4890ED1A0AB8EE400A5FED720A20EE200ABCEEC00A10EE105AC6E1844890ED1A0AB8EE400A5FED790A20EE200ABCEEC00AEE
:40CAC00010EE105AB8E17D4890ED190AB8EE400A5FED800A20EE200ABCEEC00A10EE105AAAE1764890ED190AB8EE400A5FED870A20EE200ABCEEC00A10EE105A9CE16F48F8
:40CB000090ED0A0AB8EE400A5FED8E0A20EE200ABCEEC00A10EE105A8EE1684890ED0A0AB8EE400A5FED950A20EE200ABCEEC00A10EE105A80E1614890ED090AB8EE400A53
:40CB40005FED9C0A20EE200ABCEEC00A10EE105A72E15A4890ED090AB8EE400A5FEDA30A20EE200ABCEEC00A10EE105A64E1534890ED280AB8EE400A5FEDAA0A20EE200A76
:40CB8000BCEEC00A10EE105A56E14C4890ED280AB8EE400A5FEDB10A20EE200ABCEEC00A10EE105A48E1454890ED180AB8EE400A5FEDB80A20EE200ABCEEC00A10EE105AAD
:40CBC0003AE13E4890ED080AB8EE400A5FEDBF0A20EE200ABCEEC00A10EE105A2CE1374890ED180AB8EE400A5FEDC60A20EE200ABCEEC00A10EE105A1EE1F5F755FF012839
:40CC00000DD12E4890ED300AB8EE400A5FEDCE0A20EE200ABCEEC00A10EE105A0CE0274890ED300AB8EE400ADFED250A20EE200ABCEEC00A10EE105AFEE0F5F735FF012889
:40CC40000DD11E4890ED310AB8EE400A5FEDDE0A20EE200ABCEEC00A10EE105A0CE0174890ED310AB8EE400ADFED150A20EE200ABCEEC00A10EE105ADEE0F5F715FF0128A7
:40CC80000DD10E4890ED320AB8EE400A5FEDEE0A20EE200ABCEEC00A10EE105A0CE0074890ED320AB8EE400ADFED050A20EE200ABCEEC00A10EE105ABEE00000B4160020E4
:40CCC0001F058944F5F7F0FE01280DD1DB4890ED330AB8EE400ADFEDDA0A20EE200ABCEEC00A10EE105A0CE0D44890ED330AB8EE400A5FED0D0A20EE200ABCEEC00A10EE12
:40CD0000105A99E0F5F7D0FE01280DD1CB4890ED340AB8EE400ADFEDCA0A20EE200ABCEEC00A10EE105A0CE0C44890ED340AB8EE400A5FED1D0A20EE200ABCEEC00A10EE1D
:40CD4000105A79E0F5F7B0FE01280DD1BB4890ED350AB8EE400ADFEDBA0A20EE200ABCEEC00A10EE105A0CE0B44890ED350AB8EE400A5FED2D0A20EE200ABCEEC00A10EE3B
:40CD8000105A59E0F5F790FE01280DD1AB4890ED360AB8EE400ADFEDAA0A20EE200ABCEEC00A10EE105A0CE0A44890ED360AB8EE400A5FED3D0A20EE200ABCEEC00A10EE59
:40CDC000105A39E0F5F770FE01280DD19B4890ED370AB8EE400ADFED9A0A20EE200ABCEEC00A10EE105A0CE0944890ED370AB8EE400A5FED4D0A20EE200ABCEEC00A10EE77
:40CE0000105A19E08D4890ED080AB8EE400ADFED8D0A20EE200ABCEEC00A10EE105A0BE000BF00BF00BF00BF00BF00BF00BF00BF00BF00BF00E000BF00BF284670BD014623
:40CE40004FF0FF30562972D2DFE801F0F6F5F4F3F2F1F0EFEEED72808EECEBEAE9E8E79CE6E5E4E3E2E1E0DFDEDDDCDBDAD9D8D7D6D5D4D3D2D1D0CFCECDCCCBCAC9C8C7F5
:40CE8000C6C5C4C3C2C1C0BFBEBDBCBBBAB9B8B7B6B5B4B3B2B1B0AFAEADACABAA2B39475563664A92ED0D0AB8EE400ADFED660A20EE200ABCEEC00A10EE100AD6E25F4AA0
:40CEC00092ED1E0AB8EE400ADFED600A20EE200ABCEEC00A10EE100AC8E2584A92ED1D0AB8EE400ADFED590A20EE200ABCEEC00A10EE100ABAE2514A92ED2D0AB8EE400AEF
:40CF0000DFED520A20EE200ABCEEC00A10EE100AACE24A4A92ED0F0AB8EE400ADFED4B0A20EE200ABCEEC00A10EE100A9EE29CE2424A92ED410AB8EE400ADFED450A20EE09
:40CF4000200ABCEEC00A10EE100A8FE23B4A92ED130AB8EE400ADFED3E0A20EE200ABCEEC00A10EE100A81E2344A92ED230AB8EE400ADFED370A20EE200ABCEEC00A10EE6D
:40CF8000100A73E22D4A92ED000AB8EE400ADFED300A20EE200ABCEEC00A10EE100A65E262E241E232E223E214E25CE25AE203E2F4E1E5E1D6E154E252E250E2C4E1B5E103
:40CFC000A6E197E188E179E16AE15BE146E244E242E240E23EE247E138E13AE238E227E118E134E232E214E112E110E1F9E0EAE00CE10AE108E106E1D7E0C8E002E100E14B
:40D00000FEE0FCE0B5E0A6E097E088E079E06AE05BE04CE04AE02BE01CE046E044E042E040E03EE03CE03AE038E036E034E032E030E02EE02CE02AE028E00000B4160020A7
:40D040009AA94145291C1545527845465C8F5145C0A99A44FB4A92ED200AB8EE400A5FED040A20EE200ABCEEC00A10EE100AFDE1F44A92ED440AB8EE400A5FED0B0A20EEE7
:40D08000200ABCEEC00A10EE100AEFE100BF00BF00BF00BF00BF00BF00BF00BF00BF00BF00BF00BF00BF00BF00BF00BFDEE1E54A92ED070AB8EE400A5FED1B0A20EE200AE3
:40D0C000BCEEC00A10EE100AD0E1DE4A92ED160AB8EE400A5FED220A20EE200ABCEEC00A10EE100AC2E1D74A92ED170AB8EE400A5FED290A20EE200ABCEEC00A10EE100A69
:40D10000B4E1D04A92ED1F0AB8EE400A5FED300A20EE200ABCEEC00A10EE100AA6E1C94A92ED250AB8EE400A5FED370A20EE200ABCEEC00A10EE100A98E1C24A92ED260AA1
:40D14000B8EE400A5FED3E0A20EE200ABCEEC00A10EE100A8AE1BB4A92ED270AB8EE400A5FED450A20EE200ABCEEC00A10EE100A7CE1B44A92ED2C0AB8EE400A5FED4C0A56
:40D1800020EE200ABCEEC00A10EE100A6EE1AD4A92ED040AB8EE400A5FED530A20EE200ABCEEC00A10EE100A60E1A64A92ED050AB8EE400A5FED5A0A20EE200ABCEEC00A70
:40D1C00010EE100A52E19F4A92ED240AB8EE400A5FED610A20EE200ABCEEC00A10EE100A44E1984A92ED140AB8EE400A5FED680A20EE200ABCEEC00A10EE100A36E100BFF7
:40D2000000BF00BF00BF00BF00BF00BF00BF00BF00BF2BE18B4A92ED120AB8EE400ADFED8A0A20EE200ABCEEC00A10EE100A1DE1844A92ED010AB8EE400A5FED7B0A20EE82
:40D24000200ABCEEC00A10EE100A0FE17D4A92ED020AB8EE400ADFED7C0A20EE200ABCEEC00A10EE100A01E1764A92ED100AB8EE400A5FED890A20EE200ABCEEC00A10EEFC
:40D28000100AF3E06F4A92ED450AB8EE400A5FED900A20EE200ABCEEC00A10EE100AE5E0684A92ED460AB8EE400A5FED970A20EE200ABCEEC00A10EE100AD7E0614A92ED98
:40D2C000420AB8EE400A5FED9E0A20EE200ABCEEC00A10EE100AC9E05A4A92ED430AB8EE400A5FEDA50A20EE200ABCEEC00A10EE100ABBE0534A92ED030AB8EE400A5FED72
:40D30000AC0A20EE200ABCEEC00A10EE100AADE04C4A92ED220AB8EE400A5FEDB30A20EE200ABCEEC00A10EE100A9FE0454A92ED400AB8EE400A5FEDBA0A20EE200ABCEE2F
:40D34000C00A10EE100A91E03E4A92ED150AB8EE400A5FEDC10A20EE200ABCEEC00A10EE100A83E0374A92ED110AB8EE400A5FEDC80A20EE200ABCEEC00A10EE100A75E0C4
:40D38000304A92ED210AB8EE400A5FEDCF0A20EE200ABCEEC00A10EE100A67E0294A92ED490AB8EE400A5FEDD60A20EE200ABCEEC00A10EE100A59E0224A92ED4C0AB8EEE4
:40D3C000400A5FEDDD0A20EE200ABCEEC00A10EE100A4BE01B4A92ED470AB8EE400A5FEDE40A20EE200ABCEEC00A10EE100A3DE0144A92ED4B0AB8EE400A5FEDEB0A20EE10
:40D40000200ABCEEC00A10EE100A2FE00D4A92ED480AB8EE400A5FEDF20A20EE200ABCEEC00A10EE100A21E0064A92ED4A0AB8EE400A5FEDF90A20EE200ABCEEC00A10EEF6
:40D44000100A13E0B416002018421B4500BF00BF00BF00BF00BF00BF00BF00BF00BF00BF00BF00BF00BF00BF00E000BF00BF704770B5054600262846FFF76CF804461CB1FF
:40D480002046F6F7E2FE0646304670BD0246002031B101290DD0022916D0032928D11CE09369DBB2602B01D1012300E00023184620E0936903F47F43B3F5C04F01D10123FA
:40D4C00000E00023184615E0D369DBB2602B01D1012300E0002318460CE0D36903F47F43B3F5C04F01D1012300E00023184601E0002000BF00BF70477CB5054600262846F6
:40D50000FEF740FD0446002C3DD06A4601A92046F8F7F5FD78B39DF800100198FFF7B6FF48B39DF8000030B101280CD0022812D0032821D117E00198406B08B1012000E0ED
:40D54000002006461AE00198806B08B1012000E00020064612E00198C06B08B1012000E0002006460AE00198006C08B1012000E00020064602E002E0002600BF03E02046B8
:40D58000F6F7AEFE064630467CBD00000020002106E0F94A52F821200AB1012002E0491C0229F6D300BF704710B5002447F0CEFCF2490968081AB0F5806F00D801242046A6
:40D5C00010BD10B5002447F0C1FCEC490968081AB0F5483F08D247F0B9FCE8490968081AB0F5806F00D90124204610BD10B50024E34803F0A0FA0446204610BD10B5002437
:40D60000DF4802F0FFFB0446204610BD38B50446002500200090DA4802F00AFD40B36A460221D74801F0ABFA10B300984AF0ACFDF0B1012C0ED100984AF0B9FDDFEDD10A9E
:40D64000B4EEE00AF1EE10FA01DD012000E0002005460DE000984AF0AAFDDFEDCB0AB4EEE00AF1EE10FA01D2012000E000200546284638BD38B50446002500200090C048B9
:40D6800002F0BDFC58B16A462146BD4801F077FA28B100984AF078FD08B9012000E000200546284638BD70B505460024282D16D2DFE805F014171C21262B3035393D4145E1
:40D6C000636D8B95B5C2F8F6F5F4F3F2F1F0EFEEEDECEBEAE9E8E7E6E5E4E3E200BF00248DE20020FFF7C6FF044688E20120FFF7C1FF044683E20220FFF7BCFF04467EE28B
:40D700000320FFF7B7FF044679E20120FFF77EFF044674E20020FFF779FF04466FE2FFF76DFF04466BE2FFF761FF044667E2FFF748FF044663E2FFF737FF04465FE23CF087
:40D7400063FEB0F57A7F09D23CF05EFE8F490968C1F57A71884201D3012000E000200446012C09D18948006830B13CF04DFEC0F57A70401E8549086041E23CF045FEB0F552
:40D780007A7F01D3012000E00020044637E23DF037FBB0F57A7F09D23DF032FB7C490968C1F57A71884201D3012000E000200446012C09D17648006830B13DF021FBC0F5FA
:40D7C0007A70401E7249086019E23DF019FBB0F57A7F01D3012000E0002004460FE26D48F1F7BDFD68B93EF032FA192809D23EF02EFA69490968C1F11901884201D30120C2
:40D8000000E000200446012C08D16348006828B13EF01DFAC0F118005F490860EFE15D48F1F79DFD28B93EF012FA192801D3012000E000200446E2E15648F1F790FD68B905
:40D840003FF05CF8322809D23FF058F853490968C1F13201884201D3012000E000200446012C08D14D48006828B13FF047F8C0F131004A490860C2E1B6E1AAE19EE192E198
:40D8800086E17AE16EE160E13FE131E110E104E1E2E0D7E0B8E0AAE089E062E03FE030E00DE0FFE73B48F1F75AFD28B93FF026F8322801D3012000E0002004469FE1354840
:40D8C000F1F74DFD70B93FF0C2FDB0F5FA7F09D23FF0BDFD32490968C1F5FA71884201D3012000E000200446012C09D12C48006830B13FF0ACFDC0F5FA70401E28490860F5
:40D900007DE12448F1F72BFD30B93FF0A0FDB0F5FA7F01D3012000E0002004466FE11D48F1F71DFD70B940F0CFFCB0F57A7F09D240F0CAFC1B490968C1F57A71884201D39D
:40D94000012000E000200446012C09D11548006830B140F0B9FCC0F57A70401E114908604DE10C48F1F7FBFCF0B940F0ADFCB0F57A7F19D3012018E0C00000100CA80F08CA
:40D98000E0390010481C264A481C26CACC000010D00000107C220010D4000010D8000010DC000010E00000100020044627E1FE48F1F7D5FC68B941F0C0F9322809D241F022
:40D9C000BCF9FA490968C1F13201884201D3012000E000200446012C08D1F448006828B141F0ABF9C0F13100F049086007E1EE48F1F7B5FC28B941F0A0F9322801D3012044
:40DA000000E000200446FAE042F052F8B0F57A7F09D242F04DF8E6490968C1F57A71884201D3012000E000200446012C09D1E048006830B142F03CF8C0F57A70401EDC490C
:40DA40000860DCE042F034F8B0F57A7F01D3012000E000200446D2E043F0CBF942F2107188420AD243F0C5F9D249096842F21072511A884201D3012000E000200446012C6F
:40DA80000AD1CC48006838B143F0B3F942F21071081A401EC7490860B1E043F0AAF942F21071884201D3012000E000200446A6E0BD48F1F754FC68B949F0DEF9322809D24C
:40DAC00049F0DAF9BC490968C1F13201884201D3012000E000200446012C08D1B648006828B149F0C9F9C0F13100B349086086E0AD48F1F734FC28B949F0BEF9322801D3BE
:40DB0000012000E00020044679E0A748F1F727FC68B949F059FF642809D249F055FFA7490968C1F16401884201D3012000E000200446012C08D1A148006828B149F044FF54
:40DB4000C0F163009D49086059E09748F1F707FC28B949F039FF642801D3012000E0002004464CE0964802F057F8044624B100221146934802F054F841E0914802F05AF8E9
:40DB8000044624B1002211468D4802F057F836E08B4802F05DF8044624B100221146884802F05AF82BE0864802F060F8044624B100221146824802F05DF820E0804802F055
:40DBC00063F8044624B1002211467D4801F02EFA15E07B4802F05CF8044624B100221146774801F019FA0AE0754802F055F8044624B100221146724802F052F800BF00BF09
:40DC0000204670BD10B528216E4874F0C2F9A0216D4874F0BEF9A0216C4874F0BAF96C480021016041606B48016041606A480160416010BD0EB501260321684880F87D1081
:40DC4000FFF7E0FF00BF2821002076F047FD8DE807000098082841D1019800F4804060B100215E4880F87D1000205C49886776F065FD804676F07AFD30E0019800F00100C4
:40DC800060B3002427E06009524951F8200004F01F0201219140084008B1012000E0002001280BD100BF01214D480155024611194C4AA0180122EDF713FC0BE000BF00211D
:40DCC0004748015502461119464AA0180122EDF707FC00BF641C282CD5D301264248007801285FD1002496E104EB84013F4A02EBC101C879FFF7D7FC05466009344951F8F3
:40DD0000200004F01F0201219140084008B1012000E00020A8426BD0002D6AD1002760092C4951F8200004F01F0201219140084008B1012000E0002078B96009264951F822
:40DD4000200004F01F0201219140084008B1012000E0002008B9012779E004EB8400234901EBC00090F8240000F0010010B1012701266CE004EB84001C4901EBC00090F887
:40DD8000240000F0080070B104EB84020B4603EBC202116A0D4A52F824004CF069FA48BB084828E03AE12CE07C220010E4000010E8000010EC000010F0000010F4000010B3
:40DDC000E03900102838001050380010F0380010B0000010B8000010C0000010300A00204808002000500068C800001070C7090859E059E002E0005D012802D101270126C4
:40DE000025E004EB8400F74901EBC00090F8240000F0040030B1F448005D012802D10127012614E004EB8400EE4901EBC00090F8240000F0020050B104EB840001EBC00011
:40DE4000407A20B9FFF7A2FB08B101270126012F40D10020E44908556009E44951F8200004F01F020121914088436109DF4A42F821006009DE4951F8200004F01F02012199
:40DE8000914088436109DA4A42F821006009D94951F8200004F01F020121914088436109D44A42F8210015E00020CF4908556009CE4951F8200004F01F020121914008436D
:40DEC0006109CA4A42F82100CB4800688047CB4941F82400012D7CD16009C54951F8200004F01F0201219140084008B1012000E00020C8BB04EB8400BA4901EBC0004069C3
:40DF000058B104EB84020B4603EBC2025169BB4A52F824004CF0ACF930B36009B44951F8200004F01F020121914008436109B04A42F821000126B04800688047B04941F80E
:40DF40002400B048005D7E280EDA00BFAD48005D401CC1B2AB48015502461119AA4AA0180122EDF7BDFA00BF04EB84009D4901EBC000407A012830D160099E4951F8200034
:40DF800004F01F0201219140084008B1012000E0002010BB04EB8400924901EBC000806958B104EB84020B4603EBC2029169934A52F824004CF05CF978B160098D4951F881
:40DFC000200004F01F020121914008436109894A00E01FE042F82100012604EB8400814901EBC000C069A8B104EB84020B4603EBC202D169824A52F824004CF039F948B152
:40E000007D48006880477E4941F824000020764908550126641C282CFFF466AE012E7FF412AE00260320EEF75AF878480CF03BF909E601464FF6FF70282905D201EB810237
:40E04000684B03EBC2029089704701464FF6FF70282905D201EB8102624B03EBC202108A704701460020282905D201EB81025D4B03EBC202107A704701460020282901D205
:40E08000604A505C70470146FF20282905D201EB8102544B03EBC2021079704701460020282905D201EB81024E4B03EBC2025079704701460020282905D201EB8102494B6A
:40E0C00003EBC2029079704701466FF00040282904D201EB8102434B53F83200704701464FF6FF70282905D201EB81023D4B03EBC202D089704727201DE03B49095CC9B9E5
:40E1000000EB8001374A02EBC10189894FF6FF7291420FD04109364A52F8211000F01F0301229A40114009B1012100E00021012900D102E0401E0028DFD100BF704710B5F9
:40E140000146002028290DD24A09294B53F8222001F01F040123A3401A400AB1012200E00022104610BD10B50020002113E0254A525C002A0EDD4A091D4B53F8222001F0D8
:40E180001F040123A3401A400AB1012200E0002202B9401C491C2829E9D310BD1C48007870471B4908707047282802D201210E4A115470470020002106E00D4A52F82120BC
:40E1C0000AB1012002E0491C0229F6D300BF704710B51049886F012176F074FA10BD0E480068704770C7090828380010B0000010B8000010C0000010082000105038001065
:40E20000F0380010480800200050006890390010C8000010300A0020CC000010424800687047424800687047414800687047414800687047404800687047404800687047A7
:40E240003F48006870473F48006870473E48006870473E48006870477CB5044600250020019000903A4801F0FCFE002847D001AA0021374800F083FC002840D06A460121B7
:40E28000334800F07CFC08B3019849F07DFFE8B1009849F079FFC8B1012C18D1019849F069FF0646009849F065FF864227DD019849F060FF0646009849F05CFF301A254919
:40E2C000884201DD012000E00020054617E0019849F050FF0646009849F04CFF86420EDA009849F047FF0646019849F043FF301A1849884201DD012000E000200546284636
:40E300007CBD70B5144C28231A46144920460BF060FF04461248206000BF2546114A1249284673F0A1FC70BDD0000010D4000010D8000010DC000010E0000010E40000103C
:40E34000E8000010EC000010F0000010F4000010E039001080841E0090390010A8550010F8D00F08008000083B3D09082DE9F04107460C460025012F02D0022F04D101E090
:40E38000C02602E0C42600E000BF00BF27B1012F2DD0022F49D12BE004F0010028B10121BA480078F4F70DFF04E00021B7480078F4F707FF04F0020028B10121B4480078BF
:40E3C000F4F7FFFE04E00021B1480078F4F7F9FE04F0040028B10121AE480078F4F7F1FE04E00021AB480078F4F7EBFE1EE000BF04F0010010B145F0030501E045F0010592
:40E4000004F0020010B145F00C0501E045F0040504F0040010B145F0300501E045F0100529463046F5F775FF00E000BF00BFBDE8F081024600210CE0974800EB0110007811
:40E44000904205D1944800EB0110407B00B102E0491C0B29F0D300BFC8B27047F8B5044600250B2C5FD2DFE804F006101517282C435153575C0089480DF0DBFB064641F2F0
